S00A000047572E737265637C
S214400000A55AA55A0100000000000000001040005C
S21440100000F0422021144400CD294500CF29450058
S214401010D1294500D3294500D529450000000000C8
S214401020000000000000000000000000D729450036
S2144010300B2A4500000000000D2A45000F2A4500F7
S21444010047573334342056302E322E352032303250
S214440110332E31312E362031323A30300A0D00003B
S20C4401803412AA5500000000E9
S214440200A55AA55A01000000000000000010440052
S2144402100000000000104400000000000000000041
S2144402200000000000000000000000000000000085
S2144402300000000000000000000000000000000075
S2144402400000000000000000000000000000000065
S2144402500000000000000000000000000000000055
S21444100000F0422021144400CD294500CF29450054
S214441010D1294500D3294500D529450000000000C4
S214441020000000000000000000000000D729450032
S2144410300B2A4500000000000D2A45000F2A4500F3
S214441040112A4500112A4500112A4500112A450057
S214441050112A4500112A4500112A4500112A450047
S214441060112A4500112A4500112A4500112A450037
S214441070112A4500112A4500112A4500112A450027
S214441400112A4500112A450000BF00BF00BF00BF97
S214441410FFF7FABF000000000000000000000000D4
S21444142072B64FF000004FF000014FF000024FF04C
S21444143000034FF000044FF000054FF000064FF055
S21444144000074F4801684FF0807201EA0201002904
S2144414501CD14C4801684FF0807241EA0201016099
S214441460494801684FF0010241EA020101604748D9
S21444147045F6F02101604AF20F5101604048016888
S2144414804FF0807201EA02010029F7D040484149F2
S2144414900160414801684FF00000814200D003E0FB
S2144414A03E4880F3088803E03D4880F3088822E0FD
S2144414B03C484CF2205101604DF6281101603A48F0
S2144414C03A4901600AE03A484CF2205101604DF630
S2144414D028110160374835490160FFE7364800283F
S2144414E009D03649364A521A013A04DD0020002310
S2144414F009C1083AFCDA3348002810D03249086853
S2144415004FF0010240EA020008603049304A521A5D
S214441510013A04DD0020002309C1083AFCDA2D48CC
S214441520002810D02C4908684FF0010240EA020017
S21444153008602A492A4A521A013A04DD0020002348
S21444154009C1083AFCDA274800684FF05A31884205
S214441550F9D0114801684FF00000814200D001E004
S21444156011F058FA11F082FA62B611F07DFA00F0E2
S2144415703BF800BFFEE700BFAFF30080AFF3008048
S21444158010C32D4030C32D4004C32D4000C02D4011
S21444159008ED00E0001043200400264000F04220FE
S2144415A0000043201000274000002740400000FF72
S2144415B010C0464000C046400100000000004020E5
S2144415C0004044200100000094EF00E000000020AA
S2144415D0000001200100000090EF00E00000000041
S2144415E000800000B02340202DE9F04F87B05A4CCD
S2144415F002F054FA594812F05BFF59494E20002530
S21444160023F006F957481AF0E3F857481AF004F955
S21444161002F0B7F94CF24453E05800F075FE02F07D
S214441620F3FB00F099FF00F075FF00F0F3FE4F491E
S21444163000201DF049FA4E4900201DF05BFA0021B7
S21444164008461DF001FB002144F6206208461DF0C2
S214441650B7FA2846013502F051FD062DF9D102F0BD
S2144416608DF94CF23853434D4FF47A7054F8038056
S214441670E75805F1040BE25854F803900592E258F3
S2144416800292E2580392E2580492E25854F803A0B5
S214441690E6582C46019202F038F908F0FBFB36482F
S2144416A002F064FA2A6806F57A739A4202D32E68E0
S2144416B008F0DFFB22680AF1C8039A4203D3D4F841
S2144416C000A008F0CFFB019B226864339A4203D300
S2144416D02368019308F0B3FB049B226832339A4292
S2144416E001D323680493039B226814339A4203D39A
S2144416F02368039302F096FF029B22680A339A42B9
S21444170003D32368029308F094F8226809F105038A
S2144417109A4203D3D4F8009008F075FB059B2268E0
S21444172002339A4203D32368059300F0CDFD226822
S2144417307B1C9A4200D32768DBF8002008F101039B
S2144417409A4203D3DBF8008008F068FB08F0A8FB55
S2144417500BF096FEA6E700BF74354120A86046000D
S214441760E8034020EC6D46001C6946007417402090
S21444177068174020ACFA41202C594600024B586862
S21444178000F00300704700BF00002640024600F009
S2144417903F00931010B583EA52035408534084EA3A
S2144417A0121483EA121384EAD2049B0184EA521484
S2144417B003F0400314F0010F43EA00030CBF8024F7
S2144417C00024234319B99A4218BFFF2010BD0129AB
S2144417D00CBF1846FF20F9E73C2A0CD07D2A0AD0D5
S2144417E0FE2A08D0BF2A06D092B20144814204D1D0
S2144417F0D043C0B270470022F7E710F8013B1A44C2
S21444180092B2FF2A84BFFF3A92B2EFE7F8B51D4B77
S2144418101D4D1C781D4E012C18D12F7857B91C49E4
S214441820384600F0AFFD0021204600F0ABFD2C709A
S2144418303770F8BD0021002000F0A4FD00212046AA
S21444184000F0A0FD00232B703370F2E733781C437E
S2144418500BD10F49012000F095FD0021204600F0F1
S21444186091FD01232C703370E3E70021012000F042
S21444187089FD0021002000F085FD002333702B7085
S214441880D7E700BF2E1E4020F1174020F017402017
S2144418900000C84208B5044B9889C0F3C7100CF042
S2144418A039FE024B186008BD90734020201E40202D
S2144418B0074B10B59C89C4F3C71420460CF02AFE87
S2144418C0044B1E2C18609EBF0322034B1A7010BD97
S2144418D090734020201E4020241E4020034B044A80
S2144418E05B6AC3F309231370704700BF90734020AC
S2144418F0F41D4020084B1B78013B022B0AD80023DA
S214441900064A00211370064A1160064A13700322E1
S214441910054B1A60704700BFEE1D4020ED1D402069
S2144419201C1E4020EC1D4020481D4020064B074A04
S2144419301B7BC3F3020103F00703013B1170012B29
S21444194001D8FFF7D7BF704790734020EE1D402064
S214441950FE28D4BF01300020704770B50022FF2314
S214441960064ED4B2551C8C4202D3D843C0B270BD86
S214441970025D53402A46F35CF3E700BF8A4D4600B7
S2144419800721013008B5FFF7E8FFC0B208BDB0F53F
S214441990447F38B5144617D1244D204695F8BC33B9
S2144419A0FF2B14BF01330023DBB285F8BC335370DE
S2144419B01F4A1370FFF7E4FF1E4BC0B285F8BD0301
S2144419C020701870012038BD402818D0B0F5547FD8
S2144419D0F8D1164D204695F8B833FF2B14BF013383
S2144419E00023DAB285F8B8236270134A1360FFF70F
S2144419F0C7FFC0B2114B85F8B903207014E00B4DF5
S214441A00204695F8B033FF2B14BF01330023DAB2D7
S214441A1085F8B02362700A4A1360FFF7B1FF094B9A
S214441A20C0B285F8B10320701860CBE790734020AD
S214441A304B1B40204A1B4020301B40202C1B402080
S214441A40401B40203C1B4020402838B5144616D145
S214441A50254D204695F8E833FF2B14BF0133002369
S214441A60DAB285F8E8236270204A1360FFF788FFED
S214441A701F4BC0B285F8E9032070186005E0B0F546
S214441A80547F04D0B0F5447F17D0012038BD164D9E
S214441A90204695F8F033FF2B14BF01330023DAB207
S214441AA085F8F0236270134A1360FFF769FFC0B2EB
S214441AB0114B85F8F1032070DFE70B4D204695F86F
S214441AC0F433FF2B14BF01330023DBB285F8F43321
S214441AD053700A4A1370FFF753FF094BC0B285F898
S214441AE0F50320701870D0E790734020D41A402035
S214441AF0D01A4020241B4020201B4020471B402057
S214441B00461B4020402838B5144617D1254D20465C
S214441B1095F8E833FF2B14BF01330023DAB285F877
S214441B2024246270204A1360FFF72AFF1F4BC0B27A
S214441B3085F8250420701860012038BDB0F5547F20
S214441B4018D0B0F5447FF7D1164D204695F830347A
S214441B50FF2B14BF01330023DBB285F830345370B7
S214441B60134A1370FFF70CFFC0B2124B85F83104CA
S214441B70207014E00B4D204695F82C34FF2B14BFF0
S214441B8001330023DBB285F82C3453700A4A1370B1
S214441B90FFF7F6FE094BC0B285F82D042070187086
S214441BA0CAE700BF90734020B01A4020AC1A4020C9
S214441BB0A41A4020A31A4020A01A40209F1A40206E
S214441BC0402838B5144616D1254D204695F8343469
S214441BD0FF2B14BF01330023DAB285F83424627035
S214441BE0204A1360FFF7CCFE1F4BC0B285F835047D
S214441BF02070186005E0B0F5547F04D0B0F5447FFB
S214441C0017D0012038BD164D204695F84034FF2B9A
S214441C1014BF01330023DAB285F840246270134AB5
S214441C201360FFF7ADFEC0B2114B85F84104207037
S214441C30DFE70B4D204695F83C34FF2B14BF0133A9
S214441C400023DBB285F83C3453700A4A1370FFF71E
S214441C5097FE094BC0B285F83D0420701870D0E753
S214441C6090734020981A4020941A4020841A4020AA
S214441C70801A40208B1A40208A1A4020502870B57B
S214441C800546144616D18C4A92F88C32FF2B14BF64
S214441C9001330023D9B282F88C12884A217013602B
S214441CA040F285339D4200F0DD80162D00F0F08032
S214441CB0012070BD642826D065283BD032284FD0FA
S214441CC0702863D0712877D0332800F08C806A2837
S214441CD000F09F80B0F5617FE2D1774D204695F8BD
S214441CE0C033FF2B14BF01330023DBB285F8C03367
S214441CF05370734A1370FFF743FEC0B2714B85F8B6
S214441D00C10320706DE06C4E204696F87833FF2B66
S214441D1014BF01330023DBB286F8783353706A4A23
S214441D201370FFF72DFE694BC0B286F87C03207013
S214441D301870B5E7604E204696F8E033FF2B14BF84
S214441D4001330023DBB286F8E0335370604A1370E5
S214441D50FFF716FEC0B25F4B86F8E4032070E7E751
S214441D60554E204696F89033FF2B14BF013300237C
S214441D70DBB286F890335370574A1370FFF700FE71
S214441D80C0B2564B86F891032070D1E74A4E20469F
S214441D9096F88433FF2B14BF01330023DBB286F856
S214441DA0843353704E4A1370FFF7EAFDC0B24D4B6E
S214441DB086F885032070BBE73F4D204695F8D4331C
S214441DC0FF2B14BF01330023DBB285F8D4335370A2
S214441DD0454A1370FFF7D4FD444BC0B285F8D5038B
S214441DE02070187064E7344D204695F8F833FF2B7E
S214441DF014BF01330023DBB285F8F83353703C4AF2
S214441E001370FFF7BDFDC0B23A4B85F8F903207056
S214441E10E7E7294D2046D5F8A833D5F8A823C3F3D9
S214441E20C733FF2B14BF01330023DBB263F3D63230
S214441E30C5F8A8236370D5F8A8332F4AC3F3C7332D
S214441E401360FFF79DFDB5F8AA33C0B22B4A60F382
S214441E50CE13A5F8AA332070B5F8AA33C3F3C71334
S214441E60136025E7144D2046254A95F81034FF2B79
S214441E7014BF01330023DBB285F81034637013704B
S214441E80FFF77EFDC0B21F4B85F811042070A8E70B
S214441E900949B1F87423C2F34313013303F00F0323
S214441EA063F34812A1F874236370B1F87433164A86
S214441EB0C3F34313D4E700BF907340207C1C4020F8
S214441EC0C71A4020C61A4020DA1D4020DB1D402099
S214441ED0D81D4020D91D4020561B4020551B40206D
S214441EE0F91A4020F81A4020191B4020181B40209D
S214441EF0DA1A4020D91A4020C8194020C419402074
S214441F00BD1A4020BC1A4020F81740200F28D4BFE2
S214441F1001300020704770B50022FF23074ED4B22C
S214441F20551C8C4205D3DB4383EA131303F00F009E
S214441F3070BD025D53402A46F35CF0E78A4E460085
S214441F400721013008B5FFF7E6FFC0B208BDB0F57B
S214441F50AE6F70B5054614461AD1C04D204695F866
S214441F60E9221309013363F3071203F00F0385F8DC
S214441F70E922BB4A1360FFF7E3FF95F8EA3260F3C1
S214441F80030300F00F0085F8EA32B64B18601EE0F3
S214441F90B0F5B06F1DD0B0F5B26F35D1AF4D204619
S214441FA095F8FA325A1C02F00F0262F3030385F8DE
S214441FB0FA32AD4B1A70FFF7C3FF95F8FA3200F0C9
S214441FC00F0060F3071385F8FA32A84B1870012007
S214441FD070BDA24D2046B5F8F022C2F383130133F8
S214441FE063F3891203F00F03A5F8F022A04A1360A6
S214441FF0FFF7A6FF95F8F13260F3850300F00F0073
S21444200085F8F1329B4BC1E740F29553984223D072
S21444201040F28553984259D0502800F09780512872
S21444202035D18E4D204695F8142302F00F03013324
S21444203063F3030203F00F0385F814238E4A1360F8
S214442040FFF77EFF95F8143360F3071300F00F0094
S21444205085F81433894B99E7804E204696F8FF223C
S214442060C2F38303013303F00F0363F3850286F858
S214442070FF22834A1370FFF763FF96F8003300F09D
S2144420800F0060F3030386F800337E4B1870602D10
S21444209077D0612D35D1714D204695F8242302F032
S2144420A00F03013363F3030203F00F0385F824237D
S2144420B0754A1360FFF744FF95F8243360F307131B
S2144420C000F00F0085F82433704B5FE7634E2046DC
S2144420D0D6F80423C2F38333013363F3913203F017
S2144420E00F03C6F804236A4A1360FFF729FF96F8DD
S2144420F0063360F3850300F00F0086F80633654B1D
S2144421001860132D58D0142D71D0152D00F08A80E8
S214442110162D7FF45CAF514D2046B5F87423C2F3B8
S2144421204313013363F3481203F00F03A5F87423F3
S214442130594A1360FFF704FF95F8753360F3440378
S21444214000F00F0085F87533544B1FE7434D204687
S21444215095F80C2302F00F03013363F3030203F0F4
S2144421600F0385F80C234E4A1360FFF7E9FE95F8F3
S2144421700C3360F3071300F00F0085F80C33494B1B
S21444218004E7364D204695F81C2302F00F0301332E
S21444219063F3030203F00F0385F81C23424A1360DB
S2144421A0FFF7CEFE95F81C3360F3071300F00F00DC
S2144421B085F81C333D4BE9E6284D2046B5F82E23DA
S2144421C0C2F38313013363F3891203F00F03A5F8B4
S2144421D02E23374A1360FFF7B3FE95F82F3360F388
S2144421E0850300F00F0085F82F33324BCEE61B4DA7
S2144421F0204695F83323C2F34303013363F3440282
S21444220003F00F0385F833232B4A1360FFF798FE39
S21444221095F8343360F3030300F00F0085F8343345
S214442220264BB3E60D4D204695F83E2302F00F03A9
S214442230013363F3030203F00F0385F83E23204A79
S2144422401360FFF77DFE95F83E3360F3071300F006
S2144422500F0085F83E331B4B98E600BF9073402032
S214442260E0194020DC194020891740208817402078
S2144422709C18402098184020E81B4020E41B40202F
S2144422808B1740208A174020C81B4020C41B402080
S214442290001D4020FC1C4020F8174020F417402026
S2144422A0F81B4020F41B4020D81B4020D41B402061
S2144422B0A01B40209C1B4020801B40207C1B4020B1
S2144422C0681B4020641B402007F0B2BF09F0BAB92F
S2144422D010B5084C09F048F8002001F079FA20803F
S2144422E0012001F075FA044B22881880034B1A80AB
S2144422F010BD00BF2A1E4020281E40201A1B402026
S2144423007047704770477047002110B5044608462A
S21444231015F088FA0121002015F084FA02210020E5
S21444232015F080FA0321002015F07CFA002015F001
S21444233075F90E49002015F087F80D4BA2B200201F
S214442340197815F0BFF90B49002015F031FD0A49FC
S214442350002015F02DFD0949002015F029FD0849F7
S2144423600020BDE8104015F023BD00BF646546005C
S2144423709C654600EC664600CC664600AC66460065
S2144423808C664600F8B50D4606461F4928461F4F3C
S2144423900CF0CAFA044670B14CF24453F85806F5A9
S2144423A04553123307EB83077D60032E2BD8DFE8B3
S2144423B006F01A212427002128460CF0ABFA80B9EF
S2144423C04CF24453F8580CF0A5F829460CF0FAF8A9
S2144423D00BF04AFC00220E4B0BF0C8FD0BF074FFCA
S2144423E0DDE72046DBE782B200210020BDE8F84066
S2144423F015F028BF82B20121F7E782B20221F4E742
S21444240082B20321F1E7F8BD0000C842743541208A
S2144424100000594008B503481AF0CCFB024B18702C
S21444242008BD00BFE47046007C464020F7B5012353
S214442430104C114D6370A21CEB68A91C0F48023562
S214442440009335F8023C1AF057FA00222073A01C79
S2144424506178134615F8017B013310F8016BDBB243
S214442460B7421CBF012200210A2BF3D102B161708E
S21444247003B0F0BD7C464020501E4020F870460015
S2144424804B7C062B0AD10122054B1A74CA7B1A2AA6
S21444249004D1032203F111011AF06EBD704700BF48
S2144424A0501E40204B7C062B0AD10122054B1A7441
S2144424B0CA7B2A2A04D1032203F111011AF05CBD17
S2144424C0704700BF501E40201FB500231A21044603
S2144424D0039301238DF807301AF094FE0B4B0393B5
S2144424E00B4B1A7C002AFCD01B7C63B102A9204605
S2144424F01AF08CFD8DF80700039B5A1E039213B105
S2144425009DF80730F1E704B010BD00BF006A18001C
S214442510501E402008B5A12019F0A0F900220A490F
S214442520A12019F09AF9094B094902220120C3F85F
S214442530F413C3F8982DC3F8F813C3F8902D05493F
S214442540BDE8084019F08ABE53C64500000029403D
S214442550040028005870460008B5A22019F07EF9F9
S21444256000220B49A22019F078F90A4B0A4A0121A5
S2144425700020C3F8E023C3F8AC1DC3F8E4230222CA
S2144425800649C3F8A42DBDE8084019F0A7BB00BF10
S21444259059C6450000002940020028007C704600C9
S2144425A010B50822174901204FF4803419F012FF61
S2144425B0012308221449002019F07CFC0021084617
S2144425C019F0C6FD022801D1013CF7D14FF48034FE
S2144425D00021012019F008FF022801D1013CF7D15F
S2144425E0094A0823A2F1080012F8011B013B10F81F
S2144425F0014BA14204BF013102F8011C13F0FF0352
S214442600F2D110BD641E40206C1E402082B0019062
S214442610019B5A1E0192002BFAD102B07047044B1C
S2144426204FF400224FF4FA70C3F8C022FFF7EEBF0F
S21444263000002940044B4FF420124FF4FA70C3F8BC
S214442640C022FFF7E3BF00BF000029402DE9F04158
S21444265004460D46104600293ED1DFF890805026A9
S2144426600B46C1B2564308F110072846BA19B0447F
S21444267016F0F8FD1C484FF4FB534FF4FB62D8F8B1
S2144426801410083603FB04033744D3F8FC3802FB23
S214442690043203F17A0602F5107C02F5427240F8E1
S2144426A02C1098F8581040F82210FB2212FB0462B3
S2144426B000EB4212A94211D84FF4FB520133642175
S2144426C002FB0404B3FBF1F201FB1233C4F8FC38FA
S2144426D004F5215401232360BDE8F08117F8016B0B
S2144426E0013502F8016BE5E7743541207C4640200D
S2144426F02DE9F04104460D46104600293ED1DFF848
S214442700908050260B46C1B2564308F5F267012026
S214442710BA19B04416F0A6FD1C484FF4FB534FF4C8
S214442720FB62D8F89417083603FB04033744D3F8FF
S214442730FC3802FB043203F17A0602F5107C02F5FB
S214442740427240F82C1098F8D81740F82210FB2212
S21444275012FB046200EB4212A94211D84FF4FB521A
S2144427600133642102FB0404B3FBF1F201FB123390
S214442770C4F8FC3804F5215401232360BDE8F081F5
S21444278017F8016B013502F8016BE5E77435412013
S2144427907C4640202DE9F04104460D46104600296B
S2144427A03ED1DFF8908050260B46C1B2564308F51A
S2144427B071670220BA19B04416F054FD1C484FF411
S2144427C0FB534FF4FB62D8F8141F083603FB04038C
S2144427D03744D3F8FC3802FB043203F17A0602F598
S2144427E0107C02F5427240F82C1098F8581F40F8B6
S2144427F02210FB2212FB046200EB4212A94211D8BB
S2144428004FF4FB520133642102FB0404B3FBF1F2A0
S21444281001FB1233C4F8FC3804F521540123236029
S214442820BDE8F08117F8016B013502F8016BE5E766
S214442830743541207C4640202DE9F04104460D463F
S214442840104600293ED1DFF8908050260B46C1B290
S214442850564308F5B3670320BA19B04416F002FD90
S2144428601C484FF4FB534FF4FB62D8F89C150836CB
S21444287003FB04033744D3F8FC3802FB043203F169
S2144428807A0602F5107C02F5427240F82C1098F84D
S214442890E01540F82210FB2212FB046200EB4212C1
S2144428A0A94211D84FF4FB520133642102FB0404BD
S2144428B0B3FBF1F201FB1233C4F8FC3804F521549F
S2144428C001232360BDE8F08117F8016B013502F857
S2144428D0016BE5E774354120745740202DE9F041FB
S2144428E004460D46104600293ED1DFF89080502617
S2144428F00B46C1B2564308F618570420BA19B044DA
S21444290016F0B0FC1C484FF4FB534FF4FB62D8F867
S2144429101C1D083603FB04033744D3F8FC3802FB7B
S214442920043203F17A0602F5107C02F5427240F84E
S2144429302C1098F8601D40F82210FB2212FB04620B
S21444294000EB4212A94211D84FF4FB5201336421E2
S21444295002FB0404B3FBF1F201FB1233C4F8FC3867
S21444296004F5215401232360BDE8F08117F8016B78
S214442970013502F8016BE5E7743541207457402071
S2144429802DE9F04104460D46104600293ED1DFF8B5
S214442990908050260B46C1B2564308F5687705200A
S2144429A0BA19B04416F05EFC1C484FF4FB534FF47F
S2144429B0FB62D8F8A413083603FB04033744D3F861
S2144429C0FC3802FB043203F17A0602F5107C02F569
S2144429D0427240F82C1098F8E81340F82210FB2274
S2144429E012FB046200EB4212A94211D84FF4FB5288
S2144429F00133642102FB0404B3FBF1F201FB1233FE
S214442A00C4F8FC3804F5215401232360BDE8F08162
S214442A1017F8016B013502F8016BE5E77435412080
S214442A206C6840204FF4FB52054B02FB0033D3F84E
S214442A30F808D3F8FC38C31A58425841704700BFC8
S214442A40743541202DE9F74FD04D0021D04E4FF438
S214442A50FB692C4641F6987837464FF0640A084698
S214442A60FFF7E0FF58BBD6F8F83809FB013202F509
S214442A70427257F822C008FB014200924FF4FB52C0
S214442A804A4302EB43123A44019200F1010EC0B2AB
S214442A90844500F2A88009FB0132013385F820C042
S214442AA002F5107257F822206A624FF0010285F848
S214442AB02120B3FBFAF20AFB1233C6F8F838013188
S214442AC0454406F5FB560629C9D194F82130012B16
S214442AD019D1002384F82130636AB3F5407F00F0AF
S214442AE0D68000F29F80B3F5BA7F00F0D98000F21A
S214442AF08B80412B00F0D1807FD8202B00F0C480FF
S214442B00402B00F0C78041F6B973E25C012A0FD12E
S214442B100022E25441F6BC73E358932B00F0D8806D
S214442B2000F2C980912B00F0CD80922B00F0CD802E
S214442B3043F65173E25C012A14D10022E25443F670
S214442B405473E358962B00F0EB8000F2CC80822B33
S214442B5000F0E38000F2BF80722B00F0E780732B16
S214442B6000F0E78045F6E963E25C012A14D10022CE
S214442B70E25445F6EC63E3589B2B00F0FB8000F2EE
S214442B80E6808D2B00F00B8100F2D980722B00F08A
S214442B90FA80732B00F0008147F68163E25C012AD9
S214442BA00BD10022E25447F68463E358722B00F0BC
S214442BB0FC80732B01D103F00DF849F61963E25CEF
S214442BC0012A40F0FA800022E25449F61C63E35896
S214442BD0722B00F0ED80732B40F0EF8003B0BDE81D
S214442BE0F04F03F037B8019A02EB000B009A9BF8BB
S214442BF040BF02F800B0704647E740F25512934291
S214442C0081D102F049F87EE7B3F5BE7F4BD040F25F
S214442C10212293424AD0B3F5BC7F7FF474AF01F0CF
S214442C2051FF70E740F2855293422AD011D8B3F54B
S214442C30AE6F1DD0B3F5B06F1DD040F20132934253
S214442C407FF461AF01F096FE524A13880133138035
S214442C5059E740F29552934210D040F2777293422D
S214442C6026D0B3F5B26F7FF44EAF01F08FFD4AE73E
S214442C7001F0E9FC47E701F03DFD44E701F0B6FD0D
S214442C8041E701F0CBFD3EE701F0E6FD3BE701F00E
S214442C9021FE38E701F07AFE35E701F0B7FE32E769
S214442CA001F0D2FE2FE701F043FF2CE701F074FF5A
S214442CB001F09AFE27E7B3F5A87F7FF439AF02F018
S214442CC091F835E702F013F832E702F041F82FE7BF
S214442CD002F06AF82CE78C2B25D0922B7FF442AF77
S214442CE002F00AFA3EE7AA2B26D007D89A2B0ED033
S214442CF0A02B7FF437AF02F06DF933E7C82B09D029
S214442D00B3F5F36F7FF42EAF02F0EEFA2AE702F043
S214442D10BFF827E702F020F924E702F0C3F921E7D9
S214442D2002F07AFA1EE702F0F3FA1BE702F058FBC9
S214442D3018E702F0A7FB15E702F0E2FB12E7932B35
S214442D4030D0972B7FF428AF02F0EEFD24E7C92B52
S214442D5013D007D8A12B13D0AA2B7FF41DAF02F0B3
S214442D608FFD19E740F2997293427FF415AF02F053
S214442D701DFF11E702F018FC0EE702F079FC0BE7A2
S214442D8002F0B4FC08E702F0EBFC05E7D8774020F5
S214442D90743541200A1E402002F034FDFCE602F061
S214442DA02BFEF9E602F090FEF6E602F02FFF04E76B
S214442DB003B0BDE8F04F02F069BF03B0BDE8F08F42
S214442DC0EA4B0021DFF8C8C31A68586A02F070421A
S214442DD000EA0C002DE9F04F1A6000261A890027F5
S214442DE0586202F47042986ADFF8A8B31A8100F079
S214442DF07F40DA68986202F00042DD485960DA6043
S214442E001A8AD86202EA0B021863DA481A82002247
S214442E10586393F83800596162F303009961D961A5
S214442E2083F8380093F83C0083F8202020F00F0005
S214442E301964D96483F83C0093F84400DFF858A337
S214442E4000F0E000DFF85493DFF854E362F34510F3
S214442E50DFF8508383F84400C74898644FF04740EF
S214442E601865C6485865C648C3E916225C6F586656
S214442E70C44819662040D3F8DC4099665867D3F8AE
S214442E80A800A3F86C2000EA0A0083F8BC20C3F824
S214442E90C010C3F8A800D3F8AC00C3F8C81000F0BC
S214442EA00040C3F8CC1083F8D020C3F8AC00D3F865
S214442EB0B000C3F8E490C00DC005C3F8B000D3F822
S214442EC0C40000F07F40C3F8C40093F8D40020F058
S214442ED00F0083F8D400D3F8D40020F4FF3020F455
S214442EE0F870C3F8D400D3F8D80000F07C40C3F898
S214442EF0D800A5480440C3F8DC40D3F8E04004407A
S214442F00C3F8E04093F8E84062F3000483F8E840EE
S214442F1093F8F440C3F8EC1024F00704C3F8F01018
S214442F20A3F8002183F8F44093F80841C3F8041149
S214442F3062F30004C3F80C11C3F8141183F8084173
S214442F4093F81041C3F81C1162F30004A3F824213B
S214442F50C3F8281183F8104193F81841C3F82C118C
S214442F6062F30004A3F83C21C3F8401183F81841E7
S214442F7093F82041C3F8481162F30004C3F834E1DF
S214442F8083F82041D3F8304104F00044C3F830417C
S214442F9093F8384124F0030483F83841B3F83841B1
S214442FA024F47F6424F00C04A3F8384193F8444195
S214442FB062F3010483F8444193F84C41D3F8A45196
S214442FC062F30104C3F8501105EA0805C3F8581122
S214442FD083F84C4193F8544145F48035C3F8801146
S214442FE062F30104C3F88811A3F8902183F854418E
S214442FF093F85C41C3F8941162F30104C3F89C113E
S21444300083F85C41D3F8704104F04044C3E95C4221
S21444301093F8784124F0030483F87841D3F87C414C
S21444302004F07F44C3F87C4193F8844162F300047F
S21444303083F8844193F88C4124F07F0483F88C41D0
S21444304093F8984162F3000483F8984193F8A041BA
S21444305062F30004C3E95A2283F8A041C3E95867DF
S214443060C3F8A45193F8BC41D3F8B45162F30004B6
S214443070C3F8A8110540C3F8AC1183F8BC4193F8D3
S214443080C841C3F8B45124F00704D3F8CC51C3F86C
S214443090B01183F8C84105F0604593F8DC41C3F8A5
S2144430A0CC5162F30004D3F8E851C3F8C01183F856
S2144430B0DC4105F07F4593F8E441C3F8C41162F35C
S2144430C0000483F8D021A3F8D42183F8E44193F88C
S2144430D0F041C3F8D81162F30004C3F8E011C3F812
S2144430E0E85183F8F04193F8F841C3F8EC1124F022
S2144430F07F04C3F8F411A3F8FC21C3F80012C3F804
S214443100B89183F8F84193F80442C3F8081262F37E
S2144431100004C3F81412C3F8181283F8044293F850
S2144431200C42C3F81C1262F30004A3F82022C3F82E
S214443130241283F80C42D3F81042C3F82C1204EA43
S2144431400804C3F83412C3F83C1244F48034C3F879
S21444315054E20E4DC3F8104293F8284262F3010439
S21444316083F8284293F830421EE000BF9073402014
S21444317014AE23C10AD723C3000048C2000048C384
S214443180004026C400F807F80000C0FF0000FEFF19
S2144431900000FCFF00C0FFFF0000F0FF33336FC1A8
S2144431A0CDCC4CBD0000F8FF62F3010483F83042F6
S2144431B093F8384262F3010483F8384293F8404265
S2144431C062F3010483F84042D3F8444204F0404496
S2144431D0C3E9914293F84C4224F0030483F84C42EA
S2144431E0D3F8504204F06044C3F8504293F858422F
S2144431F024F03F0483F8584293F87442C3F870129C
S21444320062F30304C3F87812C3F87C1283F874425A
S21444321093F88042C3F8841262F30304B3F8A81206
S214443220C3F8882283F88042B04CA3F88C2221400D
S214443230C3F8902283F89422A3F8A812D3F8A812CD
S214443240C3F8982221F07F7183F89C22C3F8A02209
S21444325021F47F3183F8A422C3F8BC22C3F8A81211
S214443260D3F8AC1283F8C4220140C3F8AC12D3F8A6
S214443270B41201F00041C3E9AD12D3F8C01201F014
S2144432807F41C3F8C012D3F8C8122940C3E99867EF
S214443290C3E9B212D3F8E012C3F8DC2201EA0A0109
S2144432A083F8E822C3F8F422C3F8E012B3F8E41231
S2144432B083F80C230C40C3F8102383F81423A3F894
S2144432C0E4428B4CD3F8E412C3F818230C40D3F8EA
S2144432D0EC1283F81C2301F00041C3F8E442C3F81F
S2144432E02023C3F8EC12B3F8F01283F8242301EA3F
S2144432F00B0BD3F8F812C3F8282301F07F41A3F848
S214443300F0B27C4CC3F8F812D3F8FC1201EA0C0174
S214443310C3F8FC12D3F804130140C3E9C112D3F82E
S2144433202C130840C3E9B522C3F82C03D3F8301352
S214443330A3F8AC2301F06041C3F8B023C3F83013BC
S21444334093F8341362F3030183F83413D3F87813F1
S21444335001F07E41C3F87813D3F87C1301F00041A2
S214443360C3F87C1393F8801321F00F0183F880137D
S214443370D3F8841301F07841C3F88413D3F8881340
S21444338001F07F41C3F88813B3F88C132140A3F8A7
S2144433908C13D3F890132940C3F89013D3F8A8138A
S2144433A001F00041C3F8A81393F8B41362F3000184
S2144433B083F8B413D3F8B81301F07F41C3F8B813B5
S2144433C0D3F8BC1301EA0C01C3F8BC13D3F8C013FA
S2144433D001F04041C3F8C013D3F8C41301F0784158
S2144433E0C3E9E667C3F8C41393F8D013D3F8C80305
S2144433F062F30001C3F81C2400F0784083F8D0132D
S214443400B3F8DC132140A3F8DC13D3F8E01301F03F
S2144434107E41C3F8E013D3F8E4132940C3E9F91214
S21444342093F8EC1362F3000183F8EC13D3F8F0132B
S21444343001F07F41C3F8F013D3F8F41301EA0C010A
S214443440C3F8F413D3F8F8130D4003F58061C1E9CB
S2144434500067D3F81014C3F8F85301F04041C3E9A9
S214443460F202C3F81014D3F8D403D3F8141400F0BB
S214443470784001F07841C3F8D403C3F81414D3F861
S214443480D803D3F8181400F07F4001F07841C3F80D
S214443490D803C3F8181493F82014C3F8242462F30A
S2144434A00001C3F8342483F8201493F8281462F3F4
S2144434B0000183F82814D3F82C1401F07F41C3F894
S2144434C02C1493F8321421F0030183F8321493F841
S2144434D0381462F3000193F83E2422F0030283F882
S2144434E0381483F83E24BDE8F08F00BF00FCFFFF8D
S2144434F0FF0300F000E0FFFF41F6987308490022FE
S21444350058430B182830DA64084483F848202023AC
S214443510013B00F8012B13F0FF03F9D1704700BFBD
S214443520D877402041F6987310B558430B4C41F673
S21444353092732218D35A28225A4300231118503023
S214443540104421441A46204481F870304B670133B6
S21444355000F8012BDBB2202BF9D110BDD8774020E0
S2144435602DE9F8439946234B0546884603EB00135A
S2144435709B6A402B31D820494FF4FB5303FB00137E
S21444358042F644015B5843B341F698761B4C0027F9
S2144435904FF0280C06FB00F3E11801F5FC511031FE
S2144435A0F8B248451BD328467543FFF7A5FF41F6B6
S2144435B09071601928260122435A06FB035513448A
S2144435C02C4484F87120C4F8748084F87090C8241D
S2144435D0B3FBF4F204FB12334352BDE8F883088885
S2144435E012F807E00CFB003020443844013780F8DA
S2144435F050E0D5E7501E402074354120D87740200F
S21444360041F6987241F692732DE9F347444D02FB16
S21444361000F10446434F6A18D35A282202FB031289
S2144436202A4492F87020082A2FD807EB0012082163
S214443630916241F698764FF0280941F6947A2046EE
S214443640664309FB03F206F1500305EB060891199D
S2144436501344354A29442B4402EB041200934B6F1F
S21444366018F80A1015F086FD18F80A300D210133B3
S214443670B3FBF1F201FB123308F80A308246E0B19C
S21444368002282FD002B0BDE8F087102A03D807EBF3
S21444369000121021CCE7182A03D807EB0012182191
S2144436A0C6E7202A03D807EB00122021C0E7402AA9
S2144436B0BFD807EB00124021BAE72046FFF732FF97
S2144436C041F69271C82038F8013009FB036601338D
S2144436D0B3FBF0F2354400FB123385F871A028F8AA
S2144436E00130CFE72046FFF71DFF41F692710022D6
S2144436F0C82038F8013009FB03660133354485F8A1
S2144437007120B3FBF0F200FB123328F80130D7E9FE
S2144437102232013342F10002C7E92232B2E700BF47
S214443720D8774020501E4020741E4020F8B5002410
S2144437300A4D41F698760A4F06FB04F22821E0B279
S214443740D35B01FB03232B4493F87130012B01D147
S214443750FFF756FF0134062CEED1F8BDD87740204B
S2144437606A97402008B50B21034820F099FF034B85
S21444377083F8200B08BD00BF021729406C68402020
S21444378001290A4628BF0122072819D8DFE800F095
S21444379004070B0D1012141600210A4801E00A21F2
S2144437A0094820F044BF0C21F7E702210748F8E710
S2144437B00D21F2E70E21F0E70F21EEE70021F5E7B1
S2144437C0704700BF021729401017294000172940A8
S2144437D007281AD8DFE800F004070B0E1013151755
S2144437E008210B4801E00B210A4820F059BF01216B
S2144437F00948FAE70B21F4E704210848F5E70521D0
S214443800FBE70821F9E70A21F7E7FF20704700BFE6
S2144438100617294002172940121729400417294041
S21444382001284FF002010CBF0022012210B50446C5
S214443830034820F0FCFE034A4CF24053D45010BDDB
S214443840081729407435412005281DD8DFE800F0C4
S21444385003080C1014180D4A4CF27453D05A70478F
S2144438600A4A4CF27653F9E7084A4CF27853F5E79D
S214443870064A4CF27A53F1E7044A4CF27C53EDE79D
S214443880024A4CF27E53E9E7FF20704774354120E4
S21444389008B5062100200FF04AFC024A4CF2745345
S2144438A0D05208BD7435412010B5022101200FF0D6
S2144438B03EFC064C4CF276532B21E05201200FF08E
S2144438C036FC4CF27E53E05210BD00BF74354120A6
S2144438D010B5032102200FF02AFC094C4CF2785311
S2144438E00421E05202200FF022FC4CF27A530521C8
S2144438F0E05202200FF01BFC4CF27C53E05210BD09
S2144439007435412000210FF0FFBA084A4CF2385370
S21444391082B00749D35800930B68009A9B1A0193C8
S214443920019B8342F8D902B0704700BF74354120EA
S214443930ACFA412038B50F4D0F4C95F890305BB932
S21444394001234CF23C5285F89030A3580133A350DF
S214443950BDE8384006F062BA08F04AFB4CF23C52E6
S214443960002385F89030A3580133A3504CF23852C4
S214443970EBE700BF501E4020743541200020FFF77F
S2144439804FBF10B58D20244C17F068FF0022234902
S2144439908D2017F062FF8F2017F060FF0022204929
S2144439A08F2017F05AFF972017F058FF00221D4922
S2144439B0972017F052FF9A2017F050FF00221A491A
S2144439C09A2017F04AFF194900201AF08FFA18492E
S2144439D002201AF08BFA17490A201AF087FA164979
S2144439E00D201AF083FA2146012200201AF000FD29
S2144439F004F59671012202201AF0FAFC04F26C5186
S214443A0001220A201AF0F4FC04F28C5101220D2003
S214443A10BDE810401AF0ECBC80384120F9E8450077
S214443A20FFE8450005E945000BE94500E47146001A
S214443A30B87146008C7146006071460010B48AB96D
S214443A400949D1F86C3891F8B848CA18013301F6D8
S214443A50B801DBB282F8584610BC012241F84C3C0F
S214443A601AF016BE10BC70477435412010B48AB99B
S214443A700949D1F8743891F8D848CA18013301F680
S214443A80D801DBB282F8584710BC012241F8643CA6
S214443A901AF0FEBD10BC704774354120194B012105
S214443AA042F644000022195044F2A470195046F2DB
S214443AB00470195048F2646019504AF2C4501950C0
S214443AC04CF22450195042F648015A5044F2A87118
S214443AD05A5046F208715A5048F268615A504AF2AF
S214443AE0C8515A504CF22851C3E9C1225A504CF29C
S214443AF048524CF2503199504CF244524FF448617B
S214443B00995070477435412010B5064B4FF4FB541A
S214443B1004FB003042F64803C15042F64C03C25000
S214443B2010BD00BF74354120094BD3E9C1218A42F8
S214443B300BD01A4492F8042202700020D3F80423CF
S214443B400132D2B2C3F8042370470120704700BF45
S214443B507435412007B501220DF107018DF80700A1
S214443B6000201AF099FA03B05DF804FB0FB470B560
S214443B70C2B0002446AA02AE52F8041B3046019254
S214443B800CF016FE304609F0ADFEC5B2E3B29D42D7
S214443B9004D842B0BDE8704004B07047305D01348C
S214443BA0FFF7D8FFF2E708B58E2017F057FE9620A9
S214443BB017F054FE0748FFF7D9FF0749002019F0CD
S214443BC015F90120054919F011F90548BDE80840E2
S214443BD0FFF7CCBF80574600347146000871460054
S214443BE0885746000B2938B5044614D142F6440398
S214443BF00E4D00220E48EA50FFF7B8FF42F648033F
S214443C00EB581BB142F64C02A85898472046BDE8EC
S214443C10384016F025B8074B1A6832B100220648D9
S214443C201A60BDE83840FFF7A1BF38BD743541205F
S214443C308E574600B45D4120AA5746000B2938B536
S214443C4005460E4C13D144F2A47300220C48E250AD
S214443C50FFF78CFF44F2A873E3581BB144F2AC72EE
S214443C60A05898472846BDE8384015F0F9BF44F2B6
S214443C70A073E2580AB10022E25038BD74354120A0
S214443C80C95746000B2938B5044614D146F2047386
S214443C900E4D00220E48EA50FFF768FF46F20873BE
S214443CA0EB581BB146F20C72A85898472046BDE81C
S214443CB0384015F0D5BF074B1A6832B10022064883
S214443CC01A60BDE83840FFF751BF38BD743541200F
S214443CD0E5574600749C4120015846000B2938B5E8
S214443CE004464FF4FB55134815D105FB040542F62C
S214443CF0440300221048EA50FFF738FF42F64803D0
S214443D00EB581BB142F64C02A85898472046BDE8EB
S214443D10384015F0A5BF05FB040404F52154236878
S214443D2033B1002305482360BDE83840FFF71EBF83
S214443D3038BD00BF743541201F5846003B584600E6
S214443D400B2938B504464FF4FB55134815D105FBEB
S214443D50040542F6440300221048EA50FFF706FFE3
S214443D6042F64803EB581BB142F64C02A858984713
S214443D702046BDE8384015F073BF05FB040404F53F
S214443D802154236833B1002305482360BDE83840F6
S214443D90FFF7ECBE38BD00BF743541205A58460084
S214443DA0765846000B2938B504464FF4FB5513485D
S214443DB015D105FB040542F6440300221048EA5098
S214443DC0FFF7D4FE42F64803EB581BB142F64C02CA
S214443DD0A85898472046BDE8384015F041BF05FB33
S214443DE0040404F52154236833B1002305482360B2
S214443DF0BDE83840FFF7BABE38BD00BF7435412031
S214443E0095584600B158460038B50A243C4D2946D4
S214443E1000200FF09DFD38B1013C14F0FF04F6D1AC
S214443E2021463848FFF7A2FE0A24374D294601208A
S214443E300FF08EFD38B1013C14F0FF04F6D1012199
S214443E403048FFF793FE0A24304D294602200FF0EF
S214443E507FFD38B1013C14F0FF04F6D10221294815
S214443E60FFF784FE00222A49B4200A2417F0F5FC02
S214443E7000222849B52017F0F0FC00222649B62037
S214443E8017F0EBFCB42017F0E9FCB52017F0E6FC7D
S214443E90B62017F0E3FC00200FF0F0F938B1013CEF
S214443EA014F0FF04F7D121461C48FFF75FFE0A24AE
S214443EB001200FF0E3F938B1013C14F0FF04F7D1C8
S214443EC001211648FFF752FE0A2402200FF0D6F9C5
S214443ED038B1013C14F0FF04F7D102210F48FFF734
S214443EE045FE012100200FF04BFA012108460FF051
S214443EF047FA01210220BDE838400FF041BA00BF1E
S214443F00D0644600EC584600746446001864460084
S214443F102D3F4500333F4500393F4500D0584600C5
S214443F2038B51C4C0546206804302044FFF7FCFD99
S214443F30012801D1012038BD2368E21810790A28E7
S214443F4010D00D280ED0082815D123B1013B1248B5
S214443F502360FFF70BFE2368AB42EBD325440020D7
S214443F60E87006E00D48FFF701FE2368002023446E
S214443F7018712060DFE7A0F120035E2BEBD8FFF733
S214443F80E9FD2368E11801330A792360303A81F861
S214443F900421E0E774354120015946001059460093
S214443FA010B58020FFF7BCFF90B90A4C23797BB14B
S214443FB00949201D09F08CFC20B90848BDE810408A
S214443FC0FFF7D4BD211D0648BDE81040FFF7CEBD1F
S214443FD010BD00BF74354120055946000B594600B4
S214443FE0135946002DE9F04F082389B00024924621
S214443FF03B4A054689464FF064081068EDB251685E
S21444400002AF012622468DF810408DF81C40DFF89A
S214444010E8B0CDE905346B4403C35146484620F026
S21444402006FB04AA214640F255532846CDF80480A0
S21444403000978DF81C608DF81040059415F0FEFC32
S214444040284B04AA2146284602934FF607738DF858
S2144440501060ADF80C300623CDE9007805935B4636
S21444406015F0ECFC204A0623214602924FF6FF72D6
S214444070059328465B46ADF80C2004AA8DF81060DC
S214444080CDE9007815F0DAFC184A06232146029258
S214444090284604AA05935B46ADF80C408DF810609C
S2144440A0CDE9007815F0CAFC114B124A2146284641
S2144440B08DF81060CDE90232082304AA05935B46C6
S2144440C0CDE9007815F0BAFC0A20FFF71EFC32460C
S2144440D05146484620F0ABFA09B0BDE8F08F00BF21
S2144440E08C4F46001000500010019FFF1002C00085
S2144440F07102030405060708F100DA182DE9F041B9
S2144441000446002855D16D2017F0A8FB2246C04926
S2144441106D2017F0A2FB6E2017F0A0FB2246BD4987
S2144441206E2017F09AFB01220821BB4820F07FFA44
S21444413001220521B84820F07AFAB84AB849204600
S21444414014F00EFF0121204615F0CCFE22460D2128
S214444150204615F023FD204615F0A2FE2346B14A1C
S2144441600D21204615F03AF82346AF4A0D21204645
S21444417015F078F8FEF724FE2046FFF7BDF9AB4B62
S214444180012242F644015A5003F521531A6041F67F
S21444419098700023A64A4443A648A35004441A46AB
S2144441A0013384F871202834C82BF9D10020BDE8A7
S2144441B0F081012846D0022840F0898074209E4F22
S2144441C017F04CFB00229D49742017F046FB7520DF
S2144441D017F044FB00229A49752017F03EFB012253
S2144441E00421984820F023FA01220621964820F01C
S2144441F01EFA0025954A20469549DFF8B88214F001
S214444200AFFE204615F04CFE05F10D0658F8353045
S214444210904A0220F6B223F060430135314614F04A
S214444220DDFF3A46002331460220503715F01AF88F
S2144442300B2DE9D17D4B012246F204715A5003F509
S214444240CE43A3E77120844F17F008FB002283492E
S214444250712017F002FB722017F000FB0022804901
S214444260722017F0FAFA22460721774820F0DFF941
S21444427022460221734820F0DAF90025794A20467E
S2144442807949DFF8348214F06BFE204615F008FEB8
S21444429005F10D0658F83530744A0120F6B223F07D
S2144442A060430135314614F099FF3A4600233146BF
S2144442B00120503714F0D6FF042DE9D144F2A471FE
S2144442C05A4B01225A5044F2A0715A505FE70328D1
S2144442D059D0042800F0F48005287FF458AF7B209A
S2144442E0634D17F0BBFA002262497B2017F0B5FAFB
S2144442F07C2017F0B3FA00225F497C2017F0ADFA11
S21444430001220E21504820F092F901225B481146C2
S21444431020F08DF95A4A5B49204614F021FE204687
S21444432015F0BEFD012255492046FFF75BFE564A6E
S2144443305449204614F014FE204615F0B1FD2B686F
S214444340524A0D2123F06043204614F047FF0023D1
S2144443504F4A0D21204614F085FFAB684B4A0E2188
S21444436023F06043204614F039FF0023494A0E21C7
S214444370204614F077FF4CF224512C4B01225A501D
S2144443804CF22051A1E77720434F17F067FA0022FA
S2144443904249772017F061FA782017F05FFA002236
S2144443A03F49782017F059FA012200213D4820F071
S2144443B03EF901223B4800251146DFF8008120F0F3
S2144443C036F9394A3949204614F0CAFD204615F0D4
S2144443D067FD05F10D0658F83530354A0320F6B228
S2144443E023F060430135314614F0F8FE3A46002384
S2144443F031460320503714F035FF0A2DE9D148F2F0
S21444440064610A4B01225A5048F260615DE700BF7E
S2144444105DB6450063B6450008172940C4684600A3
S21444442048404020E41E40209C4A402074354120A9
S21444443068974020D87740209C594020A5B6450030
S214444440ABB645000E1729400C17294014684600A1
S214444450F8364020041F40201C52402087B64500B2
S2144444608DB645006C684600A03B4020F41E4020B4
S21444447078524600E7B64500EDB645001017294089
S214444480944F4600002940200C674600341F4020C5
S2144444901C7040206C7040201C614020C3B6450010
S2144444A0C9B6450006172940BC674600503240202E
S2144444B0141F4020E8524600405346009852460097
S2144444C07920294D17F0CAF900222849792017F097
S2144444D0C4F97A2017F0C2F9002225497A2017F049
S2144444E0BCF901220A21234820F0A1F8012209211F
S2144444F0204820F09CF8204A2049204614F030FDFD
S214444500204615F0CDFC09221A492046FFF76AFDDD
S2144445101B4A1A49204614F023FD204615F0C0FCD9
S2144445202B68184A0D2123F06043204614F056FEAB
S2144445300023154A0D21204614F094FEAB68114A18
S2144445400E2123F06043204614F048FE00230F4A11
S2144445500E21204614F086FE4AF2C4510C4B01222A
S2144445605A504AF2C051B0E688524600D5B6450085
S214444570DBB6450008172940944F4600A82D402036
S21444458064674600241F40209C684020EC68402016
S2144445907435412041F69872084B02FB003310B53F
S2144445A003EB8104E278A07800EB0220627802EB09
S2144445B0002213F8210000EB022010BDD8774020DB
S2144445C010B5094B41F6987404FB0030130A00EB0F
S2144445D0810181F8282081F82930130C120E81F8C5
S2144445E02A3081F82B2010BDD877402013B502AB73
S2144445F0044603E9060041F69871094A9DF80430DA
S21444460001FB0022009903F03F0321F06041FEF7CE
S214444610A7FF204602B0BDE81040FEF76DBF00BFBE
S21444462000784020FDF76CBEFDF76CBE70477047BF
S2144446307047704770477047704770477047704779
S21444464070477047704770B5274C284D617823787B
S21444465001F00300A678E27843EA0023C1F3810020
S21444466043EA8023C1F30110890943EA00332079E1
S21444467043EA8133C6F3011143EA0143B10906F024
S2144446800F0643EA814302F0030143EA0153C2F3AF
S214444690810143EA8153C2F30111920943EA01635B
S2144446A043EA82632A6802F0704213432B6009F09F
S2144446B035FF0F4909F086FFE179627901F00F036F
S2144446C0090968601B0143EA121302F0030243EA35
S2144446D0012343EA0636AB689B0C46EA02469B0433
S2144446E01E43AE6070BD00BFD87740209073402014
S2144446F0CDCCCC3DF0B5234D234A2E782879C6F34D
S214444700401706F00F03EC7843EA0713C6F3801706
S214444710F609E97943EA471343EA86136E78AD7897
S21444472043EAC61343EAC53304F0030543EAC553D4
S214444730C4F3810543EA4563C4F30115A40943EA77
S214444740C56343EA4473D46804F000442343C0F387
S2144447500014D36000F0030343EA8403C0F3401418
S21444476043EAC403C0F38014C00943EA041343EA8B
S214444770401343EA8113118A01F440410B431382E8
S214444780F0BD00BFD877402090734020F8B5134D55
S214444790134FEB78AC782E7944EA03246B79288857
S2144447A046EA032624B209F0B9FE0E4909F00AFF88
S2144447B0786136B2204609F0B1FE0A4909F002FF94
S2144447C0B861304609F0AAFE064909F0FBFEEB79CB
S2144447D0F86187F82030044B1C60F8BDD877402039
S2144447E090734020CDCCCC3D90174020084A0949D0
S2144447F01378907881F8243053781843D378064A4F
S2144448009B0443EA0023486A024013434B627047C2
S214444810D877402090734020FF0000FC0C490D4898
S21444482010B54A78CC790B7802F0030143EA0123A9
S214444830C2F38101120943EA812343EA0233826ABE
S21444484043EA044302F07F421343836210BD00BF31
S214444850D87740209073402070B5184D184C28885F
S2144448606E78C0F30A0009F059FE164909F0AAFE0C
S214444870154909F09DFDE062F608A87846EA40101E
S214444880C0F30A0009F04AFE0E4909F09BFE0E49A1
S21444489009F08EFD2063A88809F040FE0B4909F014
S2144448A091FE0B4909F084FD94F83830EA79606348
S2144448B062F3030384F8383070BD00BFD8774020D5
S2144448C0907340200AD7233C14AE23410AD7A33B17
S2144448D00AD723432DE9F041224C234D94F83C203B
S2144448E095F80080EB7922F00F02AE7948F3021077
S2144448F095F9027046EA032608F00F03134336B2CE
S21444490084F83C3009F00AFE6A782064A7F1320045
S2144449105300520003F01E0302F0200243EAD81369
S214444920134394F8442022F03F02134384F844305F
S21444493009F0F4FDA064E878323809F0EFFDE0644D
S214444940A888A0F5004009F0E9FD2065304609F046
S214444950E5FD064909F036FE054909F029FD60657E
S214444960BDE8F08190734020D87740200AD7233C96
S21444497000004843034A044B116852689965DA6557
S214444980704700BFD87740209073402038B5104D0C
S214444990104C288809F0C2FD0F4909F013FE206622
S2144449A0688809F0BBFD0D4909F00CFE0C4909F076
S2144449B0FFFC6066A88809F0B1FD0A4909F002FECA
S2144449C0AB79A06684F86C30EB7984F86D3038BDEA
S2144449D0D877402090734020CDCCCC3D0AD7A33C1A
S2144449E000C02344ACC5273708B5054B188809F0E2
S2144449F095FD044909F0E6FD034B186708BD00BF62
S214444A00D8774020CDCCCC3D907340200C4A0D48FE
S214444A1010B55178137801F00104C1F3410143EA1B
S214444A20042343EA41239178D27843EAC12343EAF4
S214444A30C243426F02F078421343436710BD00BF3F
S214444A40D87740209073402038B5174D174C2888A7
S214444A5009F064FD164909F0B5FD164909F0A8FCAD
S214444A60AB78A06703F00F03E87884F87C3009F04D
S214444A7055FD114909F09CFC09F090FF84F87D002F
S214444A80A88809F04BFD0D4909F09CFD0C4909F036
S214444A908FFCAB79C4F8800003F00F0384F88430AD
S214444AA0EB7984F8853038BDD87740209073402021
S214444AB00AD7A33B0AD72343000048420AD7A33A5F
S214444AC0F8D3234238B5144D144C288809F026FDF3
S214444AD0134909F077FD134909F06AFCAB78C4F82A
S214444AE0880003F00F03A88884F88C30EB7884F8A9
S214444AF08D3009F013FD0C4909F064FD0B4909F0AB
S214444B0057FCAB79C4F8900003F00F0384F8943054
S214444B10EB7984F8953038BDD877402090734020A0
S214444B200AD7A33B0AD723430AD7A33AF8D3234248
S214444B3038B5134D134C288809F0F0FC124909F097
S214444B4041FD124909F034FCAB78C4F8980003F0F0
S214444B500F03A88884F89C3009F0E0FC0C4909F05F
S214444B6031FD0C4909F024FCAB79C4F8A00003F0ED
S214444B700F0384F8A430EB7984F8A53038BD00BF21
S214444B80D8774020907340200AD7A33B0AD72343C4
S214444B900AD7A33AF8D3234270B53B4E3B4C7078C1
S214444BA009F0BCFC35783A4909F00CFD05F07F0560
S214444BB009F0F4FEC0B245EAC015B07809F0AEFC80
S214444BC0334909F0FFFC09F0E9FEC0B245EAC035B6
S214444BD0F07809F0A3FC2F4909F0EAFB09F0DEFE61
S214444BE0D4F8AC30C0B2717903F00043B27945EAE8
S214444BF0C055C1F340001D43337984F8B03001F00A
S214444C000103C4F8AC501B0243EA4023C1F38000BE
S214444C1043EA8023C1F3C00043EAC023C1F3001033
S214444C2043EA0033C1F3401043EA4033C1F38010F3
S214444C30C90943EA803343EAC13302F0010143EA37
S214444C400143C2F3400143EA4143C2F3800143EACD
S214444C508143C2F3C00143EAC143C2F3001143EAAD
S214444C600153C2F34011C2F3801243EA415343EA6C
S214444C708253D4F8B02022F4FF0222F4FE421343B7
S214444C80C4F8B03070BD00BFD87740209073402041
S214444C900AD7233C00002042124B134810B55A78DA
S214444CA0997802F003041B7843EA0423C2F3810490
S214444CB043EA8423C2F30114920943EA043343EAE1
S214444CC0823301F00302C1F3810143EA0243D0F880
S214444CD0A820120D43EA814312051343C0F8A830B6
S214444CE010BD00BFD877402090734020704738B539
S214444CF0124D41F69873124CEB5C84F8BC3041F686
S214444D009A73E85A09F00AFC0E4909F05BFC0E490E
S214444D1009F04EFB41F69C73C4F8C000E85A09F00B
S214444D20FDFB0A4909F04EFC09F038FE41F69F7334
S214444D30A4F8C400EB5C84F8C63038BDD87740206D
S214444D4090734020ACC52737ACC5A73ECDCCCC3DF0
S214444D5038B541F69873104D104CE85A09F0DEFB0E
S214444D600F4909F02FFC0F4909F022FB41F69A73CC
S214444D70C4F8C800E85A09F0D1FB094909F022FCF6
S214444D80084909F015FB41F69F73C4F8CC00EB5C68
S214444D9084F8D03038BD00BFD87740209073402088
S214444DA00AD7A33C00C023440C4A41F69F730C49DF
S214444DB010B541F69974D05C41F69873D35C125D95
S214444DC002F0010243EA0223D1F8D420520C43EA0B
S214444DD0402352041343C1F8D43010BDD877402042
S214444DE090734020284941F69973284A70B5C85CA8
S214444DF041F69A73CD5C41F69B7300F00306CC5C97
S214444E0041F69873CB5C43EA0623C0F3810643EA33
S214444E108623C0F30116800943EA063343EA803307
S214444E2005F00300C5F3810543EA004304F003009C
S214444E3043EA854343EA0053C4F38100A40943EAA2
S214444E408053D2F8D80043EA046300F07C4003431E
S214444E5041F69F70C2F8D83041F69C73CB5C82F81A
S214444E60DC3041F69D73CB5C095C1B0203F47C5337
S214444E7043EA8133D2F8DC1021F47F1121F47C51CB
S214444E800B43C2F8DC3070BDD87740209073402086
S214444E9070B543F630732A4D2A4CEB5A5BBAA4F8E5
S214444EA0E03043F63373EE5C43F63573E95CC6F3A1
S214444EB081030A0943EA820394F8E22022F03F027F
S214444EC0134384F8E23043F63673E85C40EA012044
S214444ED0C0F3090009F022FB1B4909F073FB1B4988
S214444EE009F066FA94F8E8303209C4F8E40062F34C
S214444EF0000384F8E83043F63473E85C40EA06205E
S214444F00C0F3090009F00AFB114909F05BFB43F6BC
S214444F103273C4F8EC00E85C09F000FB0D4909F074
S214444F2051FB94F8F420F308C4F8F00022F007028A
S214444F3003F0040343EA9613134384F8F43070BD35
S214444F40D877402090734020CDCC4C3D6666724165
S214444F509A99193E0AD7233C1B4943F631731B489A
S214444F6030B5CB5C80F8F83043F63273CA5C43F60F
S214444F703573CD5C43F63473CC5C43F63073C95C0E
S214444F8093091B0243EA8123C2F3401143EA814357
S214444F90C2F38001C2F3C00243EAC143D0F8F8101A
S214444FA043EA02532A0905F00F0543EA4253084AE6
S214444FB043EA45630A401343C0F8F830230943EAFA
S214444FC0041480F8FC4030BDD877402090734020CD
S214444FD0FF0000E0F8B5304E43F630732F4CF35ADA
S214444FE05BBAA4F8003143F63373F55C43F6327388
S214444FF0F05CAB0943EA800009F090FA284909F0CE
S214445000E1FA94F80831AA08C4F8040162F30003EC
S21444501084F8083143F63473F05C40EA0520C0F364
S214445020090009F07BFA1E4909F0CCFA94F81031CD
S214445030EA08C4F80C0162F3000384F8103143F61E
S2144450403673F75C43F63573F05CBB0943EA80007D
S21444505009F064FA124909F0B5FA94F818312A09A5
S214445060C4F814016D0962F3000384F8183143F65A
S2144450703773F05C40EA0720C0F3090009F04EFAA3
S214445080074909F09FFA94F82031C4F81C0165F3E7
S214445090000384F82031F8BDD87740209073402030
S2144450A09A99193E38B5124D43F63073114CEB5A63
S2144450B05BBAA4F8243143F63273E85A40BAC0F3D4
S2144450C00D0009F02BFA4FF07A5109F07BFA43F6BB
S2144450D03673C4F82801E85A40BAC0F30D0009F004
S2144450E01DFA4FF07A5109F06DFAC4F82C0138BD18
S2144450F0D877402090734020F8B5434A43F632733D
S214445100424ED15C43F63473D45C43F63373C1F3F6
S2144451108010D55C43F63573D75CCB0943EA40032D
S21444512043F63170105C43EA8003C1F3401043EA0F
S2144451308023C1F3001043EAC023C4F3400043EA8B
S214445140003343F63070105C43EA4033C1F3C0008A
S21444515043EA4053C1F3800043EA8053C5F300104A
S21444516043EAC053680943EA0063C7F3011043EABD
S214445170C063C1F3400001F0010143EA407343EACF
S2144451808173D6F8301101F000410B43C6F8303134
S21444519043F63673D05C40EA0720BF09C0F30900E3
S2144451A009F0BCF91A4909F00DFA1A4909F000F950
S2144451B0C5F3C00204F00103C6F8340143EA4203CF
S2144451C005F004021343C5F3400205F0010543EA23
S2144451D0C203C4F3C00243EA051343EA4713C4F3C5
S2144451E0001743EAC713A709C4F3800443EA072316
S2144451F043EA822343EAC424B6F8383103F47043BE
S2144452001C43A6F83841F8BDD87740209073402018
S214445210CDCCCC3D9A994C4270B543F630732F4D65
S2144452202F4CEB5A5BBAA4F83C3143F63373EE5C2E
S21444523043F63273E85CB30943EA800009F06EF93A
S214445240284909F0BFF994F84431B208C4F840013B
S21444525062F3010384F8443143F63473E85C40EA6D
S21444526006203609C0F3090009F058F91D4909F02B
S214445270A9F994F84C31C4F8480166F3010384F85C
S2144452804C3143F63673EE5C43F63573E85CB3094B
S21444529043EA800009F042F9124909F093F994F878
S2144452A05431B208C4F8500162F3010384F854310F
S2144452B043F63773E85C40EA06203609C0F3090033
S2144452C009F02CF9074909F07DF994F85C31C4F8E3
S2144452D0580166F3010384F85C3170BDD8774020EA
S2144452E090734020CDCCCC3D074943F63073074AF3
S2144452F0CB581BBAC2F8683143F63473CB581BBA42
S214445300C2F86C31704700BFD87740209073402075
S21444531030B543F63073304C3049E35A5BBAA1F8A3
S214445320703143F63673E05C43F63773E25C43F61B
S2144453303273E55C00F0030343EA8503C0F380055B
S21444534043EA8523C2F3800543EAC523850943EA35
S2144453500533B1F8725105F440452B43C2F3C005FA
S214445360A1F8723143F63373E35C81F87431C0F3C9
S214445370C0031B0243EA452302F0030543EA8523A0
S21444538043F63475655D43EA0533C0F30015C0F350
S214445390401043EA0553C2F3001543EA45539509C2
S2144453A0120943EA8553D1F8745102F0020225F4F7
S2144453B07F05024325F47F452B43C1F8743143F6F9
S2144453C03573E35C81F8773191F8783123F0030341
S2144453D01A4381F8782130BDD87740209073402016
S2144453E0F8B5244E43F63073234DF35A5BBAA5F80A
S2144453F07C3143F63373F45C43F63273A208F75CAD
S21444540043F6367302F00C02F05C42EA9412C0088B
S21444541042EA071200EB800085F87E213F0909F036
S2144454207DF895F88431A208C5F8800162F300033C
S21444543085F8843143F63473F05A40BA80B209F0A2
S2144454406DF80E4909F0BEF80D4908F0B1FFC4F3F3
S214445450C0036401C5F8880143EA470304F06004C6
S2144454601C4395F88C3123F07F031C4385F88C410C
S214445470F8BD00BFD877402090734020CDCC4C3D3B
S21444548000C0CC4470B543F63073194E194CF35AE9
S2144454905BBAA4F8903143F63273F05A40BA80B2FD
S2144454A009F03CF8144909F08DF8144908F080FFD7
S2144454B043F63673C4F89401F55C94F8983165F372
S2144454C000036D0884F8983143F63473F05A40BAB2
S2144454D080B2A0F5FF407F3809F020F894F8A03158
S2144454E0C4F89C0165F3000384F8A03170BD00BF86
S2144454F0D8774020907340200AD7A33C00C023446A
S21444550070B543F63073234D234CEB5A5BBAA4F87C
S214445510A43143F63273E85C43F63473EE5CC0F36E
S2144455204002B308360903F002031343820080089E
S21444553002F00402134394F8A62122F00702134310
S21444554084F8A63108F0EAFF144909F03BF81449F8
S21444555008F02EFF43F63373C4F8A801E85C46EA25
S214445560001008F0DBFF0F4909F02CF843F63673B9
S214445570C4F8AC01E85C43F63573EB5CDB0043EA05
S214445580501008F0CBFF054909F01CF8C4F8B001E8
S21444559070BD00BFD877402090734020CDCCCC3D22
S2144455A0CDCC4C400AD7233C70B545F6C8632A4D4B
S2144455B02A4CEB5A5BBAA4F8B43145F6CB63EE5C9E
S2144455C045F6CD63E95CC6F381030A0943EA8203E0
S2144455D094F8B62122F03F02134384F8B63145F6D8
S2144455E0CE63E85C40EA0120C0F3090008F096FF69
S2144455F01B4908F0E7FF1B4908F0DAFE94F8BC3173
S2144456003209C4F8B80162F3000384F8BC3145F6A5
S214445610CC63E85C40EA0620C0F3090008F07EFF4D
S214445620114908F0CFFF45F6CA63C4F8C001E85CE8
S21444563008F074FF0D4908F0C5FF94F8C821F30834
S214445640C4F8C40122F0070203F0040343EA9613A5
S214445650134384F8C83170BDD877402090734020F7
S214445660CDCC4C3D666672419A99193E0AD7233C86
S2144456701B4945F6C9631B4830B5CB5C80F8CC3132
S21444568045F6CA63CA5C45F6CD63CD5C45F6CC6345
S214445690CC5C45F6C863C95C93091B0243EA812384
S2144456A0C2F3800143EA8143C2F3C001C2F340120D
S2144456B043EAC143D0F8CC1143EA02532A0905F021
S2144456C00F0543EA4253084A43EA45630A401343F4
S2144456D0C0F8CC31230943EA041480F8D04130BDE5
S2144456E0D877402090734020FF0000E070B545F620
S2144456F0C863184D184CEB5A5BBAA4F8D43145F637
S214445700CC63E85AEE5C40BAF609C0F3090008F0E8
S21444571005FF124908F056FF94F8DC31C4F8D80166
S21444572066F3000384F8DC3145F6CA63E85AEE5C57
S21444573040BAF609C0F3090008F0F0FE074908F03D
S21444574041FF94F8E431C4F8E00166F3000384F8BA
S214445750E43170BDD8774020907340209A99193E22
S214445760F8B5244E45F6C863234DF35A5BBAA5F8FC
S214445770E83145F6CB63F45C45F6CA63A208F75CA9
S21444578045F6CE6302F00C02F05C42EA9412C0087E
S21444579042EA071200EB800085F8EA213F0908F048
S2144457A0BDFE95F8F031A208C5F8EC0162F300039B
S2144457B085F8F03145F6CC63F05A40BA80B208F02A
S2144457C0ADFE0E4908F0FEFE0D4908F0F1FDC4F3A7
S2144457D0C0036401C5F8F40143EA470304F06004D7
S2144457E01C4395F8F83123F07F031C4385F8F841B1
S2144457F0F8BD00BFD877402090734020CDCC4C3DB8
S21444580000C0CC4470B545F6C863194E194CF35ADB
S2144458105BBAA4F8FC3145F6CA63F05A40BA80B283
S21444582008F07CFE144908F0CDFE144908F0C0FD8B
S21444583045F6CE63C4F80002F55C94F8043265F38A
S21444584000036D0884F8043245F6CC63F05A40BA37
S21444585080B2A0F5FF407F3808F060FE94F80C3222
S214445860C4F8080265F3000384F80C3270BD00BF28
S214445870D8774020907340200AD7A33C00C02344E6
S21444588070B545F6C863234D234CEB5A5BBAA4F86F
S214445890103245F6CA63E85C45F6CC63EE5CC0F36A
S2144458A04002B308360903F002031343820080081B
S2144458B002F00402134394F8122222F00702134320
S2144458C084F8123208F02AFE144908F07BFE144984
S2144458D008F06EFD45F6CB63C4F81402E85C46EA6D
S2144458E0001008F01BFE0F4908F06CFE45F6CE6328
S2144458F0C4F81802E85C45F6CD63EB5CDB0043EA8B
S214445900501008F00BFE054908F05CFEC4F81C0273
S21444591070BD00BFD877402090734020CDCCCC3D9E
S214445920CDCC4C400AD7233C70B545F6C8632F4DC2
S2144459302F4CEB5A5BBAA4F8203245F6CB63EE5CA8
S21444594045F6CA63E85CB30943EA800008F0E6FD1E
S214445950284908F037FE94F82832B208C4F82402DE
S21444596062F3010384F8283245F6CC63E85C40EAE7
S21444597006203609C0F3090008F0D0FD1D4908F09A
S21444598021FE94F83032C4F82C0266F3010384F8FE
S214445990303245F6CE63EE5C45F6CD63E85CB3093B
S2144459A043EA800008F0BAFD124908F00BFE94F86A
S2144459B03832B208C4F8340262F3010384F8383249
S2144459C045F6CF63E85C40EA06203609C0F3090092
S2144459D008F0A4FD074908F0F5FD94F84032C4F8F1
S2144459E03C0266F3010384F8403270BDD877402009
S2144459F090734020CDCCCC3D30B545F6C863304C92
S214445A003049E35A5BBAA1F8443245F6CE63E05CCB
S214445A1045F6CF63E25C45F6CA63E55C00F00303F3
S214445A2043EA8503C0F3800543EA8523C2F3800531
S214445A3043EAC523850943EA0533B1F8465205F4DB
S214445A4040452B43C2F3C005A1F8463245F6CB6326
S214445A50E35C81F84832C0F3C0031B0243EA4523A3
S214445A6002F0030543EA852345F6CC65655D43EAC3
S214445A700533C0F30015C0F3401043EA0553C2F3A0
S214445A80001543EA45539509120943EA8553D1F86C
S214445A90485202F0020225F47F05024325F47F456E
S214445AA02B43C1F8483245F6CD63E35C81F84B326C
S214445AB091F84C3223F003031A4381F84C2230BD4C
S214445AC0D877402090734020F8B5344A45F6CA63E8
S214445AD0334DD15C45F6CC63D45C45F6CB63C1F319
S214445AE08017D05C45F6CD63D65CCB0943EA4703C2
S214445AF045F6C967D75D43EA8703C1F3401743EACF
S214445B008723C1F3001743EAC723C4F3400743EA95
S214445B10073345F6C867D75D43EA4733C0F30017F3
S214445B20400943EA475343EA8053C6F3011043EA25
S214445B304063C1F3400001F0010143EAC06343EA15
S214445B400173D5F8501201F060410B43C5F850324A
S214445B5045F6CE63D05C40EA0620C0F3090008F060
S214445B60DDFC104908F02EFD0F4908F021FCC5F86D
S214445B705402B30904F0010646EA43066308A4093E
S214445B8003F008031E4395F8583246EA041423F0FB
S214445B903F031C4385F85842F8BD00BFD8774020E1
S214445BA090734020CDCCCC3D9A994C42074945F65B
S214445BB0C863074ACB581BBAC2F8683245F6CC636A
S214445BC0CB581BBAC2F86C32704700BFD877402017
S214445BD09073402008B5094A47F66263D05A40BAE3
S214445BE080B208F09BFC064908F0ECFC054908F036
S214445BF0DFFB054BC3F8700208BD00BFD8774020D2
S214445C000AD7A33C00C023449073402010B50D4BE4
S214445C1047F662610C4C595C94F8742261F30302B3
S214445C2084F8742247F66462985A40BA80B208F000
S214445C3075FC064908F0C6FC054908F0B9FBC4F8EB
S214445C40780210BDD877402090734020CDCC4C3D90
S214445C5000C0CC4408B5094A49F6FA53D05A40BA6B
S214445C6080B208F05BFC064908F0ACFC054908F035
S214445C709FFB054BC3F87C0208BD00BFD877402085
S214445C800AD7A33C00C023449073402010B50D4B64
S214445C9049F6FA510C4C595C94F8802261F303029D
S214445CA084F8802249F6FC52985A40BA80B208F0EA
S214445CB035FC064908F086FC054908F079FBC4F82B
S214445CC0840210BDD877402090734020CDCC4C3D04
S214445CD000C0CC442A4B2B4A10B55C78C4F38101EF
S214445CE01170C4F30111284A1170C4F30101274A04
S214445CF0A40911701A782649C2F381100870C2F3B9
S214445D00011024490870C2F381002349C2F30102FA
S214445D10087022490A701A7A2149C2F38100C2F3F4
S214445D20010208701F490A705A7A1F49C2F30312C7
S214445D300A709A7A1D49C2F301020A709A781C497D
S214445D4002F003000860C2F381001A490860C2F3F7
S214445D50011019499209086018490A60DA78184906
S214445D6002F00300C2F381020860164958680A70BC
S214445D70154908F0DBFC154B1860154B1C6010BD2C
S214445D8090734020101940200F1940200E194020CF
S214445D900D1940200C1940200B1940200A194020A8
S214445DA00919402008194020441E4020D818402095
S214445DB000194020FC184020F8184020F4184020D1
S214445DC0F01840203D1E4020CDCCCC3DE818402065
S214445DD004194020284B29491A7B02F00700086022
S214445DE0C2F3C00026490860C2F300102549087073
S214445DF0C2F340102449C2F38012087023490A7043
S214445E009A892349C2F3C7120A60DA682149C2F361
S214445E10C7320A60DA892049C2F3C1120A60DA7BC3
S214445E201E49C2F341000860C2F3C1001C49C2F3D4
S214445E30411208601B490A601A7C1B4902F00300A1
S214445E400860C2F3800019490860C2F3C0001849CC
S214445E500860C2F300101749C2F34012086016499E
S214445E600A601A8A1549C2F383125B7C0A60C3F33C
S214445E708303134A1360704790734020D41840201D
S214445E80D0184020CE184020CD184020CC184020B2
S214445E90C8184020C4184020C0184020BC184020D1
S214445EA0B8184020B4184020B0184020AC18402001
S214445EB0A8184020A4184020A01840209C18402031
S214445EC0981840207047034B034ADB8CC3F3870380
S214445ED013707047907340208C1740200A4A0B4931
S214445EE092F82830C3F38100C3F3011308700849BD
S214445EF00B7092F82930074AC3F30101C3F38103B8
S214445F001170054A13707047907340203C1E402021
S214445F10391E40203B1E4020381E40207047184BF8
S214445F20184993F83C2002F001000860C2F3400090
S214445F3015490860C2F380001449C2F3C0020860E1
S214445F4013490A60196C134A116093F844201249A5
S214445F5002F001000860C2F343001049C2F3401245
S214445F6008600F490A60996C0E4A1160D96C0E4A53
S214445F701160196D0D4A11605A6D0D4B1A607047C9
S214445F8090734020A01940209C1940209819402026
S214445F9094194020901940208C194020881940209C
S214445FA084194020801940207C19402078194020CC
S214445FB074194020344A354992F8AC3003F0010055
S214445FC00860C3F3400032490860C3F38200314995
S214445FD0C3F34113086030490B60B2F8AC302F4924
S214445FE0C3F3C7130B60D2F8AC302D49C3F3C733A1
S214445FF00B60B2F8AE302B49C3F3C7130B6092F86C
S214446000B010294B196092F8B130284903F00100CA
S2144460100860C3F3400026490860C3F3800025495E
S2144460200860C3F3C00024490860C3F30010234942
S2144460300860C3F3401022490860C3F38010214926
S214446040DB09086020490B6092F8B2301F4A03F01F
S21444605001011160C3F340011D4A1160C3F380017E
S2144460601C4A1160C3F3C0011B4A1160C3F30011FC
S2144460701A4A1160C3F34011194AC3F380131160DE
S214446080184A1360704700BF907340206C19402034
S2144460906819402064194020601940205C1940204B
S2144460A05819402054194020501940204C1940207B
S2144460B04819402044194020401940203C194020AB
S2144460C03819402034194020301940202C194020DB
S2144460D02819402024194020201940201C1940200B
S2144460E01819402014194020704710B50E4C0F4B19
S2144460F0226E1A600E4B186894F8C9321B0703D5F3
S2144461000C4B196808F056F90B4B94F86C20186041
S2144461100A4B1A60626E0A4B1A6094F86D30094A4C
S21444612003F00F03136010BD90734020F81C40200A
S214446130F41C40207C174020F01C4020E41C4020E7
S214446140EC1C4020E01C4020114A124992F874305E
S21444615003F003000860C3F383000F499B090860FB
S2144461600E490B6092F875300D49C3F3410003F0B5
S214446170010308600B490B60536F0B49C3F3C723F5
S2144461800B60B2F87630094AC3F3C703136070470E
S21444619090734020BC1C4020B81C4020B41C4020B7
S2144461A0AC1C4020B01C4020A01C4020A81C402012
S2144461B0114B124A996F116093F87C20104902F0F3
S2144461C00F00120908600F490A6093F87D100E4AC2
S2144461D01160D3F880100D4A116093F884200C495E
S2144461E002F00F00120908600A490A6093F88520F5
S2144461F0094B1A60704700BF9073402054184020E3
S214446200501840204C18402048184020441840203D
S214446210401840203C18402038184020114B124A61
S214446220D3F88810116093F88C20104902F00F00C0
S214446230120908600E490A6093F88D100D4A1160E1
S214446240D3F890100C4A116093F894200B4902F04E
S2144462500F00120908600A490A6093F89520094B12
S2144462601A607047907340203418402030184020FD
S2144462702C1840202818402024184020201840205D
S2144462801C184020181840200F4B104AD3F898107A
S214446290116093F89C200E4902F00F001209086022
S2144462A00C490A60D3F8A0100B4A116093F8A42056
S2144462B00A4902F00F001209086009490A6093F877
S2144462C0A520084B1A60704790734020141840204D
S2144462D0101840200C18402008184020041840206D
S2144462E000184020FC1740207047174A174992F878
S2144462F0A83003F003000860C3F381001449086023
S214446300C3F3011013499B09086013490B6092F8C4
S214446310A930124903F003000860C3F38100104912
S2144463200860C3F301100F499B0908600E490B60CF
S21444633092F8AA300D4A03F00301C3F381031160B7
S2144463400B4A1360704700BF90734020281C4020BF
S214446350241C4020201C40201C1C4020181C40208C
S214446360141C4020101C40200C1C4020081C4020BC
S214446370041C402010B50C4C0C4B94F8BC20B4F8CC
S214446380C4001A60D4F8C020094B1A6008F0C2F85A
S214446390084B094A186094F8C63003F00F011B09ED
S2144463A01160064A136010BD907340209418402034
S2144463B0901840208C18402088184020841840208C
S2144463C0094B0A4AD3F8C8101160D3F8CC10084ACF
S2144463D093F8D030116003F00F01064A1B09116090
S2144463E0054A1360704700BF9073402080184020D1
S2144463F07C1840207818402074184020114A1249CE
S21444640092F8D43003F003000860C3F381000F49C8
S2144464100860C3F301100E499B0908600D490B60E0
S21444642092F8D5300C4903F00100C3F343030860E7
S2144464300A490B60D2F8D430094AC3F34333136095
S214446440704700BF90734020701840206C1840205E
S2144464506818402064184020601840205C1840208B
S21444646058184020164A174992F8D83003F00300CB
S2144464700860C3F3810014490860C3F3011013494C
S2144464809B09086012490B6092F8D930114903F011
S21444649003000860C3F381000F490860C3F301108A
S2144464A00E499B0908600E490B6092F8DA300D4A93
S2144464B003F00301C3F3810311600B4A1360704772
S2144464C090734020781C4020741C4020701C402050
S2144464D06C1C4020681C4020641C4020601C4020EB
S2144464E05C1C4020581C4020541C402008B5054BDA
S2144464F00549D3F8EC0008F019F908F04FFA034BB5
S214446500186008BD907340209A99193E301D40206B
S21444651008B5FFF7DFFBFFF75DFCFFF7D4FCFFF79A
S214446520DDFCFFF7FCFCFFF7E0FDFFF70DFEFFF791
S21444653021FFFFF745FFFFF761FFFFF793FFFFF7E4
S214446540D5FFFFF7D2FEBDE80840FFF733BD7047DE
S214446550704770477047704770477047024BD3F890
S2144465608821024B1A60704790734020C017402021
S214446570024BD3F89421024B1A6070479073402024
S214446580EC17402008B5FFF7E9FFBDE80840FFF7E1
S214446590EFBF704770477047704770477047704703
S2144465A070477047704770477047704770477047EA
S2144465B010B5184C1849D4F8940107F0FBFE174957
S2144465C008F0B4F807F050FB0CF0AAF907F054FEB4
S2144465D01349A4F88802D4F8880107F0EBFE114961
S2144465E008F0A4F807F040FB0CF09AF907F044FED4
S2144465F00D4BA4F88A021B6884F88C320B4B1A683D
S2144466000B4B1B6803F00F0343EA021384F88D32E6
S21444661010BD00BF9073402000C023440AD7A33C5B
S21444662000C0CC44CDCC4C3D7C1C4020581A402065
S2144466305C1A402038B5164C1649D4F8945128466E
S21444664007F0B8FE144908F071F807F00DFB0CF09B
S21444665067F907F011FE1149A4F89002284607F09E
S214446660A9FE0F4908F062F807F0FEFA0CF058F954
S21444667007F002FE0B4BA4F892021A680A4B1B68FA
S21444668003F00F0343EA021384F8943238BD00BF84
S2144466909073402000C023440AD7A33C00C0CC4497
S2144466A0CDCC4C3D481A40204C1A4020134B186819
S2144466B010B500F28F20124C07F02CFF114908F059
S2144466C035F808F045F9104BA4F89802186800F21B
S2144466D0666007F01FFF0D4908F028F808F038F9FF
S2144466E00B4BA4F89A021A680A4B1B6803F00F0374
S2144466F043EA021384F89C3210BD00BF441A40207B
S214446700907340200AD7A33C401A4020CDCC4C3D41
S214446710381A40203C1A4020134B186810B500F233
S2144467208F20124C07F0F6FE114907F0FFFF08F0E1
S2144467300FF9104BA4F8A002186800F2666007F040
S214446740E9FE0D4907F0F2FF08F002F90B4BA4F8F6
S214446750A2021A680A4B1B6803F00F0343EA0213AB
S21444676084F8A43210BD00BF341A402090734020F1
S2144467700AD7A33C301A4020CDCC4C3D281A4020A2
S2144467802C1A40204D4B4E4A1B78012B5BD14D4B67
S2144467904D491B6809689B0001F0030103F00C0394
S2144467A00B434A490968090101F030010B43484943
S2144467B009688901C9B20B4346490968090201F4CC
S2144467C040710B4344490968890201F440610B4314
S2144467D042490968090301F440510B43404909689A
S2144467E0890389B20B433F490968090401F44031DF
S2144467F00B433D490968890401F440210B43D2F810
S214446800A812090D09050B43C2F8A832374B1B786A
S21444681003F00301364B1B7803F003031B0143EAE2
S21444682081133449097801F0030143EA0123B2F89D
S214446830AA1221F47C710B43A2F8AA322E4B1B8871
S21444684082F8AC327047002B33D12C4B2C491B6852
S21444685009689B0001F0030103F00C030B4329492C
S2144468600968090101F030010B4327490968890189
S214446870C9B20B4325490968090201F440710B4328
S21444688023490968890201F440610B432149096898
S214446890090301F440510B431F490968890389B22F
S2144468A00B431E490968090401F440310B431C4953
S2144468B0A0E7023B012BA9D8C7E700BF2E1E402005
S2144468C090734020241C4020281C4020201C40203C
S2144468D01C1C4020181C4020141C4020101C402027
S2144468E00C1C4020081C4020041C40204D1E402008
S2144468F04C1E40204E1E40204A1E40204C1C402029
S214446900501C4020481C4020441C4020401C402032
S2144469103C1C4020381C4020341C4020301C402066
S2144469202C1C4020124B13491B7803F00302124BD5
S2144469301B7803F0030343EA8203104A127802F0FA
S214446940030243EA02130E4A127802F0030243EAB1
S21444695082130C4A127802F0030243EA0223B1F887
S214446960B02202F47C421343A1F8B032704700BF11
S214446970DF1D402090734020E01D4020DE1D402057
S214446980DD1D4020DC1D402038B52F4B2F4D1C68A4
S2144469902F4B64001B6804F0020403F001031C43FD
S2144469A02C4B1B689B0003F004031C432A4B1B68B8
S2144469B0DB0003F008031C43284B1B681B01DBB2B7
S2144469C01C43274B1B681B0203F440731C43254B94
S2144469D01B689B0203F4E0531C43234B1868234B69
S2144469E0400300F4C0400443186807F093FD204970
S2144469F007F0E0FC1F4907F099FE07F0A9FF1E4B7D
S214446A001B4903EAC0331C43D5F8B43203F00043B1
S214446A101C431A4BC5F8B442186807F0CBFC15491A
S214446A2007F084FE07F094FF154B1149A5F8B80209
S214446A30186807F0BFFC0F4907F078FE07F088FF98
S214446A40A5F8BA0238BD00BF7C1D40209073402094
S214446A50801D4020781D4020741D4020701D40201D
S214446A606C1D4020681D4020641D4020601D402051
S214446A70000048430AD7233C0080FF7F5C1D40202B
S214446A801C1E4020194B186810B5C830184C07F027
S214446A9041FD184907F04AFE07F05AFF164B1749BE
S214446AA0A4F8BC02186807F085FC154907F03EFEBA
S214446AB007F04EFF134BA4F8BE021B68A4F8C0327E
S214446AC0114B186807F044FF104B84F8C2021B6849
S214446AD084F8C3320E4B1A680E4B1B6803F00F0340
S214446AE043EA021384F8C43210BD00BF381D402068
S214446AF090734020CDCCCC3D341D402000C0234470
S214446B000AD7A33C301D40202C1D4020281D402081
S214446B10201D4020241D4020194B1A4A1B681A4940
S214446B2082F8C832194B09681B6809029B0201F4B3
S214446B30407103F480630B4315490968C90201F4A4
S214446B40C0510B4313490968490301F4C0410B4340
S214446B5011490968C90301F4C0310B43D2F8C8127D
S214446B6021F4FF3121F480710B43C2F8C8320B4B39
S214446B701B68A2F8CE320A4B1B68A2F8CC32704788
S214446B80C818402090734020541D4020501D40207B
S214446B904C1D4020481D4020441D4020401D4020A0
S214446BA03C1D4020094B0A491A680A4B02F0010270
S214446BB01B6803F0030343EA820391F8D02222F0D1
S214446BC00702134381F8D032704700BF4C1B402065
S214446BD090734020501B40200A4A0B4B126883F89F
S214446BE0D4220A4A126883F8D522094A126883F8DE
S214446BF0D622084A126883F8D722074A1268C3F88E
S214446C00D8227047781A402090734020741A402047
S214446C10701A40206C1A4020681A4020194B1A49B2
S214446C20186810B507F0C6FB184C07F091FE184BD1
S214446C30154984F8DC02186807F0BCFB07F088FEA8
S214446C40144B84F8DD021B68A4F8DE32124B186835
S214446C5007F07EFE114B124A1B78126884F8E13224
S214446C60104B02F0070284F8E0021B78DB0003F0C6
S214446C700803134394F8E22222F00F02134384F8E5
S214446C80E23210BD801940200000484290734020F4
S214446C907C19402090174020E81840208C1740204C
S214446CA0D4184020CE18402038B5354B354C1D7886
S214446CB0354B05F003051B7803F00302334B1B7872
S214446CC003F0030343EA8203314A127802F00302D4
S214446CD043EA02132F4A127802F0030243EA82136D
S214446CE02D4A127802F0030243EA02232B4A127812
S214446CF002F0030243EA8223294A127802F003028E
S214446D0043EA0233274A1268920392B21343264A4E
S214446D1043EA0543127843EA854302F0030243EA12
S214446D20055343EA855343EA056343EA8263D4F84A
S214446D30E42202F070421343C4F8E4321B4B186852
S214446D4007F006FE1A4B84F8E8021B7803F00302A9
S214446D502B0243EA8223174A1568174A2D03ADB21D
S214446D602B431568D4F8E8222D0422F47F2205F438
S214446D70702522F470622B431343C4F8E83238BDBE
S214446D8008194020907340200B1940200A194020CF
S214446D900C1940200D1940200E194020101940208F
S214446DA00F194020041940203D1E4020E81840207A
S214446DB009194020E0194020DC1940201E4B1F4A88
S214446DC070B51C681E4B958904F00F041868137B35
S214446DD005F4FF45117C00F00F0003F07F032B43BE
S214446DE0D56805F4FF052B43D589C5F3C11543EA99
S214446DF0C553D57BC5F3410643EA4663C5F3C1068E
S214446E00C5F3411543EAC66343EA4573D2F8EC52E8
S214446E1005F000452B43C2F8EC3201F03F03B2F8CC
S214446E20F01243EA841301F4404143EA80230B43BF
S214446E30A2F8F03270BD00BF9C18402090734020EA
S214446E409818402010B5184C1849606907F06EFC35
S214446E5006F00AFF0BF064FD07F00EFA1349A4F897
S214446E60F402A06907F062FC06F0FEFE0BF058FD43
S214446E7007F002FA0D49A4F8F602E06907F056FC5A
S214446E8006F0F2FE0BF04CFD07F0F6F9084BA4F8BA
S214446E90F8021A78074B1B7803F00F0343EA0213F1
S214446EA084F8FA3210BD00BF90734020CDCCCC3D60
S214446EB08817402089174020124A92F8243010B58B
S214446EC082F8FC32104BD2F8FC421878D38CC3F3C9
S214446ED08701536AC3F309231B0243EA81430B49E0
S214446EE0097801F00F0143EA8163094921400B43C5
S214446EF0C2F8FC3292F8003360F3030382F800339E
S214446F0010BD00BF907340208A1740208B17402046
S214446F10FF0000C01D4B1E4A1B6812689B001D499B
S214446F2002F0030203F00C0313431B4A12681201D7
S214446F3002F030021343194A12689201D2B2134344
S214446F40174A1268120202F440721343154A126832
S214446F50920202F440621343134A1268120302F484
S214446F6040521343114A1268920302F47032134398
S214446F700F4A1268920402F470121343D1F80423A1
S214446F80920D92051343C1F804337047181D4020F0
S214446F901C1D402090734020141D4020101D40208E
S214446FA00C1D4020081D4020041D4020001D40208C
S214446FB0FC1C4020134B186810B500F28F20124C6E
S214446FC007F0A8FA114907F0B1FB07F0C1FC104BD3
S214446FD0A4F80803186800F2666007F09BFA0D49A7
S214446FE007F0A4FB07F0B4FC0B4BA4F80A031A689A
S214446FF00A4B1B6803F00F0343EA021384F80C336E
S21444700010BD00BF001C4020907340200AD7A33C0C
S214447010FC1B4020CDCC4C3DF41B4020F81B4020AC
S214447020134B186810B500F28F20124C07F072FA12
S214447030114907F07BFB07F08BFC104BA4F81003B8
S214447040186800F2666007F065FA0D4907F06EFBB3
S21444705007F07EFC0B4BA4F812031A680A4B1B6815
S21444706003F00F0343EA021384F8143310BD00BF41
S214447070F01B4020907340200AD7A33CEC1B4020D2
S214447080CDCC4C3DE41B4020E81B4020134B1868F5
S21444709010B500F28F20124C07F03CFA114907F065
S2144470A045FB07F055FC104BA4F81803186800F28B
S2144470B0666007F02FFA0D4907F038FB07F048FCE6
S2144470C00B4BA4F81A031A680A4B1B6803F00F0309
S2144470D043EA021384F81C3310BD00BFE01B402073
S2144470E0907340200AD7A33CDC1B4020CDCC4C3DBB
S2144470F0D41B4020D81B4020134B186810B500F210
S2144471008F20124C07F006FA114907F00FFB07F0E0
S2144471101FFC104BA4F82003186800F2666007F0C2
S214447120F9F90D4907F002FB07F012FC0B4BA4F8E3
S21444713022031A680A4B1B6803F00F0343EA021340
S21444714084F8243310BD00BFD01B402090734020E9
S2144471500AD7A33CCC1B4020CDCC4C3DC41B40207E
S214447160C81B40201D4B10B5186807F0F1FB1C4C9B
S2144471701C4BA4F82803186807F0EAFB1A4BA4F83B
S2144471802A031B68A4F82C33184B1A68184B02F0D1
S21444719003021B6803F0010343EA4203154A1268DC
S2144471A002F0030243EAC203134A126802F00102E1
S2144471B043EA4213114A126802F00F0243EA82136A
S2144471C00F4A126802F00F0243EA8223B4F82E23D1
S2144471D002F440421343A4F82E3310BD74194020E1
S2144471E090734020EC174020B81B40204C1D402094
S2144471F0B01B4020441D4020A41B4020A01B402020
S2144472009C1B40201C4B1D4A18681D4B12681B686B
S21444721002F00F021B491B01DBB213431A4A1268E1
S214447220120202F470621343184A1268120302F4FC
S21444723080521343164A1268520302F4C042134360
S214447240144A1268D20302F4C0321343124A126834
S214447250520602F0F05210B51343D1F830430F4AA9
S21444726022401343C1F8303391F8343360F30303B8
S21444727081F8343310BD00BF7C1B4020981B40204F
S214447280941B402090734020901B40208C1B402031
S214447290481D4020841B4020801B40200000FEE107
S2144472A00F4B10B5186807F053FB0E4B0E4C1B687B
S2144472B084F8380384F839330C4B1B68A4F83A3303
S2144472C00B4B1B68A4F83C330A4B1A680A4B1B68E2
S2144472D003F00F0343EA021384F83E3310BD00BFA5
S2144472E02C1D4020281D4020907340203C1D4020EB
S2144472F0401D4020641B4020681B40201F4B2049F3
S214447300186810B507F056F81E4907F00FFA1E4CD9
S21444731007F01EFB1D4B80B21A681D4BC4F8400391
S2144473201B6803F00F0343EA021384F84433194BF3
S214447330186807F0EFF8184907F03CF807F008FB20
S214447340164B174984F84503186807F033F815496F
S21444735007F0ECF907F0FCFA134B80B21A68134BAB
S214447360C4F848031B6803F00F0343EA021384F887
S2144473704C330F4B1B6884F84D3310BD54184020D3
S2144473800AD723430AD7A33B907340204C18402087
S21444739050184020481840200000484244184020D6
S2144473A0F8D323420AD7A33A3C184020401840203A
S2144473B0381840201C4B1D49186810B506F0FAFFD3
S2144473C01B4907F0B3F91B4C07F0C2FA1A4B80B2BC
S2144473D01A491A681A4BC4F850031B6803F00F0383
S2144473E043EA021384F85433164B1B6884F8553327
S2144473F0154B186806F0DEFF144907F097F907F0B6
S214447400A7FA134B80B21A68124BC4F858031B6889
S21444741003F00F0343EA021384F85C330E4B1B68F5
S21444742084F85D3310BD00BF341840200AD7234388
S2144474300AD7A33B907340202C184020F8D323420D
S2144474403018402028184020241840200AD7A33A51
S2144474501C18402020184020181840201A4B1B495E
S214447460186810B506F0A6FF194907F05FF9194CDD
S21444747007F06EFA184B80B218491A68184BC4F8CD
S21444748060031B6803F00F0343EA021384F8643373
S214447490144B186806F08EFF134907F047F907F0B7
S2144474A057FA124B80B21A68114BC4F868031B682B
S2144474B003F00F0343EA021384F86C330D4B1B6846
S2144474C084F86D3310BD00BF141840200AD72343F8
S2144474D00AD7A33B907340200C184020F8D323428D
S2144474E010184020081840200AD7A33A0018402015
S2144474F004184020FC174020244B2549186810B532
S21444750006F058FF234C07F023FA234B204984F80F
S2144475107003186806F04EFF07F01AFA1F4B84F8FB
S2144475207103186806F0F6FF1D4906F043FF07F09E
S2144475300FFA1C4B84F87203186807F009FA1A4BC2
S21444754084F873031A68194B02F007021B6803F0A9
S214447550010343EA4203164A127802F0010243EA60
S2144475600213144A126802F00F0243EA4213124A04
S214447570126802F00F0243EA4223B4F8742302F47A
S21444758060421343A4F8743310BD00BF80194020F2
S21444759000004842907340207C19402054194020F3
S2144475A000002042E8184020D4184020A01840206C
S2144475B0CE184020F8174020F417402008B5FFF7AF
S2144475C073FBBDE80840FFF797BFF8B53A4B3B4D11
S2144475D01B783B4985F878333A4B186807F0A6F889
S2144475E007F0B6F9384A394B03EA40231068D5F811
S2144475F07823000200F48070034335481040034368
S214447600C5F87833334B1B7885F87C33324B1C688B
S214447610324B04F003041F68314B07F001071E6821
S214447620304B44EA870406F00106186806F072FFF9
S2144476304FF0814106F0C6FF07F08AF92A4A2B4BE1
S21444764044EAC606D5F87C1303EA00231068284AA1
S214447650800595F8804300F4800024F00F0403432B
S2144476601068244A2643C005126800F4000085F8D2
S21444767080631206034302F0407213431E4A1268A4
S214447680920602F0406213431C4A1268120702F044
S214447690805213431A4A1268520702F000521343A8
S2144476A0184A1268920702F080421343164A0A4068
S2144476B01343C5F87C33F8BDDA1D40209073402050
S2144476C0CDCCCC3DD01D4020D41D402000FEFF0133
S2144476D0FF0000FEDB1D4020AC1D4020A81D4020BE
S2144476E0A41D4020CC1D4020C81D402000FF3F0064
S2144476F0C41D4020C01D4020BC1D4020B81D402055
S214447700B41D4020B01D4020FF0000803A4B4FF08F
S21444771084412DE9F047394E1B7886F88433384B3C
S2144477201B7886F88533374B186806F043FE4FF0CF
S214447730834106F047FF07F00BF9334B04463349C1
S21444774093F800A0324B0AF0010A186806F032FE9D
S214447750304906F0EBFF07F0FBF82F4B81462F49E4
S21444776093F800802E4B08F00108186806F022FEB5
S2144477702C4906F0DBFF07F0EBF82B4B05464FF0A1
S21444778084411F78294BC5F30B0507F00107186899
S21444779006F010FE4FF0834106F014FF07F0D8F8C9
S2144477A0234BC0F3090245EA07351878C4F30903A6
S2144477B000F0010043EA8A2342EA8022B6F88603B0
S2144477C000F4784002431B4800EAC929A6F88623F9
S2144477D0D6F8882343EA090302F07F4243EAC853B3
S2144477E01343C6F88833B6F88C3303F460431D431A
S2144477F0A6F88C53BDE8F087F91A402090734020D1
S214447800F81A4020EC1A4020E81A402033336F41DF
S214447810E41A40200AD7233CE01A4020CDCCCC4280
S214447820DC1A4020CDCC4C3DDB1A4020F41A4020D4
S214447830F01A402000F87F00084A094B127809499C
S21444784083F89023084A0978127883F8912393F8AA
S214447850922361F3000283F892237047561B40201C
S21444786090734020541B4020551B402038B50C4B89
S2144478700C4C5D68284606F0F7F90BF051F806F014
S21444788023FD0949C4F8A403284606F04FFF06F032
S214447890EBF90BF045F806F017FDC4F8A00338BD25
S2144478A0F04440209073402000000842F8B5204B36
S2144478B0204D186806F02EFE4FF0814106F082FEF9
S2144478C007F046F81C4B04461F681C4BC4F30D04D3
S2144478D007F001071E681A4B44EA8734186844EADE
S2144478E0C63406F017FE4FF0814106F06BFE07F0F3
S2144478F02FF8144AC0F30D03A5F8AC431068124A97
S214447900800300F4804003431068104AC0031268A2
S21444791000F4FF00D205034302F0FF421343D5F8B8
S214447920A82302F000421343C5F8A833F8BD00BFAD
S214447930C019402090734020BC194020B8194020FC
S214447940D0194020CC194020C8194020C4194020E2
S21444795070B5194C194D26682946304606F0EEFF98
S21444796008B1256006E0164D3046294606F0C8FFA5
S2144479700028F6D1134B144D1B68144985F8B033D0
S214447980134B20681B6885F8B13306F013FD114984
S21444799006F0CCFE06F068F90AF0C2FF06F06CFC6E
S2144479A00D4A95F8B4331278A5F8B20362F300038F
S2144479B085F8B43370BD00BF381B40200000C84370
S2144479C00000C8C3401B40209073402000C023449E
S2144479D03C1B40200AD7A33C341B40200C4B0D4A8A
S2144479E01B680D4982F8B8330C4B09781B6801F0C4
S2144479F0030182F8B9330A4B1B789B0003F00C034F
S214447A000B430849097843EA011382F8BA337047AE
S214447A10301B4020907340202A1B40202C1B4020C3
S214447A20291B4020281B40200D4B0E4A1B780E492C
S214447A3082F8BC330D4B09781B7801F0010182F8BB
S214447A40BD330B4B1B785B0003F002030B4392F8E9
S214447A50BE1321F003010B4382F8BE33704700BFC8
S214447A604B1B402090734020491B40204A1B40201B
S214447A70481B4020F8B5254B254C1B78254F84F8E9
S214447A80C033254B1B7884F8C133244B18783230E6
S214447A9006F044FD014606F08DFC06F059FF2049E9
S214447AA084F8C2030E781F493F780D781E4907F0C4
S214447AB001071E4B08781E491A78303009781D4B4A
S214447AC049001B7801F03E01394394F8C37327F00C
S214447AD03F07394384F8C31303F03F0102F01F0302
S214447AE006F00F0243EA411343EAC22305F03F027D
S214447AF043EAC23300F03F0243EA4253D4F8C42375
S214447B0002F078421343C4F8C433F8BDC71A402081
S214447B1090734020C41A4020C61A4020C51A4020FC
S214447B20C01A4020BF1A4020BE1A4020C21A402025
S214447B30C31A4020C11A40202DE9F74F374D384E1E
S214447B40686806F005FF86F8C803A86806F000FFD4
S214447B50344986F8C903686906F02CFC324906F0B5
S214447B60E5FD06F0F5FE8346A86906F0F1FE2D49CC
S214447B700446E86906F01EFC2B4906F0D7FDCBF315
S214447B80090B06F0E5FE8246286A06F0E1FE254922
S214447B908146686A06F00EFC234906F0C7FD06F0E7
S214447BA0D7FE8046A86A06F0D3FE1E4900F00107B9
S214447BB0E86806F0FFFB1C4906F0B8FD06F0C8FE70
S214447BC0C0F309032869019306F0C2FE019B00F046
S214447BD0010043EA8023B6F8CA0300F4784003431E
S214447BE01248A6F8CA33A30200EACA2A03F48063FA
S214447BF04FEA495043EA0B0300F4001043EA0A03F1
S214447C00034343EA8853C6F8CC3396F8D03367F335
S214447C10000386F8D03303B0BDE8F08FF04440202C
S214447C209073402066667241CDCC4C3D00F81F00F0
S214447C303A4B4FF084412DE9F047394E1B7886F88D
S214447C40D433384B1B7886F8D533374B186806F050
S214447C50B1FB4FF0834106F0B5FC06F079FE334B9A
S214447C600446334993F800A0324B0AF0010A1868D8
S214447C7006F0A0FB304906F059FD06F069FE2F4B8E
S214447C8081462F4993F800802E4B08F00108186867
S214447C9006F090FB2C4906F049FD06F059FE2B4BA6
S214447CA005464FF084411F78294BC5F30B0507F072
S214447CB00107186806F07EFB4FF0834106F082FC0D
S214447CC006F046FE234BC0F3090245EA073518780A
S214447CD0C4F3090300F0010043EA8A2342EA8022FF
S214447CE0B6F8D60300F4784002431B4800EAC92994
S214447CF0A6F8D623D6F8D82343EA090302F07F42EF
S214447D0043EAC8531343C6F8D833B6F8DC3303F40F
S214447D1060431D43A6F8DC53BDE8F087191B40209A
S214447D2090734020181B40200C1B4020081B40200A
S214447D3033336F41041B40200AD7233C001B4020AA
S214447D40CDCCCC42FC1A4020CDCC4C3DFA1A402037
S214447D50141B4020101B402000F87F00264B274968
S214447D6010B5274C1B7884F8E033264B186806F089
S214447D70DDFC06F0EDFD244A244B03EA402310685C
S214447D80D4F8E023000200F48070034320481040F7
S214447D90204A03431268C4F8E03312021E4B02F42E
S214447DA080721B7884F8E4331C4B1B685B0203F434
S214447DB0C06313431A4A1268D20202F4C0521343F1
S214447DC0184A1268520302F400521343164A1268C1
S214447DD0920302F480421343144A1268D20302F414
S214447DE0C0321343D4F8E42322F4FF3222F48072E0
S214447DF01343C4F8E43310BDD81D4020CDCCCC3D4D
S214447E00907340209C1D4020A01D402000FEFF0192
S214447E10FF0000FE981D4020D91D4020941D4020A0
S214447E20901D40208C1D4020881D4020841D4020ED
S214447E3070B5194C194D26682946304606F07EFD25
S214447E4008B1256006E0164D3046294606F058FD32
S214447E500028F6D1134B144D1B68144A85F8E833B2
S214447E60134B12781B68134985F8E93395F8EC33BD
S214447E7062F3000385F8EC33206806F09BFA0E495B
S214447E8006F054FC05F0F0FE0AF04AFD06F0F4F95C
S214447E90A5F8EA0370BD00BFCC1A40200000D743C3
S214447EA00000D7C3D41A402090734020C81A4020FC
S214447EB0D01A402000C023440AD7A33C0C4B0D4A9A
S214447EC01B680D4982F8F0330C4B09781B6801F0A7
S214447ED0030182F8F1330A4B1B789B0003F00C0332
S214447EE00B430849097843EA011382F8F233704792
S214447EF0241B4020907340201E1B4020201B402003
S214447F001D1B40201C1B40200D4B0E4A1B780E495F
S214447F1082F8F4330D4B09781B7801F0010182F89E
S214447F20F5330B4B1B785B0003F002030B4392F8CC
S214447F30F61321F003010B4382F8F633704700BF73
S214447F40471B402090734020451B4020461B402042
S214447F50441B4020084A094B1278094983F8F82301
S214447F60084A0978127883F8F92393F8FA2361F3D8
S214447F70000283F8FA237047DA1A402090734020B0
S214447F80D81A4020D91A402038B50C4B0C4C5D68A2
S214447F90284605F069FE0AF0C3FC06F095F909493F
S214447FA0C4F80C04284606F0C1FB05F05DFE0AF052
S214447FB0B7FC06F089F9C4F8080438BDF0444020FC
S214447FC0907340200000084208B5FEF7F1FAFEF729
S214447FD031FBFEF76BFBFEF79FFBFEF7D3FBFEF78A
S214447FE0A1FCFEF7D1FCFEF74DFDFEF795FDFEF72E
S214447FF0E5FEFEF727FFFEF75FFFFEF78BFFFEF773
S214448000D9FFFFF70DF8FFF741F8FFF775F8FFF7CC
S214448010A9F8FFF7F7F8FFF743F9FFF777FBFFF701
S21444802025FCFFF705FEFFF7AFFFFEF7BBFDFFF7A6
S21444803065F9FFF7BFF9FFF711FAFEF7CDFDBDE886
S2144480400840FEF7EBBDF8B5254B264C1B78264F6B
S21444805084F81034254B1B7884F81134244B187854
S214448060323006F05BFA014606F0A4F906F070FCDE
S214448070204984F812040E781F493F780D781F492A
S21444808007F001071E4B08781E491A7830300978E5
S2144480901D4B49001B7801F03E01394394F8137494
S2144480A027F03F07394384F8131403F03F0102F0E6
S2144480B01F0306F00F0243EA411343EAC22305F0C6
S2144480C03F0243EAC23300F03F0243EA4253D4F845
S2144480D0142402F078421343C4F81434F8BD00BFA5
S2144480E0BD1A402090734020BA1A4020BC1A402043
S2144480F0BB1A4020B61A4020B51A4020B41A402075
S214448100B81A4020B91A4020B71A402008B5FFF7DD
S214448110B1FCBDE80840FFF796BF2DE9F74F384D50
S214448120384E686806F014FC86F81804A86806F00A
S2144481300FFC354986F81904686906F03BF933495B
S21444814006F0F4FA06F004FC8346A86906F000FC40
S2144481502D490446E86906F02DF92C4906F0E6FA5E
S214448160CBF3090B06F0F4FB8246286A06F0F0FBD4
S21444817025498146686A06F01DF9244906F0D6FA70
S21444818006F0E6FB8046A86A06F0E2FB1E4900F0CD
S2144481900107E86806F00EF91C4906F0C7FA06F02F
S2144481A0D7FBC0F309032869019306F0D1FB019B72
S2144481B000F0010043EA8023B6F81A0400F478403D
S2144481C003431348A6F81A34A30200EACA2A03F45F
S2144481D080634FEA495043EA0B0300F4001043EA35
S2144481E00A03034343EA8853C6F81C3496F82034FB
S2144481F067F3000386F8203403B0BDE8F08F00BF71
S214448200F04440209073402066667241CDCC4C3D8D
S21444821000F81F000C4B0D4A1B780D4982F82C348D
S2144482200C4B09781B7801F0030182F82D340A4B75
S2144482301B789B0003F00C030B430849097843EA78
S214448240011382F82E347047A01A402090734020C1
S2144482509E1A40209F1A40209D1A40209C1A402077
S21444826070B5194C194D26682946304606F066FB0B
S21444827008B1256006E0164D3046294606F040FB18
S2144482800028F6D1134B144D1B68144985F8243442
S214448290134B20681B6885F8253406F08BF8114983
S2144482A006F044FA05F0E0FC0AF03AFB05F0E4FF79
S2144482B00D4A95F828341278A5F8260462F300038C
S2144482C085F8283470BD00BFA81A40200000C84373
S2144482D00000C8C3B01A40209073402000C0234416
S2144482E0AC1A40200AD7A33CA51A40200D4B0E4A90
S2144482F01B780E4982F830340D4B09781B7801F010
S214448300010182F831340B4B1B785B0003F0020307
S2144483100B4392F8321421F003010B4382F83234B3
S214448320704700BFA41A402090734020A21A4020F1
S214448330A31A4020A11A402070B5194C194D26683E
S2144483402946304606F0FAFA08B1256006E0164D8E
S2144483503046294606F0D4FA0028F6D1134B144D7D
S2144483601B68144985F83434134B20681B6885F819
S214448370353406F01FF8114906F0D8F905F074FCB8
S2144483800AF0CEFA05F078FF0D4A95F8383412789C
S214448390A5F8360462F3000385F8383470BD00BF90
S2144483A0901A40200000C8430000C8C3981A4020D2
S2144483B09073402000C02344941A40200AD7A33C1C
S2144483C08C1A40200D4B0E4A1B780E4982F83C34DA
S2144483D00D4B09781B7801F0010182F83D340B4BB4
S2144483E01B785B0003F002030B4392F83E1421F023
S2144483F003010B4382F83E34704700BF8B1A40207B
S21444840090734020891A40208A1A4020881A4020B7
S2144484100C4B0D4A1B680D4982F840340C4B0978C6
S2144484201B6801F0030182F841340A4B1B789B0019
S21444843003F00C030B430849097843EA011382F816
S21444844042347047841A4020907340207E1A40205D
S214448450801A40207D1A40207C1A402008B5FFF739
S214448460B4F8FFF7E9F9FFF721FAFFF771FAFFF7D7
S214448470B5FAFFF7D9FAFFF75FFBFFF76FFCFFF794
S214448480D7FCFFF71BFDFFF73FFDFFF763FDFFF744
S21444849044FEFFF7E5FEFFF729FFFFF7BBFEFFF7B5
S2144484A04BFFFFF78FFFBDE80840FFF7B1BF7047AB
S2144484B07047704770470E4A92F8291092F8283051
S2144484C001F0030043EA0023C1F38100C1F3011124
S2144484D043EA802343EA013392F82A1043EA81337D
S2144484E0D2F80413890D89050B43C2F80433704748
S2144484F09073402010B5114C1149D4F8000205F091
S21444850059FF104906F012F905F0AEFB0AF008FAD6
S21444851005F0B2FE0C49A4F80803D4F8F40105F0BB
S21444852049FF0A4906F002F905F09EFB0AF0F8F9FD
S21444853005F0A2FEA4F80A0310BD00BF90734020C5
S21444854000C023440AD7A33C00C0CC44CDCC4C3D09
S21444855010B5114C1149D4F8940105F02BFF10497D
S21444856006F0E4F805F080FB0AF0DAF905F084FE3C
S2144485700C49A4F81003D4F8880105F01BFF0A49F7
S21444858006F0D4F805F070FB0AF0CAF905F074FE5C
S214448590A4F8120310BD00BF9073402000C02344CB
S2144485A00AD7A33C00C0CC44CDCC4C3D7047704762
S2144485B010B5114C1149D4F8700205F0FBFE104971
S2144485C006F0B4F805F050FB0AF0AAF905F054FE9C
S2144485D00C49A4F81803D4F8780205F0EBFE0A49CF
S2144485E006F0A4F805F040FB0AF09AF905F044FEBC
S2144485F0A4F81A0310BD00BF9073402000C0234463
S2144486000AD7A33C00C0CC44CDCC4C3D10B5114C4D
S2144486101149D4F87C0205F0CDFE104906F086F8E0
S21444862005F022FB0AF07CF905F026FE0C49A4F876
S2144486302003D4F8840205F0BDFE0A4906F076F815
S21444864005F012FB0AF06CF905F016FEA4F82203B6
S21444865010BD00BF9073402000C023440AD7A33CFB
S21444866000C0CC44CDCC4C3D10B5114C1149D4F887
S214448670700205F09FFE104906F058F805F0F4FA2B
S2144486800AF04EF905F0F8FD0C49A4F89802D4F81F
S214448690780205F08FFE0A4906F048F805F0E4FA39
S2144486A00AF03EF905F0E8FDA4F89A0210BD00BFB2
S2144486B09073402000C023440AD7A33C00C0CC4457
S2144486C0CDCC4C3D10B5114C1149D4F87C0205F084
S2144486D071FE104906F02AF805F0C6FA0AF020F9A9
S2144486E005F0CAFD0C49A4F8A002D4F8840205F0AB
S2144486F061FE0A4906F01AF805F0B6FA0AF010F9CF
S21444870005F0BAFDA4F8A20210BD00BF9073402045
S21444871000C023440AD7A33C00C0CC44CDCC4C3D37
S21444872008B5FFF7A1FFFFF7CDFFFFF7C4FEFFF73D
S214448730E1FEFFF70DFFFFF73BFFBDE80840FFF7FC
S21444874065BF70B5184C194D26682946304606F064
S214448750F5F808B1256006E0154D3046294606F082
S214448760CFF80028F6D1134B134C1B68134984F8F2
S214448770E833134B606E1B6884F8E93305F01AFE41
S214448780104905F0D3FF05F06FFA0AF0C9F805F072
S21444879073FD0D4A94F8EC331278A4F8EA0362F3B6
S2144487A0000384F8EC3370BDCC1A40200000D74355
S2144487B00000D7C3D41A40209073402000C02344FE
S2144487C0D01A40200AD7A33CC81A4020FFF7C0B8A6
S2144487D0704770470B4AD2F8A832D2F8D8101B0D0F
S2144487E0C1F313011B050B43D2F8DC10C2F8A832C0
S2144487F001F47F11D2F8AC3223F47F130B43C2F852
S214448800AC3270479073402008B50A4B50200A4A51
S214448810D3F8881293F88C322832116008211371E9
S214448820F9F72CFA054B002093E80600BDE808400B
S214448830FBF7DCBE90734020D8774020EC4F4600D0
S214448840094B00200949D3F8902293F894328A625F
S21444885003F0F002C3F30303134381F82F30044BB1
S21444886093E80600FBF7C2BE90734020D8774020BA
S214448870F44F4600094B00200949D3F8982293F850
S2144488809C328A6203F0F002C3F30303134381F875
S2144488902F30044B93E80600FBF7A8BE90734020A5
S2144488A0D8774020FC4F4600094B00200949D3F8AE
S2144488B0A02293F8A4328A6203F0F002C3F30303BF
S2144488C0134381F82F30044B93E80600FBF78EBE23
S2144488D090734020D877402004504600254A2649C5
S2144488E092F8A832C3F3010003F0FC03034310B428
S2144488F081F8283092F8A932C3F3010003F0FC0350
S214448900034392F8AA0281F82930C0F3010400F028
S2144489100C0323438409C0F3011081F82A3092F8EB
S214448920AB3203F003039B0143EA8403034381F819
S2144489302B3092F8AC3281F82C3092F8AD3203F0FA
S2144489403800C3F30203034381F82D3092F8AE3265
S214448950C3F38300D2F8AC32C3F3833343EA001341
S214448960002081F82F30054B10BC93E80600FBF737
S2144489703DBE00BF90734020D87740200C50460040
S2144489800B490C4A91F8B032C3F3010003F0FC03E0
S2144489900343002082F8283091F8B132C3F3010330
S2144489A082F82930044B93E80600FBF71FBE00BF4D
S2144489B090734020D87740202C5046001049114AE6
S2144489C091F8B432C3F3000003F0FE03034382F885
S2144489D0283091F8B53203F07C00C3F30103034317
S2144489E0002082F82930D1F8B432C3F3CF3353850C
S2144489F0D1F8B832D362044B93E80600FBF7F6BDD1
S214448A0090734020D877402014504600064A0020F1
S214448A10064BD2F8BC12D2F8C0229962DA62044BF2
S214448A2093E80600FBF7E2BD90734020D8774020D9
S214448A301C5046001149124A91F8C83210B482F8C4
S214448A40283091F8C932C3F3010403F01C00C3F381
S214448A504113204382F82900D1F8C802C0F3C1303C
S214448A6043EA8003002082F82A30D1F8CC32D3621D
S214448A70044B10BC93E80600FBF7B8BD9073402047
S214448A80D877402024504600084B002093F8D03234
S214448A9003F00402C3F301031343054A82F8283063
S214448AA0044B93E80600FBF7A1BD00BF907340203B
S214448AB0D8774020345046000A4A00200A4BD2F861
S214448AC0D41292F8D822996283F82C2083F82D2069
S214448AD083F82E2083F82F20044B93E80600FBF7F8
S214448AE085BD00BF90734020D87740203C50460058
S214448AF00B4B00200B4AD3F8DC129162B3F8E01219
S214448B0093F8E232918503F00801C3F302030B4362
S214448B1082F82E30044B93E80600FBF767BD00BF8F
S214448B2090734020D877402044504600284829492E
S214448B3090F8E43201F5FE5270B5C3F3010403F035
S214448B40FC032343137090F8E532C3F3010403F0A7
S214448B50FC03234341F6C1740B5541F6C27390F8A7
S214448B60E6422501A609C4F30114CD5490F8E75211
S214448B7005F00303C5F381051B0143EA860323433B
S214448B8041F6C37443EA85130B5541F6C47390F813
S214448B90E842CC5441F6C57490F8E93290F8EA02BB
S214448BA01D01C3F3031300F00F000D5543EA0013F1
S214448BB041F6C7700B5408214FF4AE60F9F7C7F975
S214448BC0054B012093E80600BDE87040FBF70EBD58
S214448BD090734020D87740204C5046002D4991F859
S214448BE0EC0238B5C0F3001500F008032A4C43EAFB
S214448BF04513C0F3020504F5FE522B43C0F340155B
S214448C00C0F3801043EA851343EAC01341F6C170AB
S214448C101370B1F8EC32C3F3C713235441F6C27051
S214448C20D1F8EC32C3F3C733235491F8EF02C0F3C0
S214448C30C103C0F34105C0F341101B0143EA850359
S214448C40B1F8EE52C5F3C1152B4343EA801341F6FF
S214448C50C370235441F6C47091F8F0329B002354F9
S214448C6091F8F132C3F38300B1F8F03241F6C7719C
S214448C70C3F3831343EA00134FF4B06063540821EC
S214448C80F9F765F9054B012093E80600BDE838403E
S214448C90FBF7ACBC90734020D87740205450460035
S214448CA01149124B01F5FE52D3F8F40210B5B3F84D
S214448CB0F842106041F6C47093F8FA320C5203F04E
S214448CC0F000C3F30303034341F6C7700B54082173
S214448CD04FF4B260F9F73BF9054B012093E80600E0
S214448CE0BDE81040FBF782BCD87740209073402004
S214448CF05C5046001749184891F8FC3200F5FE527D
S214448D0010B5137041F6C174D1F8FC32C3F309238D
S214448D10035541F6C274B1F8FE32C3F381030355DA
S214448D2091F8003303F00F0491F8FF3241F6C7710F
S214448D30C3F3830343EA04134354082140F28550A3
S214448D40F9F705F9054B012093E80600BDE8104005
S214448D50FBF74CBC90734020D877402064504600C4
S214448D601849194891F8043300F5FE5210B5C3F378
S214448D70010403F0FC032343137091F8053303F016
S214448D803C04C3F30103234341F6C174035591F8ED
S214448D900633C3F38304D1F8043341F6C771C3F3EF
S214448DA0833343EA04134354082140F28550F9F7C9
S214448DB0CEF8064B012093E80600BDE81040FBF7CA
S214448DC015BC00BF90734020D87740206C504600B6
S214448DD008B50E480E4B00F5FE52D3F8081393F828
S214448DE00C33116003F0F001C3F303030B4341F665
S214448DF0C771435408215020F9F7A9F8054B0120C0
S214448E0093E80600BDE80840FBF7F0BBD87740205F
S214448E10907340207450460008B50E480E4B00F53B
S214448E20FE52D3F8101393F81433116003F0F00194
S214448E30C3F303030B4341F6C7714354082151203F
S214448E40F9F785F8054B012093E80600BDE808408D
S214448E50FBF7CCBBD8774020907340207C5046002C
S214448E6008B50E480E4B00F5FE52D3F8181393F887
S214448E701C33116003F0F001C3F303030B4341F6C4
S214448E80C771435408216020F9F761F8054B012067
S214448E9093E80600BDE80840FBF7A8BBD877402017
S214448EA0907340208450460008B50E480E4B00F59B
S214448EB0FE52D3F8201393F82433116003F0F001E4
S214448EC0C3F303030B4341F6C7714354082161209F
S214448ED0F9F73DF8054B012093E80600BDE8084045
S214448EE0FBF784BBD8774020907340208C504600D4
S214448EF01B4938B51B4CD1F8283304F5FE52B1F85B
S214448F002C03136041F6C473E05291F82E33C3F336
S214448F104100C3F3C1050543C3F30000C3F3401344
S214448F2040EA850040EA430341F6C670235491F86C
S214448F302F33C3F38300B1F82E3341F6C771C3F31E
S214448F40831343EA0013132063540821F8F7FFFF02
S214448F50054B012093E80600BDE83840FBF746BBC6
S214448F6090734020D8774020945046001E4B1F49AB
S214448F7093F8300301F5FE5210B500F0F004C0F348
S214448F8003002043107093F8310300F07004C0F3DC
S214448F900300204341F6C174085541F6C274D3F821
S214448FA03003C0F3C130085541F6C374B3F83203F6
S214448FB0C0F34700085593F8340393F8333300F06E
S214448FC00F00C3F3430343EA001341F6C7700B5440
S214448FD008211420F8F7BBFF054B012093E8060050
S214448FE0BDE81040FBF702BB90734020D877402082
S214448FF09C504600154B164903F5FE5291F838032B
S21444900010B51070002441F6C1701C5441F6C2706D
S214449010B1F83A431C5241F6C470B1F83C4391F857
S2144490203E131C5201F0F000C1F30301014341F624
S214449030C770195408211520F8F789FF054B0120FD
S21444904093E80600BDE81040FBF7D0BAD877402036
S21444905090734020A4504600194B1A4A03F5FE511B
S214449060B2F84003088092F8441301F0F000C1F3CC
S2144490700301014341F6C270195441F6C37192F894
S2144490804503585441F6C47092F84813195441F6AF
S214449090C570195492F84C1301F0F000C1F3030163
S2144490A0014341F6C6701954012092F84D1341F617
S2144490B0C7729954044B93E80600FBF797BA00BF6F
S2144490C0D877402090734020AC504600194B1A4A3B
S2144490D003F5FE51B2F85003088092F8541301F099
S2144490E0F000C1F30301014341F6C270195441F63E
S2144490F0C37192F85503585441F6C47092F8581305
S214449100195441F6C570195492F85C1301F0F000F6
S214449110C1F30301014341F6C6701954012092F885
S2144491205D1341F6C7729954044B93E80600FBF767
S2144491305DBA00BFD877402090734020B4504600B4
S214449140174B184A03F5FE51B2F86003088092F8AC
S214449150641301F0F000C1F30301014341F6C27009
S214449160195441F6C370D2F868131954090A41F6E3
S214449170C470195492F86C1301F0F000C1F3030163
S214449180014341F6C6701954012092F86D1341F616
S214449190C7729954044B93E80600FBF727BA00BFFE
S2144491A0D877402090734020BC50460010B51249F2
S2144491B00020124C01F5FE52D4F87033136041F689
S2144491C0C473C85494F87533C3F34300B4F8743383
S2144491D0C3F3431343EA001341F6C7700B54082104
S2144491E01620F8F7B4FE064B012093E80600BDE8C7
S2144491F01040FBF7FBB900BFD8774020907340205F
S214449200C4504600FFF7D2BF08B5F9F77AF8FEF720
S214449210D5F9BDE80840FFF7C9BF3048304A90F852
S2144492207C3390F8781370B543F6587590F87F43BE
S214449230535543F65973D15443F65A71D0F878339C
S214449240C3F34F235BBA5352C4F3801304F01001A4
S21444925041EAC301C4F30103194390F8793303F098
S214449260010341EA4311C4F3810304F0200441EAB4
S214449270831143F65C73D15490F88013C1F380068F
S21444928001F00803C1F3010143EA06130B4390F8C7
S2144492907E13D0F87C032343CC09C1F3801143EA00
S2144492A0841343F65D741355C0F30D2343F65E747E
S2144492B0C0F305409B001055642043EA410343F63F
S2144492C05F7153542A440821F8F7D8FC054B022012
S2144492D093E80600BDE87040FBF788B990734020D9
S2144492E0D8774020CC50460038B52C4B43F65870BF
S2144492F02B4AB3F88413B3F88C5349BA115293F8F3
S2144493008A13CC09C5F3032141EA041193F88D432B
S214449310C4F3001441EA441193F88743C4F3800429
S21444932041EA841193F88943C4F3800441EAC411A2
S21444933043F65A74115543F65B71B3F88643555455
S21444934043F65C71C4F30905C4F387045454B3F874
S2144493508813D3F88833C1F30904C1F3051141EAED
S214449360851143F65D755155C3F3CB21C3F3C3430F
S21444937043EA041343F65E74135543F65F73D154BD
S214449380024408217020F8F779FC064B022093E843
S2144493900600BDE83840FBF729B900BF907340206B
S2144493A0D8774020D45046000D4843F65872B0F85B
S2144493B0901308B549BA0B4B99521A4490F8921335
S2144493C043F65A70C901195403213220F8F756FC63
S2144493D0054B022093E80600BDE80840FBF706B9B3
S2144493E090734020D8774020DC504600094943F625
S2144493F05870094AD1F8A0331BBA13500220D1F84A
S214449400A43343F65C711BBA5350044B93E80600EE
S214449410FBF7ECB890734020D8774020E4504600E1
S2144494201F4843F658721F4BB0F8AA13C1F3C7112E
S21444943070B5995443F65974D0F8A8131A44B0F842
S214449440A853C1F3C731C5F30526195590F8AD4363
S21444945004F08001C4F38014314343F65A76995598
S21444946043F65B715D54B0F8AC5390F8A913C5F35A
S214449470052001F04001014343F65C7041EAC41103
S214449480195443F65D716A205D540621F8F7F6FBDD
S214449490054B022093E80600BDE87040FBF7A6B8EB
S2144494A090734020D8774020EC504600114B43F64A
S2144494B05870114AB3F8B01349BA10B5115243F66E
S2144494C05A74B3F8B21393F8B43349BA03F00103A9
S2144494D0115343F65C719B015354024405214020CA
S2144494E0F8F755FA054B022093E80600BDE810400D
S2144494F0FBF77CB890734020D8774020F450460061
S214449500134843F65872134BB0F8B81349BA10B51B
S21444951099521A4490F8BA1343F65A70C1F30104A8
S2144495201C54C1F3031443F65B70C1F381011C540D
S21444953043F65C70195405214FF45470F8F727FA33
S214449540054B022093E80600BDE81040FBF74EB8F2
S21444955090734020D8774020FC504600104843F68D
S2144495605871104A08B5B0F8BC335BBA535290F8F9
S214449570BE3303F00100C3F3400343EA400343F61B
S2144495805A7013540A444FF444700321F8F7FFF911
S214449590054B022093E80600BDE80840FBF726B8D2
S2144495A090734020D877402004514600254943F61E
S2144495B05872B1F8C00338B540BA234B91F8C34348
S2144495C098521A44D1F8C40304F00105C4F3440481
S2144495D0C0F3C53040EAC51043F65A75585543F6AD
S2144495E05B75B1F8C403C0F34510585543F65C7533
S2144495F091F8C403C0F304005855B1F8C603C0F349
S214449600022500F4FC6045EAC40443F65D755C55E7
S21444961091F8C543C4F3C304204343F65E74185517
S21444962091F8C20343F65F71585408214FF46170B1
S214449630F8F724FB054B022093E80600BDE83840C3
S214449640FAF7D4BF90734020D87740200C51460098
S214449650284A43F658702849B2F8C8335BBA30B43F
S2144496600B5243F65A73B2F8CA03B2F8CC53C0F35B
S2144496700904C0F38700C854C5F3012092F8CB33DD
S21444968003F00403034392F8CD03C0F3800043EA97
S214449690C00392F8CE03C0F3401043EA001392F896
S2144496A0D00300F0010043EA401343F65B7043EAFC
S2144496B0841343F65D740B5443F65C73D2F8CC03C0
S2144496C0CD54C0F3C923B2F8CE23C0F347309B0130
S2144496D00855900943EA923343F65E728B5443F638
S2144496E05F73C8540220054B30BC93E80600FAF773
S2144496F07DBF00BF90734020D87740201451460069
S21444970038B52C4B45F6F0602B4AB3F8D413B3F86F
S214449710DC5349BA115293F8DA13CC09C5F3032142
S21444972041EA041193F8DD43C4F3001441EA4411BA
S21444973093F8D743C4F3800441EA841193F8D94399
S214449740C4F3800441EAC41145F6F264115545F663
S214449750F361B3F8D643555445F6F461C4F30905AA
S214449760C4F387045454B3F8D813D3F8D833C1F3A6
S2144497700904C1F3051141EA851145F6F5655155CD
S214449780C3F3CB21C3F3C34343EA041345F6F66459
S214449790135545F6F763D154024408217120F8F76F
S2144497A06DFA064B032093E80600BDE83840FAF706
S2144497B01DBF00BF90734020D87740201C51460000
S2144497C008B5FFF721F8FFF73BF8FFF787F8FFF7F0
S2144497D0D7F8FFF7F3F8FFF719F9FFF72BF9FFF778
S2144497E087F9FFF7A3F9FFF75BFAFFF7F7F9FFF7F7
S2144497F081FAFFF7B5FAFFF7EBFAFFF70DFBFFF731
S2144498002FFBFFF751FBFFF773FBFFF7AFFBFFF7A9
S214449810F1FBFFF721FCFFF759FCFFF791FCFFF73C
S21444982063FDFFF76DFFFFF72FF9BDE80840FFF72C
S21444983043B908B5FCF76CFEF8F74AFDFEF7C4FBDF
S214449840FEF76EFFBDE80840FFF7BABF2248234A3A
S21444985090F8E01338B590F8E43345F6F0641355C1
S21444986045F6F163D15445F6F261D0F8E033C3F3DC
S2144498704F235BBA535290F8E513C1F34013C1F338
S21444988080151B0143EAC503C1F341052B4390F8F9
S214449890E15305F0010543EA4513C1F3C10501F060
S2144498A0010143EA851345F6F4655355D0F8E4338D
S2144498B06520C3F3C13343EA811145F6F563D154B9
S2144498C022440821F8F7DAF9054B032093E806000A
S2144498D0BDE83840FAF78ABE90734020D8774020D7
S2144498E024514600114B45F6F060114AB3F8E8138C
S2144498F049BA10B5115245F6F264B3F8EA1393F830
S214449900EC3349BA03F00103115345F6F4619B0165
S2144499105354024405214020F8F796F8054B03209B
S21444992093E80600BDE81040FAF760BE9073402006
S214449930D87740202C514600134845F6F062134B26
S214449940B0F8F01349BA10B599521A4490F8F21385
S21444995045F6F260C1F301041C54C1F3031445F602
S214449960F360C1F381011C5445F6F4601954052193
S2144499704FF45470F8F768F8054B032093E8060054
S214449980BDE81040FAF732BE90734020D8774020A6
S21444999034514600104845F6F061104A08B5B0F810
S2144499A0F4335BBA535290F8F63303F00100C3F332
S2144499B0400343EA400345F6F26013540A444FF426
S2144499C044700321F8F740F8054B032093E806005B
S2144499D0BDE80840FAF70ABE90734020D877402086
S2144499E03C5146000E4845F6F062B0F8F81308B508
S2144499F049BA0C4B99521A4490F8FA1345F6F26059
S214449A00C1F30001195403213320F8F737F9064B04
S214449A10032093E80600BDE80840FAF7E7BD00BF18
S214449A2090734020D877402044514600094945F673
S214449A30F060094AD1F808341BBA13500320D1F811
S214449A400C3445F6F4611BBA5350044B93E80600B5
S214449A50FAF7CCBD90734020D87740204C5146004E
S214449A60254945F6F062B1F8100438B540BA234BA0
S214449A7091F8134498521A44D1F8140404F001059A
S214449A80C4F34404C0F3C53040EAC51045F6F26555
S214449A90585545F6F365B1F81404C0F345105855C7
S214449AA045F6F46591F81404C0F304005855B1F82B
S214449AB01604C0F3022500F4FC6045EAC40445F6E7
S214449AC0F5655C5591F81544C4F3C304204345F644
S214449AD0F664185591F8120445F6F761585408216F
S214449AE040F28530F8F7CAF8054B032093E80600A1
S214449AF0BDE83840FAF77ABD90734020D8774020C6
S214449B005451460008B5FFF751FDBDE80840FFF73D
S214449B10A7BF08B5F8F7F7FBFEF7F8FABDE8084024
S214449B20FFF7F0BF284A45F6F0602849B2F81834E3
S214449B305BBA30B40B5245F6F263B2F81A04B2F884
S214449B401C54C0F30904C0F38700C854C5F301206D
S214449B5092F81B3403F00403034392F81D04C0F345
S214449B60800043EAC00392F81E04C0F3401043EA60
S214449B70001392F8200400F0010043EA401345F62F
S214449B80F36043EA841345F6F5640B5445F6F463F0
S214449B90D2F81C04CD54C0F3C923B2F81E24C0F333
S214449BA047309B010855900943EA923345F6F662DE
S214449BB08B5445F6F763C8540320054B30BC93E8F2
S214449BC00600FAF713BD00BF90734020D8774020B4
S214449BD05C514600114B47F68860114AB3F824148A
S214449BE049BA10B5115247F68A64B3F8261493F866
S214449BF0283449BA03F00103115347F68C619B019C
S214449C005354024405214020F7F77CFF054B0420BB
S214449C1093E80600BDE81040FAF7E8BC907340208D
S214449C20D877402064514600134847F68862134B61
S214449C30B0F82C1449BA10B599521A4490F82E1418
S214449C4047F68A60C1F301041C54C1F3031447F673
S214449C508B60C1F381011C5447F68C60195405216E
S214449C604FF45470F7F74EFF054B042093E8060074
S214449C70BDE81040FAF7BABC90734020D87740202D
S214449C8074514600104847F68861104A08B5B0F843
S214449C9030345BBA535290F8323403F00100C3F3C5
S214449CA0400343EA400347F68A6013540A444FF499
S214449CB044700321F7F726FF054B042093E806007B
S214449CC0BDE80840FAF792BC90734020D87740200D
S214449CD06C51460008B50A4B49F6226209494020B1
S214449CE0B3F836345BBA8B520521074AF7F768FF58
S214449CF0064B052093E80600BDE80840FAF776BC14
S214449D0090734020D8774020F81541207C51460077
S214449D10134849F62062134BB0F8401449BA10B5BC
S214449D2099521A4490F8421449F62260C1F3010449
S214449D301C54C1F3810449F62360C1F303111C5437
S214449D4049F62460195405214FF45470F7F738FF48
S214449D50054B052093E80600BDE81040FAF746BCDC
S214449D6090734020D87740208C514600104849F6DE
S214449D702061104A08B5B0F83C345BBA535290F8A8
S214449D803E3403F00100C3F3400343EA400349F67C
S214449D90226013540A444FF444700321F7F710FF2B
S214449DA0054B052093E80600BDE80840FAF71EBCBC
S214449DB090734020D87740208451460008B5FFF77A
S214449DC02CFAFFF7F1FAFFF72BFBFFF76FFBFFF7D1
S214449DD097FBFFF7C3FBFFF739FDFFF783FDFFF75C
S214449DE0ABFDFFF7D7FDFFF7FDFDFFF7F3FEFFF7EB
S214449DF049FFFFF719FFFFF76DFFFFF7B7FFBDE811
S214449E000840FFF785BF08B5FCF7BCFBF8F75EFAD9
S214449E10FEF724FBBDE80840FFF7D0BF08B5F9F7C6
S214449E2085FCBDE80840F8F70DBE7047F8F74CBA15
S214449E30FFF7E9BFFFF7FDBCFAF7F4BB7047074AE4
S214449E401378632B96BF01330023DBB21370044AA6
S214449E50136801331360FFF7D7B900BF703541204C
S214449E60901F402008B5FAF7DFFBBDE80840F7F737
S214449E70CDBC08B5FFF74DFE4CF24053044AD058CB
S214449E80B0FA80F0BDE808404009F9F7C9BC00BF05
S214449E9074354120014900201AF03ABE107246003B
S214449EA000201AF039BE0022114610461AF038BE79
S214449EB0704700BF0000000038B5294D2A78012AB3
S214449EC01ED1284B284C186803F0CEFE274BC4E915
S214449ED0000118681EA3D3E90023C4E9042340F212
S214449EE0DB53984225D903F09DFEC4E9020101F0F4
S214449EF039F91F4BD3E9000104F006FA1D4B1860EC
S214449F002B781D4C022B1DD123680BB1012B16D187
S214449F101A4B1B686360022323601949606804F087
S214449F2051FBA16804F04EFB164B1860164B1860A4
S214449F3007E009A3D3E90023C4E90223D7E7022BA9
S214449F40EBD038BD00232360FBE700BFAFF30080AF
S214449F5000000000007097C00000000000709740AA
S214449F602E1E4020F81C402078FC412080174020BC
S214449F7090FC4120F41C4020981F40202C1D40207B
S214449F8000002041D01D40209C1D4020224B1B68D1
S214449F9043B9224A07211160214A13600122214B0A
S214449FA01A6008E0012B22D102231C4A13601C4A83
S214449FB013601C4A13601C4A1C49106850B90B684D
S214449FC0012B07D11A4803601A4803601A480360F5
S214449FD01A4803601A4B1B6813605022194B1B78AF
S214449FE00B60194B1A60194B194A1A607047022BBA
S214449FF006D10A4A032111600021094A1160D8E7B4
S21444A000032BD8D1054B04221A600122044B1A6054
S21444A0100222044BC4E700BF4C1D4020701D402064
S21444A0206C1D4020501B4020681D4020641D40206D
S21444A030741D4020781D40207C1D4020801D4020FB
S21444A040181D4020CE184020601D40205C1D402036
S21444A050000048C208B50C4B1B6853B90B4B1B6831
S21444A060012B07D10A4B0B49186804F0ABFA0A4B8C
S21444A070186008BD002BFCD1084B18680523B0FBBC
S21444A080F3F004F047FAF2E7481D4020B01B4020A6
S21444A09090184020000020411C1E40209418402068
S21444A0A0104B70B51D68104C25F00045616825605E
S21444A0B0084604F07FF9A16804F084FA0646E1688D
S21444A0C0284604F033FB0146304604F07BFA074941
S21444A0D004F078FA064904F029FB064B2061186020
S21444A0E070BD00BF78194020A81F40200000704271
S21444A0F000007A442C1D402038B5204D204C286D55
S21444A10003F0B2FD1F4B1B78C4E90001002B32D18B
S21444A110686D03F0A9FDC4E90201286E03F0A4FDAE
S21444A120C4E9040195F86C0003F07CFDC4E906011B
S21444A130686FC0F3C72003F075FDC4E9080195F8BD
S21444A140C20203F06FFDC4E90A0195F87400C0F337
S21444A150830003F067FDC4E90C010B4CD4E900010D
S21444A16004F0D2F8094B1860D4E9020104F0CCF8A4
S21444A170074B186038BD00200021CCE79073402080
S21444A180F8FA4120321E402040FC41207C174020F3
S21444A1901C1E402038B51F4D1F4C286D03F064FD2F
S21444A1A01E4B1B78C4E90001002B2FD1686D03F0C9
S21444A1B05BFDC4E90201B5F8C40003F033FDC4E90D
S21444A1C0040195F8BC0003F02DFD0022144BC4E9AD
S21444A1D00601C4E9082395F8C20203F023FDC4E946
S21444A1E00A0195F8D400800903F01CFDC4E90C016B
S21444A1F00C4CD4E9000104F087F80B4B1860D4E902
S21444A200020104F081F8094B186038BD0020002193
S21444A210CFE700BF90734020F8FA4120321E40201A
S21444A2200000444040FC41207C1740201C1E402037
S21444A2302DE9F04FDFF8ACA29FB0DAE90845DAE939
S21444A24006672046294632463B4603F0E1FF08B9F6
S21444A25034463D4620462946DAE94A6732463B4676
S21444A26003F0A2FB804689467FA3D3E9002303F08C
S21444A270E3FF002800F0CB80304639467AA3D3E982
S21444A280002303F093FB04460D46DAE90C23CAE99F
S21444A2904A45CDE90023DDE900010022002303F00E
S21444A2A0A3FF0646002840F0C48000224FF08043B7
S21444A2B0DDE9000103F098FF88B90022844BDDE90C
S21444A2C0000103F091FF002840F0B5800022814B46
S21444A2D0DDE9000103F088FF061E18BF01260022B0
S21444A2E07D4B2046294603F017FD61A3D3E900239E
S21444A2F003F03CFE60A3D3E9002303F00DFD0022E7
S21444A300764B03F009FD5EA3D3E9002303F02EFE4B
S21444A31004460D46304603F095FC22462B4603F091
S21444A320FBFC02460B46DAE94C45CDE904232246BB
S21444A3302B4603F039FB06460F4653A3D3E90023C6
S21444A34003F07AFF002879D0204629464EA3D3E965
S21444A350002303F02BFBCDE90401DDE90434DDE9F9
S21444A3600401CAE94C34DAE91E2303F01FFB48A370
S21444A370D3E9002303F0D0FC04460D4646A3D3E9B4
S21444A3800023DAE9200103F0C7FC02460B462046C8
S21444A390294603F00BFB42A3D3E9002303F0E6FD72
S21444A3A002460B46CDE90223DAE9002303F0FCFA21
S21444A3B000224B4B04460D4603F03EFF002840F077
S21444A3C014842046294638A3D3E9002303F016FF15
S21444A3D000223F4B002840F01584DDE9000103F0DD
S21444A3E003FF00283BD100223A4BDDE9000103F08D
S21444A3F0FBFE061E18BF01260022002320462946DF
S21444A40003F01AFF002873D12046294672E028A399
S21444A410D3E900234046494603F0F0FE00283FF4C3
S21444A42034AF3046394624A3D3E9002303F0BCFABC
S21444A43029E7002653E74FF0FF3650E720A3D3E939
S21444A44000233046394603F0D9FE002885D02046FE
S21444A45029461DA3D3E9002303F0A6FA7BE74FF071
S21444A460FF36C9E7AFF30080FCA9F1D24D62703FD6
S21444A470000000000020AC405C8FC2F528DC27407A
S21444A480B46155D0CC38FB3F9A9999999999D93F5C
S21444A490FCA9F1D24D62603FB428207983A6BA3F26
S21444A4A054434F56A8ACBB3F0000000000409FC03A
S21444A4B0FCA9F1D24D6280BFFCA9F1D24D62803F27
S21444A4C09A9999999999E9BF9A9999999999E93F45
S21444A4D00000F03F0000084000408F4000004E401F
S21444A4E000409F40F8FA41204FF0FF360024C44D08
S21444A4F000200021AAA3D3E9002303F00DFC8046E4
S21444A50089463046BF4E03F09DFB42464B4603F019
S21444A51003FC82468B46D6E94E8942464B4603F0B8
S21444A52043FA02460B46CDE906230022B64B03F017
S21444A53083FE0022002800F01483B34B404649466D
S21444A54003F034FA82468B464FF00008DFF8C09298
S21444A5505046594642464B46C6E94EAB03F06CFE5F
S21444A560002800F00D83C6E952890022A74B2046F6
S21444A570294603F061FE0022002800F01183A34B15
S21444A5802046294603F010FACDE906019D4CDDE944
S21444A5900201D4E9222303F007FA00229C4B03F07D
S21444A5A0BBFBD4E9242303F0FFF902460B46CDE96E
S21444A5B00823D4E9262303F0F7F90022944B03F04A
S21444A5C0ABFBD4E9282303F0EFF902460B46CDE96A
S21444A5D00A23D4E92A2303F0E7F900228C4B03F03C
S21444A5E09BFBD4E92C2303F0DFF96FA3D3E90023C4
S21444A5F0CDE91601DDE9020103F08EFB804689466B
S21444A6006BA3D3E90023DDE9080103F085FB42464A
S21444A6104B4603F0CBF906460F4667A3D3E900231F
S21444A620DDE90A0103F078FB02460B46304639461C
S21444A63003F0BCF9DDE9162303F0B8F960A3D3E9C7
S21444A640002303F069FBD4E92E23CDE90C01104620
S21444A650194603F0ABF9DDE90C2303F0A7F9D4E976
S21444A6600E2303F0A3F958A3D3E9002303F054FBC5
S21444A67006460F4656A3D3E90023D4E9300103F037
S21444A6804BFB02460B463046394603F08FF90646E6
S21444A6900F4651A3D3E90023D4E9120103F03CFB4F
S21444A6A002460B463046394603F07EF94CA3D3E9BE
S21444A6B0002303F05BFC02460B46CDE90E23D4E9A7
S21444A6C0322303F073F948A3D3E9002303F024FBB1
S21444A6D006460F4646A3D3E90023D4E9340103F0E3
S21444A6E01BFB02460B463046394603F05FF942A34D
S21444A6F0D3E9002303F03AFCD4E93623CDE9180124
S21444A700DDE9020103F050F90022414B03F004FB5B
S21444A710D4E9382303F048F902460B46CDE9102322
S21444A720D4E93A2303F040F90022394B03F0F4FA13
S21444A730D4E93C2303F038F902460B46CDE912230C
S21444A740D4E93E2303F030F90022314B03F0E4FA17
S21444A750D4E9402303F028F915A3D3E90023CDE92F
S21444A7601A01DDE9100103F0D7FA42464B4603F0DE
S21444A7701DF906460F4610A3D3E90023DDE912016E
S21444A78003F0CAFA02460B463046394603F00EF941
S21444A790DDE91A2303F00AF93CE000BFAFF300807A
S21444A7A09A9999999999E9BF9A99999999996340E7
S21444A7B09A99999999996A40CDCCCCCCCCCC3540D1
S21444A7C0E3F36EFB79D0E33E277845D92444D93F5A
S21444A7D0FB50D7647BD71C403043BB3975F10440EB
S21444A7E06D0D4BFEC9AF1840FCA9F1D24D62603FD7
S21444A7F0EBF33CDE4AA2813FE9C8B5C771D3893F33
S21444A80000409F40F8FA41200000084000004940BC
S21444A81000408F40AAA3D3E9002303F07DFAD4E98D
S21444A820502303F0C1F802460B46CDE91C23D4E975
S21444A830422303F0BBF8A4A3D3E9002303F06CFA45
S21444A84006460F46A2A3D3E90023D4E9440103F005
S21444A85063FA02460B463046394603F0A7F89EA3F1
S21444A860D3E9002303F082FB82468B46D4E9462391
S21444A8701046194603F09AF852465B4603F096F89B
S21444A880D4E9162303F092F895A3D3E9002303F002
S21444A89043FA06460F4694A3D3E90023D4E9480175
S21444A8A003F03AFA02460B463046394603F07EF841
S21444A8B006460F468EA3D3E90023D4E91A0103F0D3
S21444A8C02BFA02460B463046394603F06DF88AA307
S21444A8D0D3E9002303F04AFB00228F4BCDE9140151
S21444A8E0D4E90A452046294603F088FC002840F06F
S21444A8F069810022884B2046294603F055F880A3F8
S21444A900D3E9002303F008FA0022844B04460D469C
S21444A91003F088FC08B10024804D7BA3D3E90023D0
S21444A920DDE9140103F0F8F900227D4B884606461B
S21444A93003F064FC8146002840F047810022794BAE
S21444A9403046414603F078FC002840F04381B14647
S21444A95008F100486EA3D3E90023DDE9060103F0BD
S21444A960DBF9DDE9182303F021F806460F462246B4
S21444A9702B464846414603F0CFF932463B4603F061
S21444A98015F80022684B04460D4603F055FC002893
S21444A99040F023810022654B2046294603F02EFCD6
S21444A9A008B10024614D00220023DDE9000103F0D4
S21444A9B01BFC002840F0148100224FF08043DDE960
S21444A9C0000103F011FC002840F00A810022534B9A
S21444A9D0DDE9000103F008FC002840F00381002272
S21444A9E0534BDDE9000103F0FFFB003818BF01209C
S21444A9F003F028F922462B464E4F03F08DF9DDE945
S21444AA000423C7E95401C7E91E23DDE90223C7E945
S21444AA105045C7E92023C7E92223DDE90823C7E9CF
S21444AA202423C7E92623DDE90A23C7E92823C7E9FF
S21444AA302A23DDE91623C7E92C23DDE90C23C7E9DD
S21444AA402E23D7E91023C7E90E23DDE90C23C7E9F3
S21444AA501023DDE90E23C7E93023D7E91423C7E9D9
S21444AA601223DDE90E23C7E91423C7E93223DDE9BF
S21444AA701823C7E93423DDE90234C7E944ABC7E900
S21444AA803634DDE91034C7E946ABC7E93834C7E99C
S21444AA903A34DDE91234C7E93C34C7E93E34DDE9EB
S21444AAA01A34C7E94034DDE91C34C7E94234D7E9EF
S21444AAB01823C7E918ABC7E916233DE0AFF3008077
S21444AAC0E3F36EFB79D0E33EFCA9F1D24D62603FDE
S21444AAD05ED817C2038C9E3F6F216A9B4B52A13FA0
S21444AAE02ED7D19C0A49373F7119ABB745FF1F4053
S21444AAF0ECBC164D8E930F401988C921F33610408E
S21444AB009A9999999999C93FCDCCCCCCCCCCEC3F69
S21444AB103B08AA2A23DCA63F000014400000F03F6E
S21444AB2000003EC000003E4000005440000054C0B8
S21444AB3000000840F8FA4120DDE91434C7E94834F7
S21444AB40D7E91C23C7E91A23DDE91434C7E91C34C2
S21444AB501FB0BDE8F08F4FF0FF3631A5D5E900456C
S21444AB6052E4314BDDE9060103F048FB00283FF48C
S21444AB70EBAC00222D4B4046494602F015FFE1E47B
S21444AB804FF000084FF000095046594642464B469F
S21444AB9003F034FB00287FF4E6ACC6E952ABE4E4A9
S21444ABA0234B2046294603F03DFB30B90022214B77
S21444ABB02046294602F0FAFEE6E400230024CDE9C6
S21444ABC00634E3E400240025A7E64FF00009DFF846
S21444ABD07480BFE6DFF87080BCE60024164DE2E6DB
S21444ABE0002005E74FF0FF3002E70022134BDDE973
S21444ABF0000103F0F9FA00287FF476AC0024104DE7
S21444AC00FFF7F1BBDDE9000103F0EEFA0028A2D11C
S21444AC1003A5D5E90045FFF7E6BB00BFAFF30080C8
S21444AC200000000000409FC0000008C0000008402C
S21444AC30000049C000004940000054400000F03F76
S21444AC4000409F4000003E4000003EC0704700BFAA
S21444AC501C4B1B68012B1C4B07D01C4A1288012A2C
S21444AC6003D01B4A1268012A0CD102221A601B68C0
S21444AC70184A1370184B1B78013B012B21D8032329
S21444AC8013707047154A11681A68012903D1032ABC
S21444AC9001D10022EAE712480068012803D1032ABA
S21444ACA00AD11860E3E711B90AB90322DEE700289F
S21444ACB0DDD1012ADBD1F8E70029D8D1002AD6D144
S21444ACC0F3E77047B01C4020481D40201A1B402024
S21444ACD0601840202E1E4020EE1D40207018402054
S21444ACE0BC1C402008B5114A00231360104A136068
S21444ACF0104A1360104A136000F070FB0F4B1B8819
S21444AD006BB90F4B0F4A1B681268134307D10E4AA0
S21444AD1013600E4A13600E4A13600E4A13600023F3
S21444AD200D4A13600D4A136008BD00BFD01D402075
S21444AD301C1E4020A01740209C1740201A1B402071
S21444AD40B01C402060184020501C40204C1C402022
S21444AD50241C4020281C4020501D4020A41B40207A
S21444AD6010B500F0CEFA0F4B0F4C1A680F4B1A6012
S21444AD700F4B1A680F4B1A60226822F00202012A0F
S21444AD8001D1FFF707FA0C4B1B68012B1EBF0B4B78
S21444AD9000221A600A4B1B6823600A4B1A680A4B47
S21444ADA01A6010BD801840204C1D4020A01740203B
S21444ADB07C1840209C17402060184020A41B40204C
S21444ADC0641840208C184020D01D40202DE9F843BC
S21444ADD000F097FA3A4B3B4E4FF00008186802F0E2
S21444ADE043FF394B3746DFF8EC90C6E90001186854
S21444ADF002F018FF354B04460D46186802F034FF3F
S21444AE000022334B02F088FF02460B462046294672
S21444AE1002F0CAFD05460C4600222E4B2846214623
S21444AE2003F0ECF968B904F100434246284621464B
S21444AE3073614B46356103F0E1F938B1C7E90289DD
S21444AE4008E00022244BC6E90423F7E72A462346B3
S21444AE50C6E9022300F044F9204B0025D3E900015B
S21444AE6003F052FA1E4B18601E4B18601E4B1860B7
S21444AE701E4B1D601E4B1D60FFF73EF91D4B1A68A6
S21444AE801D4B1A60FFF718F81C4B29461C682046D1
S21444AE9003F02CFD08B11A4B1C681A4B1C601A4B65
S21444AEA01A681A4B1A601A4B1B68012B1EBF194BA3
S21444AEB000221A60184B1A68184B1A60BDE8F883CB
S21444AEC0EC1C402058FC4120841740202C1D402078
S21444AED000001A4000806140008061C070FC412040
S21444AEE0A0174020381B4020CC1A4020A81A4020E7
S21444AEF0901A4020EC174020341D4020F01C40207F
S21444AF00F41C4020D01D4020B81C40204C1D40203E
S21444AF10B01C4020501D4020A01C4020281D40202E
S21444AF20F8B50223104F114E3B6033600123104D99
S21444AF30104C2B60236000F051FA0F4B00221A602D
S21444AF400E4B1B887BB90E4B0E4A1B681268134384
S21444AF500D4A1268134306D103223B6033602B60CC
S21444AF6023600A4B1A60F8BD501C40204C1C4020FD
S21444AF70501D4020A41B40201C1E40201A1B40206D
S21444AF80B01C402060184020D41C4020481D40205F
S21444AF9008B5184B186803F001FD174B174A18609C
S21444AFA0012317491360174A1360174A12680A6048
S21444AFB016490B6016490A60164A17491370174A11
S21444AFC01370174A1370174A1370174A1370174AA8
S21444AFD0137000220A7016490A7016490B701649F7
S21444AFE00B7016490B7016490B70164B1A70164B9D
S21444AFF01A7008BD1C1E4020CC1D4020C81D402091
S21444B000C01D4020B81D40204C1D40208C1D4020B3
S21444B010941D4020541B4020451B4020D81A4020F5
S21444B020341B4020C81A4020491B4020481B40205F
S21444B030441B4020A51A4020A11A4020A21A4020B2
S21444B0408C1A4020881A4020891A402000230A4A35
S21444B05015211370094A1370094A11700621094ACA
S21444B0601370094A1370094A1170094A137018225A
S21444B070084B1A70704700BFC51A4020C41A4020B7
S21444B080C31A4020C21A4020C11A4020C01A402089
S21444B090BF1A4020BE1A402008B5FFF779FFFFF7D5
S21444B0A0D5FFFFF7D5FD0D4B1B781BB9BDE808400F
S21444B0B0FFF756BE012B03D1BDE80840FFF786BE16
S21444B0C0022B03D1BDE80840FFF72ABF032B03D168
S21444B0D0BDE80840FFF706BE08BD00BF2E1E402050
S21444B0E02DE9F047DFF878A01BA3D3E90023DAE97B
S21444B0F0020102F011FE04460D46DAE90689DAE951
S21444B100000142464B4602F04FFC06460F460246B6
S21444B1100B462046294603F071F888B90EA3D3E9B6
S21444B1200023DAE9040102F0F7FD04460D46024620
S21444B1300B463046394603F061F808B934463D4676
S21444B14022462B464046494602F030FCCAE90601F0
S21444B150BDE8F087AFF300807B14AE47E17A743FD6
S21444B16058FC41202DE9F047DFF874A01AA3D3E930
S21444B1700023DAE90A0102F0CFFD04460D46DAE977
S21444B1800E89DAE9080142464B4602F00DFC0646B3
S21444B1900F4602460B462046294603F02FF888B948
S21444B1A00DA3D3E90023DAE90C0102F0B5FD044609
S21444B1B00D4602460B463046394603F01FF808B99A
S21444B1C034463D4622462B464046494602F0EEFB70
S21444B1D0CAE90E01BDE8F0877B14AE47E17A743FB6
S21444B1E058FC412070477047074B18221A600622C5
S21444B1F0064B1A601722064B1A600122054B1A604A
S21444B200054B064A1A607047781A4020741A402044
S21444B210701A40206C1A4020681A4020EFAB030096
S21444B220044B05491B78054A022B18BF00230B60C4
S21444B230136070472E1E4020781C4020741C40200B
S21444B2407047044B1B88012B02BF034B00221A6035
S21444B250704700BF2A1E40201C1E4020704770477F
S21444B260044B1A78044B1B78134302BF034B022249
S21444B2701A707047371E4020341E40203A1E402025
S21444B280034B1B78012B02BF024B00221A707047F7
S21444B290341E40203A1E4020124B134870B519788D
S21444B2A0124B012900781C78114B124D1A78124B18
S21444B2B01B780CD1012C0AD1012A08D1012B06D1C6
S21444B2C0012804D1002328700C4A137070BD214312
S21444B2D000260A432E70134303430CBF0123334610
S21444B2E0F2E700BF441E40203F1E4020421E40203E
S21444B2F0411E4020491E4020401E4020481E4020FB
S21444B3007047064B01221A70054B1B78934204D1B2
S21444B310044A13707822044B1A8070474D1E40200E
S21444B320341E40204C1E40204A1E4020044B01221E
S21444B3301A600022034B1A700322034B1A7070479C
S21444B340BC1F4020461E40203A1E402008B5FFF74A
S21444B350A3FF044B1B78012B03D1BDE80840FFF73D
S21444B360E5BF08BD491E4020074B08480849094A1E
S21444B37010B51B78084C012B18BF002323700370AC
S21444B3800B70137010BD00BF4E1E4020411E40205F
S21444B390401E40203F1E4020421E4020FFF77CBFF8
S21444B3A0094B1A78094B2AB909490878012804BF79
S21444B3B01A700A70002207490A7007490A801A78E8
S21444B3C001321A70704700BF331E4020E31D4020F0
S21444B3D04D1E40204C1E40204A1E4020FFF7E0BF32
S21444B3E0044B054A1B78042B94BF00230123137097
S21444B3F0704700BFF41D40204E1E4020FFF74CBF50
S21444B40008B5FFF749FF0A4B1B78022B01D1FFF71B
S21444B410C7FFFFF7E5FFFFF73FFF064B1B78012BFF
S21444B42004D1054A00211160044A137008BD00BFC8
S21444B4303E1E4020481E4020BC1F40203A1E40204E
S21444B440054B1B78012B06D1044B1B78012B02BFFE
S21444B450034B00221A707047341E4020451E40207D
S21444B4603A1E4020074B08480849094A10B51B783D
S21444B470084C012B18BF0023237003700B70137005
S21444B48010BD00BF4E1E4020411E4020401E40209E
S21444B4903F1E4020421E4020114B70B51878114B79
S21444B4A001281D78104B1978104B1A78104B1C78CD
S21444B4B0104B0BD1012D09D1012907D1012A05D101
S21444B4C0012C03D11C7000225A7008E02843002641
S21444B4D001435E700A432243F5D101221A7070BDBF
S21444B4E0441E4020421E4020411E4020401E402014
S21444B4F03F1E4020C41F4020094B1A78094B2AB9E6
S21444B50009490878012804BF1A700A7000220749BE
S21444B5100A7007490A801A7801321A70704700BFC9
S21444B520331E4020E31D40204D1E40204C1E40202C
S21444B5304A1E4020054B02221A70054B054A1B78CA
S21444B540003B18BF01231370704700BF4D1E4020B8
S21444B550F41D40204E1E4020FFF79EBF08B5FFF75F
S21444B5609BFFFFF7C9FFFFF7E5FFFFF7E3FFFFF792
S21444B57093FF034B00225A600122024B1A7008BD07
S21444B580C41F40203A1E40201D4B1A781D4B1B7882
S21444B590134333D11C4B1B78013B18BF01231B4A72
S21444B5A013701B4B1A681B4B1B6813431A4B14BF70
S21444B5B0012200221A70194B1A78194B1B78134330
S21444B5C0184B14BF012200221A70174B174A1B78D7
S21444B5D0003B18BF01231370154B164A1B78003BDB
S21444B5E018BF01231370144B144A1B78013B18BF31
S21444B5F0012313700022124B1A7070470123CEE7C2
S21444B6003C1E40203B1E4020CC184020371E402085
S21444B6109819402094194020321E4020391E40205C
S21444B620381E4020361E4020CE184020341E40206F
S21444B630D8184020331E4020CD184020351E4020C8
S21444B6402F1E402038B5FFF79FFF254B1C78ACB91A
S21444B650244D2B78012B0BD1234B1C70FFF7FFFD99
S21444B660FFF7C2FDF6F716F9BDE83840F6F720B9FD
S21444B670022B26D1BDE83840FFF770BF012C25D1F8
S21444B680184B1B78012B07D1174A1370FFF7E8FDB8
S21444B690BDE83840F6F7FEB8022B02D1FFF756FE57
S21444B6A0F6E7032B12D1FFF7F7FCF6F7F3F8F6F7B5
S21444B6B03DF9FFF7C6FDFEF769FCBDE83840FEF7E6
S21444B6C0EFBC032B03D1F6F709F92C7038BD002BD9
S21444B6D0FCD1064B02221A70BDE83840FFF790BEF4
S21444B6E03D1E40203A1E40204E1E40203E1E402016
S21444B6F07047704730B53D4C85B03D48237801A926
S21444B7000193019B1B020193019A637813440193AE
S21444B710019B1B020193019AA37813440193019B56
S21444B7201B020193019AE37813440193237902930D
S21444B730029B1B020293029A637913440293029B70
S21444B7401B020293029AA37913440293029B1B02A0
S21444B7500293029AE37913440293237A0193019B5A
S21444B7601B020193019A637A13440193019B1B02C3
S21444B7700193019AA37A13440193019B1B020193FC
S21444B780019AE37A13440193237B0293029B1B02A0
S21444B7900293029A637B13440293029B1B02029316
S21444B7A0029AA37B13440293029B1B020293029ABF
S21444B7B0E37B1344029342F21273019342F21373EF
S21444B7C0029300F0B0FB04F1100004F1080104F108
S21444B7D01802082314F8015B013B00F8015B11F8DA
S21444B7E0015B02F8015BF5D105B030BD9CFC4120FD
S21444B7F0808080000C4A0823002102F1280030B4DF
S21444B80002F1080502F12004013B02F8011B05F889
S21444B810011B13F0FF0304F8011B00F8011BF3D1CE
S21444B82030BCFFF767BF00BF9CFC41204F4BF0B5D0
S21444B8301B688BB002934E4B1A6803925A68049264
S21444B8409B68059342F21273029A9A4200F08980EA
S21444B850484800F013FBFFF7CDFF002346480AAAEA
S21444B86050F8231002EB83020133082B42F8201CC5
S21444B870F5D1002340480AAA50F8231002EB83026D
S21444B8800133082B42F8201CF5D102990025039A6F
S21444B890049B0598394C00903948264600F0EEFA49
S21444B8A0029B38481B0E2370029B1B0C6370029B42
S21444B8B01B0AA370029BE370039B1B0E2371039B1E
S21444B8C01B0C6371039B1B0AA371039BE371049BCC
S21444B8D01B0E2372049B1B0C6372049B1B0AA372ED
S21444B8E0049BE372059B1B0E2373059B1B0C63731F
S21444B8F0059B1B0AA373059BE37300F0B6FA013558
S21444B90016F8010B00F0DAFA082DF8D11E4D002681
S21444B91000F0CBFA1D482F4600F0A7FA013617F878
S21444B920010B00F0CBFA082EF8D100F0BEFA184B03
S21444B930002203F1080703F1100003F118019446AE
S21444B940013214F8016B15F801EB082A03F8016B71
S21444B95007F801EB00F8016B01F801CBF0D10BB00E
S21444B960F0BD0C4800F08AFA77E700BF808080007C
S21444B9708480800042594600108080009CFC412010
S21444B9806659460083594600A4FC41208D5946001A
S21444B990ACFC412058594600194A08211948F0B5CC
S21444B9A092F8A53100F1100C00F1080500F11807D3
S21444B9B0012B9CBF002382F8D431002310F8014B9E
S21444B9C001391CF8016B17F801EBB4422E7818BF06
S21444B9D0013344EA060418BFDBB2764505F8014B4A
S21444B9E01CBF0133DBB211F0FF01E7D133B1B2F82B
S21444B9F0BE301BB9BDE8F040FFF77CBEF0BD00BFCB
S21444BA00D8FC41209CFC41201FB5144B01A953F897
S21444BA1020305A1E073312F8010F9A4201F8010BE0
S21444BA20F9D19DF804300024502B8DF80C4007D0F3
S21444BA30432B0CD0422B0DD0552B08BF4FF440045B
S21444BA400DF1050000F04CFA204404B010BD4FF44C
S21444BA508004F5E74FF40004F2E700BFCC1F402013
S21444BA602DE9F04F5C4D8DB082462B6805F10808F1
S21444BA7006AC09A963F07C4340462E46A9462B6093
S21444BA804246082316F8017B013B04F8017B9BB22F
S21444BA9010F8017B01F8017B002BF3D1BAF10A0FB1
S21444BAA00BD141464C4C0823FF20013B04F8010BC4
S21444BAB001F8010B9BB2002BF7D1484BC824002158
S21444BAC0013C03F8011BA4B2002CF9D12646444994
S21444BAD0DFF808B104F1080380279BB200932B7863
S21444BAE01F4203D198F800301F4248D051F8243002
S21444BAF00DF10C0C581E073310F801EF98420CF861
S21444BB0001EBF9D14FF000038DF814309DF80C305A
S21444BB10502B59D0432B59D0422B5AD0552B34D185
S21444BB204FF440030DF10D00019300F0D9F9019B49
S21444BB3095F800C0184498F800302A4A3B404FEA2B
S21444BB40102E274918BF082317EA0C0F4FEA104C4B
S21444BB5018BF43F001030BF806C006F1010C1FFAA8
S21444BB608CFC0BF80CE006F1020C1FFA8CFC0BF86C
S21444BB700C00F01C043680B2B6B20BF80030013428
S21444BB80009B7F08A4B2A342A9D1013508F101085D
S21444BB9095429FD1BAF10A0F0FD19DF81A30BDF8DD
S21444BBA0182089F80230A9F800209DF82630BDF800
S21444BBB0242089F80A30A9F80820084B0022304689
S21444BBC09A550DB0BDE8F08F0023ABE74FF48003E1
S21444BBD0A8E74FF40003A5E79CFC4120022140203F
S21444BBE0CC1F4020A4FC4120F0B50D4C0822002078
S21444BBF004F1080514F8016B082380210E4202D193
S21444BC002F78394201D0013080B2013B49089BB2BB
S21444BC10002BF3D1013A013592B2002AEAD1F0BDA5
S21444BC209CFC41202DE9F04FDFF8B480002685B017
S21444BC308346A8F1080A3446284B022E4FF0800962
S21444BC404FF0000234BF082703272744BFB29AF8B0
S21444BC50001019EA010F04D198F8001019EA010FF0
S21444BC602DD053F8241001AD481E073110F801CFEB
S21444BC70814205F801CBF9D19DF804108DF80C20CB
S21444BC80502914D0432914D0422915D055291CD103
S21444BC904FF440050DF1050000F022F905440F4B22
S21444BCA000225D450BD1E0B205B0BDE8F08F00251B
S21444BCB0F0E74FF48005EDE74FF40005EAE701347A
S21444BCC04FEA5909A4B2A742C1D1013608F1010886
S21444BCD00AF1010A082EB0D1FF20E5E7CC1F402028
S21444BCE0A4FC41202DE9FF4700240746204EA146E8
S21444BCF0022C4FF0000834BF4FF0080A4FF0030AF6
S21444BD00336801A95A1E073312F8010F9A4201F804
S21444BD10010BF9D19DF804308DF80C90502B0DD0C2
S21444BD20432B15D0422B16D0552B17D0013404364E
S21444BD30082CDDD1FF2004B0BDE8F08700250DF1C6
S21444BD40050000F0CDF80544BD420AD1E0B2F2E762
S21444BD504FF48005F3E74FF40005F0E74FF4400551
S21444BD60EDE708F101081FFA88F39A45C8D8DDE7DD
S21444BD70CC1F40202DE9F04FDFF8C490002585B055
S21444BD808346A9F108082C462B4A022D4FF0800A18
S21444BD904FF0000134BF082703272744BFB298F862
S21444BDA000001AEA000F04D199F800001AEA000FBE
S21444BDB032D052F824000DF1040C461E073016F813
S21444BDC001EFB0420CF801EBF9D19DF804008DF870
S21444BDD00C10502818D0432818D0422819D055287B
S21444BDE020D14FF440060DF1050000F079F80644E2
S21444BDF0124B00215E45104A0ED15955E0B21D44FF
S21444BE00297205B0BDE8F08F0026ECE74FF48006B3
S21444BE10E9E74FF40006E6E701344FEA5A0AA4B2CB
S21444BE20A742BCD1013509F1010908F10108082DE2
S21444BE30ABD1FF20E5E700BFCC1F40209CFC41204F
S21444BE40A4FC41207047092894BF30303730C0B234
S21444BE50704707B501220DF107018DF80700002051
S21444BE6012F01AF903B05DF804FB10B5441E14F83A
S21444BE70010F00B910BDFFF7ECFFF8E70FB400B5AB
S21444BE80C3B044AA02A852F8041B019204F090FCE2
S21444BE90002302A88DF805318DF80631FFF7E5FF3B
S21444BEA043B05DF804EB04B070470D2008B5FFF7C7
S21444BEB0D0FF0A20BDE80840FFF7CBBF10B50446C4
S21444BEC00009FFF7C0FFFFF7C4FF04F00F00FFF7B9
S21444BED0BAFFFFF7BEFF2C20BDE81040FFF7B9BFFE
S21444BEE0002330B51A46441E184614F8011F392953
S21444BEF008D82F290AD95D1C01F00F0303EB001064
S21444BF002B4606E0A1F14105052D06D900B943B1FB
S21444BF1008220132072AE8D930BD5D1CA1F1370357
S21444BF20ECE71D46EAE7002070470000034A92F813
S21444BF309E30013382F89E30704700BFD8FC4120C3
S21444BF4010B52A4C94F89A30642B94BF01330023DE
S21444BF5084F89A3094F8C63043B1013BDBB284F897
S21444BF60C6301BB984F8C53084F88A3194F8C73093
S21444BF7053B1013BDBB284F8C7302BB994F88A211D
S21444BF80032A08BF84F88A31B4F8E4315BB1013B34
S21444BF909BB2A4F8E43133B9012284F8CF3184F853
S21444BFA0C13184F8A52194F8C231013384F8C231F2
S21444BFB0FFF7F2FC94F8A13123B1002084F8A101E4
S21444BFC001F01FFCB4F8BE3073B1013B9BB2A4F839
S21444BFD0BE304BB984F88A3184F8C53084F8A3312E
S21444BFE084F8C13184F8DC3110BD00BFD8FC412050
S21444BFF0034A92F89830013382F89830704700BF6D
S21444C000D8FC412070470323002010B5064CA4F802
S21444C010EC3104F154020823E16CF7F7A1FA00234B
S21444C02084F8953010BD00BFD8FC4120024B002256
S21444C030C3E91522704700BFD8FC412030B5224BD7
S21444C040002201244FF4FB604FF4FA61082583F87C
S21444C050A541A3F89820A3F8B420C3F8D420A3F8A5
S21444C060CA20A3F8CC2083F88121A3F8822183F840
S21444C0708C2183F89C21C3F8A02183F8D62183F829
S21444C080DB2183F8DC21A3F8E42183F8EA21A3F832
S21444C090C220C3F8C420D864196083F89450A3F827
S21444C0A0C621C3F8D02183F8D421C3E972424FF4A1
S21444C0B00C14C3E92E22C3E96122C3F8C04183F8B5
S21444C0C0C421C3E92B1030BDD8FC4120144B0022B8
S21444C0D093F88D1183F88A21E1B90322A3F88611D7
S21444C0E083F8542093F8882142F0400283F8552080
S21444C0F093F89C21012A01BF7F2283F85520002211
S21444C10083F89C21B3F8862152BAA3F8562000221D
S21444C1109A65704746F60362A3F85420E8E700BFE2
S21444C120D8FC4120054B3022A3F854200A2283F839
S21444C13056200D2283F8C720704700BFD8FC412004
S21444C140034B012283F8C5200B2283F8C620704790
S21444C150D8FC412008B5FFF783FC0330284B81B256
S21444C160284AC0B207291DD85921C3F8982183F814
S21444C170540083F8551093F89E1183F85610FF2107
S21444C18083F85710117883F85810517883F859106B
S21444C1909178D27883F85A1083F85B200422A3F867
S21444C1A0CA2008BDA3F8CC10090AC3F8982141F068
S21444C1B0100183F8550083F85410592183F856101B
S21444C1C093F89E1183F85710FF2183F8581011787E
S21444C1D083F859105178927883F85A1083F85B2084
S21444C1E00322A3F8CA20012283F8C520022283F83A
S21444C1F08A21212283F88C21222283F88821D0E7C1
S21444C200D8FC412002214020024B002283F85420CF
S21444C210704700BFD8FC412038B5CB1C40F6FF74AD
S21444C2209BB2A34228BF2346174C1D0A84F85530B8
S21444C2306223A4F8CC1045F0100584F8580084F81E
S21444C2405630030A84F85450022163F00F03C4F8AE
S21444C250982184F857300123A4F8CA301378A4F8F8
S21444C260CA1084F85930537884F85A300323A4F813
S21444C270CA30937884F85B30FFF762FF212384F852
S21444C2808A1184F88C3138BDD8FC4120F0B5C84CAE
S21444C29087B094F8C2310133DAB21B064ABF002392
S21444C2A084F8C22184F8C231B4F8C63113B1013BD4
S21444C2B0A4F8C63194F8A03123B1002384F8A03101
S21444C2C0FFF798FA94F88A51012D40F0288194F8A3
S21444C2D088312E2B3DD146F60362A4F85420628959
S21444C2E0A4F8562094F88D210D2A0BD1002384F807
S21444C2F08A31012384F8953040F2F513A4F8BE3011
S21444C30007B0F0BD0E2AF4D194F88911A9480491D7
S21444C310A9490391B4F8CA10CDE9012194F8C5207F
S21444C32029460092B4F88421FFF7A8FD94F8893191
S21444C330012B03D1002001F064FAD7E7022B03D186
S21444C340002001F079FAD1E7FF2BCFD184F8CB5106
S21444C350CCE7222BCAD1B4F88431B3F5A06F6BD1A5
S21444C360964D0022964915F8010B134601321F28B4
S21444C37092B204D9322A01F8010BF4D11346E218DA
S21444C3802C213A2082F8E4105A1C422114FA82F2F4
S21444C39082F8E4109A1C4F2114FA82F282F8E410D0
S21444C3A0DA1C14FA82F282F8E4101A1D542114FAA4
S21444C3B082F282F8E4105A1D562114FA82F282F868
S21444C3C0E410991DDA1D14FA81F192B281F8E40062
S21444C3D07C49087842281FD022444E2182F8E41033
S21444C3E003F10802302114FA82F282F8E41003F1D1
S21444C3F00A010933202289B214FA83F383F8E4202D
S21444C4006318002201314FF4A06083F8E42089B217
S21444C4106B4AFFF701FF6CE70B466B4D18781146E5
S21444C42001321F2892B2EBD901332144AB4281F842
S21444C430E400F3D11146E3E7644EB4F8862106EBF4
S21444C4404316B4F886C14FEA122E3789D0B29CFA06
S21444C4509CFCF268FB1C99B2DBB207292FD984F8FE
S21444C4605530C1F30321622384F857E041F01001AC
S21444C47084F8580084F85630002384F85410022177
S21444C480A4F8CA30C4F89821A4F8CC701378A4F859
S21444C490CA5084F859305378A4F8CA1084F85A30ED
S21444C4A0937884F85B300323A4F8CA30FFF748FE39
S21444C4B0322384F88A1184F8C630212374E062213A
S21444C4C084F85430A4F856C0013384F8551000213B
S21444C4D0C4F89821DBB2A4F8CA10A4F8CC7010783B
S21444C4E0A4F8CA5084F85800507884F859000220BA
S21444C4F0A4F8CA00907884F85A000320A4F8CA0026
S21444C500D27884F85B200422A4F8CA20DAB2082A37
S21444C5103FF4ECAEE218013382F85410F6E7022DED
S21444C5207FF4EEAE94F8C530002B7FF4E9AE94F871
S21444C5308831222B7FF4DDAE94F8C430012B06D923
S21444C540023BDBB284F8C430002B7FF4D9AE94F8B7
S21444C550C330072194F88C212E27B4F8CC50D4F855
S21444C5609861134884F8C43084F85420B4F8CA3028
S21444C57001390130AB4238BF16F803C003F101035A
S21444C5802CBF80F8547080F854C09BB211F0FF0161
S21444C590A4F8CA30EAD19D4202F10103DBB298BF47
S21444C5A084F88A112F2B88D884F88C31A1E600BFF2
S21444C5B0D8FC4120865C460070FE412000014400C1
S21444C5C0BCFD41202010400039104000E053460096
S21444C5D0FFF75CBE38B51B4C6389A4F89E31FFF761
S21444C5E013FE94F89E5105F0F703022B05D1012360
S21444C5F0002584F89D31284638BD012D0FD145F6D7
S21444C600061384F85650A4F8543094F89F3184F8AE
S21444C6105730FFF7E9FA40BAA4F85800EBE7032D81
S21444C62012BF47F6027345F6021384F856504FF08D
S21444C63001051BBFA4F854301223A4F8543084F8E0
S21444C6405630D8E7D8FC412008B5FFF7DDFD0B4B44
S21444C6504CF20252A3F854209A7A012A83F85620C0
S21444C66004D1002283F8D421012008BD022A01D136
S21444C6700122F7E77F2283F85520F5E7D8FC4120CE
S21444C680064B47F60372A3F85420012283F856005B
S21444C69083F8571083F89C21704700BFD8FC41208C
S21444C6A0074B93F8D621132A09D093F8A521032AD9
S21444C6B01FBF7F2283F8D621012283F89C2170472E
S21444C6C0D8FC4120002310B56B4C84F8D63194F83E
S21444C6D0CE30222B07D194F8D531032B09D013231F
S21444C6E084F8D63105E0202B14D194F8D531022BAA
S21444C6F0F5D894F8D63163B147F6037284F85730C8
S21444C7000123A4F8542094F8CE2084F89C3184F86D
S21444C710562010BD102B0BD194F8D531022BDED108
S21444C720A37A03F07F03013B022BE2D91223D7E717
S21444C730852B12D1A37A013B012B84BF122384F8A4
S21444C740D63194F8D531022B02D0132384F8D6314F
S21444C75094F8D601FFF7A4FFCBE7272B05D194F82E
S21444C760D53103F0FB03022BB8E7192B18D194F804
S21444C770D531012BB3D0A27A0A2AF4D0032AF2D0B8
S21444C780022AAAD0042A08D1062BA8D1A37B012BBF
S21444C790AFD0FF2BADD03123A2E7012AC6D19CE708
S21444C7A0282B1DD194F8D511A27A032902F07F03D1
S21444C7B005D0002BC9D0032BC7D0022902D0591E5E
S21444C7C00129C2D912F07C0F01D01223BEE7E27AC7
S21444C7D0013A022ABCD90BB1032BB9D13123B5E7B0
S21444C7E0142B1CD194F8D531042B7FF478AFE07A1F
S21444C7F0A37A00EB0323207B00EB03206FF07F43F8
S21444C8009842C4F8D0013FF474AF1C4B98423FF4AE
S21444C81070AFFFF767FAFF287FF46BAFBBE73E2B9A
S21444C82011D194F8D531022B7FF459AFA37A13F083
S21444C8307F0F4FF4FA7318BF1222A4F8E43118BFDE
S21444C84084F8D62155E7312B09D194F8D531062BF7
S21444C8503FF645AFA37A013B022B9CD849E72E2BE3
S21444C86005D194F8D531022B7FF639AF41E70F2B2B
S21444C8703FF63FAF112333E7D8FC4120FF0040008A
S21444C8804FF287139842134B0ED10A290AD100223D
S21444C89083F8D62193F8D621003A18BF012283F8AC
S21444C8A0DB2170471322F3E74FF28B12904201D1FB
S21444C8B00429EBE74FF29512904201D10329E5E7AC
S21444C8C04FF293129042F9D04FF28C129042DED13E
S21444C8D00729DBE7D8FC41200B4B024693F90A00B4
S21444C8E0997A0028B3BF01F07F02012083F85520CF
S21444C8F00020B8BF9A724FF00102A8BF83F85400D4
S21444C90083F8A521704700BFD8FC4120274B014639
S21444C91010B593F90A009A7A0028BBBF02F07F024A
S21444C920002001209A729A7A541E022C31D806248A
S21444C93083F85510022A4FF0000183F854404FF410
S21444C940997483F85620A3F858404FF0F40483F8BB
S21444C950571083F85A404FF4FA7483F8A521A3F885
S21444C960E44112D1124A1278422A06D102F58002D4
S21444C97002F6DF7212784F2A03D0012283F89C21F4
S21444C98003E00122084683F8CA21002283F8CF2117
S21444C99010BD47F60372A3F8542093F8CE2083F8CC
S21444C9A05620122283F85720E7E700BFD8FC4120E0
S21444C9B02010400010B5214CA37AE07A00EB032007
S21444C9C080B2B0F5754FA4F886010BD14FF4A0633E
S21444C9D0A4F884310123002084F88A31222384F881
S21444C9E0883111E0B0F5704F12D300F0A9FD4FF630
S21444C9F0FF73984209D10223012084F85430637AA5
S21444CA0043F0400384F8553010BDA4F88401E1E7B0
S21444CA1040F2DF73D4F8E001C01A47F60373A4F873
S21444CA20543018BF012094F8CE3084F85630312361
S21444CA3084F85730012384F89C31E5E7D8FC41203C
S21444CA402DE9F0414E4C2E23A27AE07A84F88831C0
S21444CA50130900EB0220217B0E2B84F88D3180B223
S21444CA6084F88911A4F886010DD10123002084F8A6
S21444CA708A3194F8DB31012B71D1424A626584F8DD
S21444CA809C31BDE8F081B0F5704F13D300F0C3FD80
S21444CA900F230246A4F8840184F88D314FF6FF73C1
S21444CAA0984204D0384E06EB4013D96921B9032383
S21444CAB084F8DB310120DCE794F8CF11012901D05A
S21444CAC00223F5E7002084F89C0194F8DB01002853
S21444CAD0F0D19B6894F8D5010333DBB2984207D073
S21444CAE013232A4884F8DB1184F8D631FFF7C6F9B5
S21444CAF0B4F884310027DFF89C80042506EB431302
S21444CB00A4F8CA70DA689B68C4F89421A4F8CC30B8
S21444CB10B4F8CA3018F8011BD4F89421D154B4F8A8
S21444CB20CA30B4F8CC2001339BB29A42A4F8CA3037
S21444CB30C0D90020FFF7CAFA94F89C3184F8DB7118
S21444CB4043B9B4F8843106EB4313DB69012B08BFC1
S21444CB5084F8A131013D15F0FF05D9D1AAE7022B8F
S21444CB6003D10B4B6365012389E7032B01BF03F114
S21444CB70445303F5391303F57C53636581E700BFDB
S21444CB80D8FC4120037F2E13E0534600D75C460072
S21444CB90037F2E33E4FC4120204B014630B593F905
S21444CBA00A009A7A0028BBBF02F07F0200200120C8
S21444CBB09A72DA7A02F0FD04012C22D19A7A02F0B3
S21444CBC0FD05012D11D183F8DC5193F8A521012AE6
S21444CBD04FF0020283F854201AD87F225A72222237
S21444CBE09A72002283F8DC2130BD12B983F8DC2126
S21444CBF0EBE7022A06BF002083F8DC4183F89C4119
S21444CC00E3E7022A1FBF7F225A7212229A72DCE797
S21444CC109A7A83F8551083F85620E5E7D8FC4120E5
S21444CC20704770477047704750B123230549013B0E
S21444CC3000284FEA40009BB2B8BF4840002BF6D1CC
S21444CC40704700BF69696C6CF8B56C4B064693F840
S21444CC50A5211C46012A0BD847F60372A3F8542094
S21444CC605A7A83F856207F2283F8572001253DE0E0
S21444CC70997A01F0FB05012D4AD1062384F8550024
S21444CC8084F8561084F8543094F8CF31012B2FD1C1
S21444CC9001292DD10023A4F8A631A4F8A83194F88C
S21444CCA0A661012994F8A72194F8A83118BF022157
S21444CCB084F8582002EB062294F8A90184F85930E7
S21444CCC003EB022384F85A0000EB032084F85760F1
S21444CCD0FFF7AAFF030E84F8A631030C40BA84F883
S21444CCE0A7310123A4F8A80184F8C1312846F8BD29
S21444CCF094F8C23103F1110284F8A63184F8A721CE
S21444CD0003F12202343384F8A82184F8A931C6E713
S21444CD10022DABD193F8C121012A4FF0000210D066
S21444CD2083F8C12147F603720125A3F8542093F8EB
S21444CD30CE2083F89C5183F85620242283F857202B
S21444CD40D4E783F8C121DA7A93F8A6319A420AD115
S21444CD50227B94F8A7319A4205D1B4F8A821B4F8B6
S21444CD600D309A421DD047F603730629A4F8543072
S21444CD7094F8CE3084F856304FF0350384F8573064
S21444CD804FF0010384F89C317FF470AF1C4B1B7842
S21444CD90422B08D001231B4884F89C31FFF76EF8D9
S21444CDA001E00629F2D094F89C51002D7FF45EAF42
S21444CDB0A37A022784F8556084F8563084F8547071
S21444CDC0FFF721F9A37A062B0ED101230E4884F8E7
S21444CDD0CF7184F8CA31FFF748F80B48FFF745F897
S21444CDE00948FFF742F881E794F8A531023B012B46
S21444CDF09CBF012384F8CF3178E700BFD8FC41209C
S21444CE0020104000EB5C4600495D4600114B002272
S21444CE1093F89C1183F8D621012904BF7F2183F817
S21444CE209C2193F8CE2008BF83F85510312A0DD1A3
S21444CE3093F8D511062903D9132283F8D62103E0A3
S21444CE40997A01390229F8D801207047342AFBD14F
S21444CE501222F2E7D8FC412070B5674C0025637A6D
S21444CE60264694F8DD2184F8CE30237A84F89C5103
S21444CE709A4284F8D53101D800200FE0013B062BB6
S21444CE80FAD8FFF71FFC94F89C31012B0FD1D4F845
S21444CE90E02140F2DF739A4201D0012070BD94F83D
S21444CEA0D631113B012BF8D884F89C51E4E7627ADA
S21444CEB094F8CE30102A43F0400003D1BDE87040C9
S21444CEC0FFF724BD202A03D1BDE87040FFF704BD18
S21444CED0852A03D1BDE87040FFF7B6BB2A2B0AD19A
S21444CEE0E37A84F8C33146F60223A4F85430A37A8E
S21444CEF084F85630D1E7222B04D16220BDE8704036
S21444CF00FFF758BD2E2B04D16E20BDE87040FFF7C6
S21444CF1097BD282B04D16820BDE87040FFF73CBE7F
S21444CF202F2B0ED146F60673344AA4F85430062303
S21444CF30013B12F8011B13F0FF0382F84B10F7D1A4
S21444CF40ABE7142B15D1FFF75FF9D4F8D0016FF097
S21444CF507F43984202D02A4B984207D1012386F851
S21444CF60A03145F20143A6F8543096E7FEF702FF97
S21444CF70F7E7272B04D16720BDE87040FFF764BE6F
S21444CF80192B03D1BDE87040FFF724BB312B0BD1DE
S21444CF901C4A0723013B12F8011B13F0FF0382F8D7
S21444CFA0DA10F7D1712079E7112B0FD145F202132D
S21444CFB0A4F85430A37A84F85630FFF724F812487D
S21444CFC0FEF753FF1148FEF750FF66E73E2B0FD19E
S21444CFD094F90A10A37A0029FFF64EAF022142F0D4
S21444CFE0400284F8563084F8541084F8552054E7A8
S21444CFF0FEF79CFF40E700BFD8FC4120E2FC4120FE
S21444D000FF004000E1FC4120F55C46000A5D460016
S21444D01038B5424C0F2384F88D312546237A217B3C
S21444D02003F00F02637AE07A03EB022304F1E4028E
S21444D03001EB0020C4F8942142F2030280B2A4F823
S21444D040CC30A4F88A2194F8CE202F2A23D1033B4F
S21444D0502E22A4F87A019BB284F8882104F22F1277
S21444D060A4F88601A4F8CC3084F87931A37BC4F8BC
S21444D070942184F831310423627BA4F8CA30E37BDC
S21444D08084F87C2184F82F1184F8302184F83231D6
S21444D090FFF748F814E0A4F8860100F051FA4FF67A
S21444D0A0FF7398420ED147F603723123A5F85420F5
S21444D0B095F8CE2085F8D63185F8562085F8573031
S21444D0C0012038BD164B03EB4013DA69002AEAD038
S21444D0D02E22A4F8840184F88821032284F88A2125
S21444D0E0DA689B68C4F89421A4F8CC300123A4F8E9
S21444D0F0CA30637B1370B4F8CA30D4F89421591CF0
S21444D100A4F8CA10A17BD154B4F8CA30D4F89421F8
S21444D110591CA4F8CA10E17BD154B9E7D8FC412085
S21444D120E053460008B51A4B0022197A83F88D213D
S21444D13001F00F00597AA3F8842101EB00219A7A72
S21444D140C82983F888211A7B88BFC82183F8E5203C
S21444D150A3F8CC10D97A02EB01205A7B83F8E4106A
S21444D16083F8E6209A7BA3F8860142F2030083F80C
S21444D170E720DA7BA3F88A0183F8E82005220548ED
S21444D180A3F8CA20C3F89401FEF7CCFF012008BDDB
S21444D190D8FC412002214020184B0022987A83F87C
S21444D1A0D62183F89C21A0F12E0283F8CE00D1B27A
S21444D1B008291DD840F24912CA40D24312F001024F
S21444D1C016D12E2883F8DB2114D193F8A521012A01
S21444D1D002D993F8CF216AB97E2283F8D62102F188
S21444D1E07E2202F5381285325A65012283F89C2144
S21444D1F0012070470020FFF70BBF00BFD8FC41203A
S21444D200002340F2F51210B5884C84F8983084F820
S21444D2109C31A4F8BE204FF4FA72C4E9153323684F
S21444D220A4F8E421B3F5FA6F17D1431E04F10802BB
S21444D230073013F8011F984202F8011BF9D14FF446
S21444D240FA63C4F8E031227A12F0F0032BD1FFF7E8
S21444D25003FE002840F08B804CE040F2DF7293429D
S21444D26020D1037813F0F00F1CD14278A2F11003BA
S21444D270DBB2182B11D9852A01D03E2A12D140F2AE
S21444D280DF736B4AC4F8E031431E073013F8011FBE
S21444D290834202F8011BF9D1D5E7664A22FA03F322
S21444D2A0DB07ECD410BD102B02D1FFF775FFD0E797
S21444D2B0202B40F08F8094F8CE302E3BD9B20629EE
S21444D2C05CD84923CB40DB4313F0010356D194F892
S21444D2D08A1103290ED194F8DD11072910D8B4F821
S21444D2E0CA3001391944B4F8CC30994202D20023EA
S21444D2F084F88A31002384F89C3184F89830D1E746
S21444D30094F88B11914205D14B4884F88A31FEF744
S21444D310ACFDEFE784F88B210D2284F8C72094F8FF
S21444D320DB2132B9E218D4F89411507AB4F8CA2002
S21444D3308854B4F8CA20B4F8CC10013292B2914260
S21444D340A4F8CA2042D894F8DB31012B1AD147F608
S21444D3500372A4F8542094F8CE2084F8562013225E
S21444D36084F8572084F89C31002384F8DB3194F801
S21444D3709C31012B04BF7F2384F85530012384F865
S21444D3809530B7E7022B0CD147F60373A4F8543014
S21444D39094F8CE3084F85630332384F8573001233B
S21444D3A0E0E70020FEF792FEB4F88421234B94F87D
S21444D3B09C1103EB42132248DA69012A08BF84F819
S21444D3C0A12194F8A131FEF759FDCDE70133072B8F
S21444D3D0A5D18FE7302B8DD194F8DD31022B86D939
S21444D3E0312A03D10B2384F8C63083E794F8C5303A
S21444D3F05BB9322A09D146F20323A4F85430B4F870
S21444D40086315BBAA4F856304CE7A37A0021312A19
S21444D41003F1030384F8C51084F8C610DBB284F81D
S21444D420C33084F8C4303FF662AF63E7D8FC41208B
S21444D430E0FC4120130204011A5D4600E053460016
S21444D440325D46000A4810B5FEF718FD72B64FF036
S21444D450005308491022084C0848C3E90012FEF756
S21444D4600DFDFCF720FD2046FEF708FDFBE700BF58
S21444D470445D46007154CA3D6B5D4600515D4600AE
S21444D48038B52C4B93F8C8211C4632B9FEF7D6FD66
S21444D4902948BDE83840FEF7E8BC93F89820002AAF
S21444D4A03FD0002293F89D1183F8982081B193F8D9
S21444D4B09E0183F89D21FEF74DFE012384F89530A6
S21444D4C040F2F513A4F8BE30BDE83840FEF79BBDE5
S21444D4D093F89550002DF3D1184A13780133DBB2F4
S21444D4E0022B01D8137038BD1570FEF7CFFE94F8A2
S21444D4F0993094F8C22101330132DBB284F8C22158
S21444D500042B84F899300CD984F89950FEF718FD0A
S21444D510B4F89C30C72B96BF0133A4F89C50A4F8AB
S21444D5209C3094F8CA2194F8CB311343DBD0FFF7F0
S21444D53089FF00BFD8FC41207A5D4600C8204020C1
S21444D5404FF22803984218D84FF20F03984259D9FD
S21444D550A0F57040113817280DD8DFE800F056299A
S21444D5602B2D2F3131333537393B3D3F41434545EC
S21444D57047494B4D4F51042070474FF293139842FE
S21444D58045D00CD84FF28713984242D04FF28812B7
S21444D5904FF6FF73904214BF1846012070474FF26F
S21444D5A095124FF6FF73904214BF184602207047F8
S21444D5B006207047072070470820704709207047A8
S21444D5C00A2070470B2070470C2070470D20704788
S21444D5D00E2070470F207047102070471120704768
S21444D5E01220704713207047142070471520704748
S21444D5F01620704717207047182070471920704728
S21444D6001A2070474FF6FF70704705207047032076
S21444D610704700207047FFF793BF1C280146F0B5BB
S21444D62085B037D83F4B420103EB40169C584FF623
S21444D630FF739C422ED0F369012B2BD1756804F5F9
S21444D6400004B368AD082246009337482B46FEF7DD
S21444D65015FCD6E903639A1E012A1DD8002315E05B
S21444D66036F82310023389B20291029909040291D2
S21444D6705088029901440291918889B20391039992
S21444D68009040391D188039A0A4403929D4206EB07
S21444D6908302E5D805B0F0BD043B012B3FD90027F3
S21444D6A0BD4206EB8701F5D916F8273020460237E7
S21444D6B00834DBB20293029B1B0602934A78029B11
S21444D6C003EB024302938A78029B03EB0223029302
S21444D6D0CB78029A134402930B79DBB20393039BF1
S21444D6E01B0603934A79039B03EB024303938A790D
S21444D6F0039B03EB02230393CB7902A9039A1344B7
S21444D7000393FEF710FCCBE756F82310023302913E
S21444D710526803929D4206EB8302F5D8BAE700238B
S21444D720F8E700BFE0534600855D46001C280146E6
S21444D73030B403D92C4830BCFEF7A0BB42012B4B77
S21444D74003EB40109B584FF6FF7293421FD0C269BA
S21444D750012A1CD10169072919D0826803F5000300
S21444D760C468881E012814D8520802340021914205
S21444D7700DD253F8040B050C24F8025C4D1C95425C
S21444D78005D2023180B28A4224F8040BEFD830BC6A
S21444D79070470439012925D822F0030222449442D2
S21444D7A0F5D053F8041B44F8041BF8E75858050E04
S21444D7B025704D1CAA42EAD9C0F3074565708D1CF6
S21444D7C0AA42E4D9C0F30725A570CD1CAA42DED9E7
S21444D7D00431C0B204348A4204F8010CD7D99142C9
S21444D7E0E4D3D4E70021FAE7A65D4600E0534600BA
S21444D7F010B50024A0B20134FFF798FF1D2CF9D1D0
S21444D80010BD1FB50024A0B20134FFF706FF1D2C3F
S21444D810F9D1074B02A902934FF47C730393054B4B
S21444D82001930198FEF77FFB002004B010BD00BFB3
S21444D83055EFCDAB1000800008B508B9FFF7D8FF08
S21444D840002008BD124B00B51B688BB00293114BE9
S21444D8501A6803925A6804929B6805930299039A3D
S21444D860049B059800900C48FEF708FB039BB3F511
S21444D8707C7F06D10948FEF701FB01200BB05DF81A
S21444D88004FB0748FEF7FAFA4FF0FF30F6E700BF0E
S21444D8901000800014008000B65D4600CE5D460051
S21444D8A0D95D460008B5FFF7CDFF012805D1FFF73F
S21444D8B09FFFBDE80840FDF7B9BFFFF7C3FF012847
S21444D8C0F5D00020FFF79DFFFFF7BCFFF1E700BF50
S21444D8D010F8012B11F8013B012A28BF9A42F7D0D1
S21444D8E0D01A7047034613F8012B002AFBD1181AA6
S21444D8F001387047000000000000000000000000EF
S21444D90001F0FF01102A2BDB10F0070F08D010F8A7
S21444D910013B013A8B422DD010F0070F42B3F6D1AB
S21444D920F0B441EA012141EA014122F007047FF0C4
S21444D93000070023F0E80256083C85EA010586EA1B
S21444D940010685FA47F5A3FA87F586FA47F6A5FA57
S21444D95087F68EB9EED1F0BC01F0FF0102F0070263
S21444D96032B110F8013B013A83EA010313B1F8D10E
S21444D9700020704701387047002D06BF35460338EF
S21444D980073815F0010F07D1013015F4807F02BF28
S21444D990013015F4C03F0130F0BC0138704700BF79
S21444D9A081F0004102E000BF83F0004330B54FEA07
S21444D9B041044FEA430594EA050F08BF90EA020F74
S21444D9C01FBF54EA000C55EA020C7FEA645C7FEA07
S21444D9D0655C00F0E2804FEA5454D4EB5555B8BF2A
S21444D9E06D420CDD2C4480EA020281EA030382EA9B
S21444D9F0000083EA010180EA020281EA0303362D2D
S21444DA0088BF30BD11F0004F4FEA01314FF4801CFF
S21444DA104CEA113102D0404261EB410113F0004F11
S21444DA204FEA03334CEA133302D0524263EB4303C8
S21444DA3094EA050F00F0A780A4F10104D5F1200E66
S21444DA400DDB02FA0EFC22FA05F2801841F10001C1
S21444DA5003FA0EF2801843FA05F359410EE0A5F195
S21444DA6020050EF1200E012A03FA0EFC28BF4CF0C6
S21444DA70020C43FA05F3C01851EBE37101F000457C
S21444DA8007D54FF0000EDCF1000C7EEB00006EEB89
S21444DA900101B1F5801F1BD3B1F5001F0CD3490813
S21444DAA05FEA30004FEA3C0C04F101044FEA44526A
S21444DAB012F5800F80F09A80BCF1004F08BF5FEAF1
S21444DAC0500C50F1000041EB045141EA050130BDD1
S21444DAD05FEA4C0C404141EB0101013C28BFB1F5E3
S21444DAE0801FE9D291F0000F04BF01460020B1FA2E
S21444DAF081F308BF2033A3F10B03B3F120020CDA01
S21444DB000C3208DD02F1140CC2F10C0201FA0CF0DE
S21444DB1021FA02F10CE002F11402D8BFC2F1200C43
S21444DB2001FA02F120FA0CFCDCBF41EA0C019040F9
S21444DB30E41AA2BF01EB0451294330BD6FEA040442
S21444DB401F3C1CDA0C340EDC04F11404C4F120022D
S21444DB5020FA04F001FA02F340EA030021FA04F33F
S21444DB6045EA030130BDC4F10C04C4F1200220FA96
S21444DB7002F001FA04F340EA0300294630BD21FAD4
S21444DB8004F0294630BD94F0000F83F4801306BF9A
S21444DB9081F480110134013D4EE77FEA645C18BF8E
S21444DBA07FEA655C29D094EA050F08BF90EA020F25
S21444DBB005D054EA000C04BF1946104630BD91EA1D
S21444DBC0030F1EBF0021002030BD5FEA545C05D120
S21444DBD04000494128BF41F0004130BD14F580045F
S21444DBE03CBF01F5801130BD01F0004545F0FE41D3
S21444DBF041F470014FF0000030BD7FEA645C1ABF08
S21444DC00194610467FEA655C1CBF0B46024650EA3E
S21444DC10013406BF52EA033591EA030F41F400216A
S21444DC2030BD00BF90F0000F04BF0021704730B5F0
S21444DC304FF4806404F132044FF000054FF00001C5
S21444DC4050E700BF90F0000F04BF0021704730B586
S21444DC504FF4806404F1320410F0004548BF40425B
S21444DC604FF000013EE700BF42004FEAE2014FEAB0
S21444DC7031014FEA02701FBF12F07F4393F07F4F8B
S21444DC8081F06051704732F07F4208BF704793F08E
S21444DC907F4F04BF41F40021704730B54FF46074A1
S21444DCA001F0004521F000411CE700BF50EA0102A4
S21444DCB008BF704730B54FF000050AE050EA01024D
S21444DCC008BF704730B511F0004502D5404261EBBD
S21444DCD041014FF4806404F132045FEA915C3FF4FE
S21444DCE0D8AE4FF003025FEADC0C18BF03325FEA9B
S21444DCF0DC0C18BF033202EBDC02C2F1200300FA4C
S21444DD0003FC20FA02F001FA03FE40EA0E0021FA70
S21444DD1002F11444BDE600BF70B54FF0FF0C4CF45E
S21444DD20E06C1CEA11541DBF1CEA135594EA0C0F10
S21444DD3095EA0C0F00F0DEF82C4481EA030621EA4B
S21444DD404C5123EA4C5350EA013518BF52EA033586
S21444DD5041F4801143F4801338D0A0FB02CE4FF038
S21444DD600005E1FB02E506F00042E0FB03E54FF068
S21444DD700006E1FB03569CF0000F18BF4EF0010E60
S21444DD80A4F1FF04B6F5007F64F5407404D25FEA5C
S21444DD904E0E6D4146EB060642EAC62141EA55510F
S21444DDA04FEAC52040EA5E504FEACE2EB4F1FD0C51
S21444DDB088BFBCF5E06F1ED8BEF1004F08BF5FEACF
S21444DDC0500E50F1000041EB045170BD06F0004681
S21444DDD046EA010140EA020081EA0301B4EB5C042E
S21444DDE0C2BFD4EB0C0541EA045170BD41F4801126
S21444DDF04FF0000E013C00F3AB8014F1360FDEBF4B
S21444DE00002001F0004170BDC4F10004203C35DA26
S21444DE100C341BDC04F11404C4F1200500FA05F3A9
S21444DE2020FA04F001FA05F240EA020001F000424A
S21444DE3021F0004110EBD37021FA04F642EB0601C0
S21444DE405EEA430E08BF20EAD37070BDC4F10C04EA
S21444DE50C4F1200500FA04F320FA05F001FA04F2AE
S21444DE6040EA020001F0004110EBD37041F100019A
S21444DE705EEA430E08BF20EAD37070BDC4F12005A5
S21444DE8000FA05F24EEA020E20FA04F301FA05F20D
S21444DE9043EA020321FA04F001F0004121FA04F2B5
S21444DEA020EA020000EBD3705EEA430E08BF20EA85
S21444DEB0D37070BD94F0000F0FD101F000464000BF
S21444DEC041EB010111F4801F08BF013CF7D041EA41
S21444DED0060195F0000F18BF704703F00046520045
S21444DEE043EB030313F4801F08BF013DF7D043EA16
S21444DEF00603704794EA0C0F0CEA135518BF95EACC
S21444DF000C0F0CD050EA410618BF52EA4306D1D152
S21444DF1081EA030101F000414FF0000070BD50EA71
S21444DF20410606BF1046194652EA430619D094EAFB
S21444DF300C0F02D150EA013613D195EA0C0F05D1E5
S21444DF4052EA03361CBF104619460AD181EA030139
S21444DF5001F0004141F0FE4141F470014FF00000F1
S21444DF6070BD41F0FE4141F4780170BD70B54FF08C
S21444DF70FF0C4CF4E06C1CEA11541DBF1CEA13550C
S21444DF8094EA0C0F95EA0C0F00F0A7F8A4EB0504EE
S21444DF9081EA030E52EA03354FEA013100F08880E5
S21444DFA04FEA03334FF0805545EA131343EA1263AE
S21444DFB04FEA022245EA111545EA10654FEA002663
S21444DFC00EF000419D4208BF964244F1FD0404F51C
S21444DFD0407402D25B084FEA3202B61A65EB030578
S21444DFE05B084FEA32024FF480104FF4002CB6EB35
S21444DFF0020E75EB030E22BFB61A754640EA0C00B5
S21444E0005B084FEA3202B6EB020E75EB030E22BFF4
S21444E010B61A754640EA5C005B084FEA3202B6EB35
S21444E020020E75EB030E22BFB61A754640EA9C00F4
S21444E0305B084FEA3202B6EB020E75EB030E22BFC4
S21444E040B61A754640EADC0055EA060E18D04FEA82
S21444E050051545EA16754FEA06164FEAC30343EA22
S21444E06052734FEAC2025FEA1C1CC0D111F4801FEF
S21444E0700BD141EA00014FF000004FF0004CB6E7E8
S21444E08011F4801F04BF01430020B4F1FD0C88BF87
S21444E090BCF5E06F3FF6AFAEB5EB030C04BFB6EB92
S21444E0A0020C5FEA500C50F1000041EB045170BD85
S21444E0B00EF0004E4EEA113114EB5C04C2BFD4EBB2
S21444E0C00C0541EA045170BD41F480114FF0000E36
S21444E0D0013C90E645EA060E8DE60CEA135594EAB2
S21444E0E00C0F08BF95EA0C0F3FF43BAF94EA0C0FB5
S21444E0F00AD150EA01347FF434AF95EA0C0F7FF42A
S21444E10025AF104619462CE795EA0C0F06D152EA7D
S21444E11003353FF4FDAE1046194622E750EA410661
S21444E12018BF52EA43067FF4C5AE50EA41047FF472
S21444E1300DAF52EA43057FF4EBAE12E74FF0FF3CD7
S21444E14006E000BF4FF0010C02E000BF4FF0010CA8
S21444E1504DF804CD4FEA410C7FEA6C5C4FEA430C21
S21444E16018BF7FEA6C5C1BD001B050EA410C0CBF70
S21444E17052EA430C91EA030F02BF90EA020F0020D2
S21444E180704710F1000F91EA030F58BF994208BF39
S21444E19090422CBFD8176FEAE37040F001007047F6
S21444E1A04FEA410C7FEA6C5C02D150EA013C07D14D
S21444E1B04FEA430C7FEA6C5CD6D152EA033CD3D098
S21444E1C05DF8040B704700BF8446104662468C4692
S21444E1D01946634600E000BF01B5FFF7B7FF0028C5
S21444E1E048BF10F1000F01BD4DF808EDFFF7F4FFEE
S21444E1F00CBF012000205DF808FB00BF4DF808ED79
S21444E200FFF7EAFF34BF012000205DF808FB00BF9B
S21444E2104DF808EDFFF7E0FF94BF012000205DF8BD
S21444E22008FB00BF4DF808EDFFF7CEFF94BF012072
S21444E23000205DF808FB00BF4DF808EDFFF7C4FF6B
S21444E24034BF012000205DF808FB00BF4FEA410CB4
S21444E2507FEA6C5C02D150EA013C0AD14FEA430C97
S21444E2607FEA6C5C02D152EA033C02D14FF00000D4
S21444E27070474FF0010070474FEA410212F5001212
S21444E28015D211D56FF47873B3EB625212D94FEAB4
S21444E290C12343F0004343EA505311F0004F23FA9E
S21444E2A002F018BF404270474FF00000704750EAF3
S21444E2B0013005D111F0004008BF6FF000407047B0
S21444E2C04FF00000704700BF4A0011D212F500120A
S21444E2D011D20DD56FF47873B3EB62520ED44FEA75
S21444E2E0C12343F0004343EA505323FA02F07047F5
S21444E2F04FF00000704750EA013002D14FF0FF3033
S21444E30070474FF0000070474FEA4102B2F1E043D5
S21444E31024BFB3F5001CDCF1FE5C0DD901F0004CC3
S21444E3204FEAC0024CEA5070B2F1004F40EB830013
S21444E33008BF20F00100704711F0804F21D113F13F
S21444E3403872BCBF01F00040704741F480114FEA78
S21444E3505252C2F11802C2F1200C10FA0CF320FA01
S21444E36002F018BF40F001004FEAC1234FEAD3231E
S21444E37003FA0CFC40EA0C0023FA02F34FEA430388
S21444E380CCE77FEA625307D150EA01331EBF4FF011
S21444E390FE4040F44000704701F0004040F0FE402C
S21444E3A040F40000704700BF80F0004002E000BF29
S21444E3B081F0004142001FBF5FEA410392EA030F27
S21444E3C07FEA226C7FEA236C6AD04FEA1262D2EB71
S21444E3D01363C1BFD218414048404140B8BF5B4276
S21444E3E0192B88BF704710F0004F40F4000020F00F
S21444E3F07F4018BF404211F0004F41F4000121F025
S21444E4007F4118BF494292EA030F3FD0A2F101026E
S21444E41041FA03FC10EB0C00C3F1200301FA03F1AC
S21444E42000F0004302D5494260EB4000B0F5000FCF
S21444E43013D3B0F1807F06D340084FEA310102F18E
S21444E4400102FE2A51D2B1F1004F40EBC25008BF40
S21444E45020F0010040EA03007047490040EB00000A
S21444E460013A28BFB0F5000FEDD2B0FA80FCACF10B
S21444E470080CB2EB0C0200FA0CF0AABF00EBC25038
S21444E48052421843BCBFD0401843704792F0000F26
S21444E49081F4000106BF80F400000132013BB5E779
S21444E4A04FEA41037FEA226C18BF7FEA236C21D0EF
S21444E4B092EA030F04D092F0000F08BF0846704754
S21444E4C090EA010F1CBF0020704712F07F4F04D122
S21444E4D0400028BF40F00040704712F100723CBF35
S21444E4E000F50000704700F0004343F0FE4040F45F
S21444E4F0000070477FEA226216BF08467FEA23631D
S21444E5000146420206BF5FEA412390EA010F40F407
S21444E510800070474FF0000304E000BF10F0004353
S21444E52048BF40425FEA000C08BF704743F096433A
S21444E53001464FF000001CE050EA010208BF704755
S21444E5404FF000030AE000BF50EA010208BF7047DC
S21444E55011F0004302D5404261EB41015FEA010CF1
S21444E56002BF84460146002043F0B64308BFA3F1E9
S21444E5708053A3F50003BCFA8CF2083AA3EBC253CB
S21444E58010DB01FA02FC634400FA02FCC2F12002EA
S21444E590BCF1004F20FA02F243EB020008BF20F021
S21444E5A00100704702F1200201FA02FCC2F1200287
S21444E5B050EA4C0021FA02F243EB020008BF20EA7C
S21444E5C0DC7070474FF0FF0C1CEAD0521EBF1CEAAA
S21444E5D0D15392EA0C0F93EA0C0F6FD01A4480EA98
S21444E5E0010C400218BF5FEA41211ED04FF0006381
S21444E5F043EA501043EA5111A0FB01310CF00040AD
S21444E600B1F5000F3EBF490041EAD3715B0040EAD2
S21444E610010062F17F02FD2A1DD8B3F1004F40EBA2
S21444E620C25008BF20F00100704790F0000F0CF075
S21444E630004C08BF49024CEA502040EA51207F3A39
S21444E640C2BFD2F1FF0340EAC250704740F4000014
S21444E6504FF00003013A5DDC12F1190FDCBF00F005
S21444E66000407047C2F10002410021FA02F1C2F1B3
S21444E670200200FA02FC5FEA310040F1000053EA4F
S21444E6804C0308BF20EADC70704792F0000F00F09D
S21444E690004C02BF400010F4000F013AF9D040EAA3
S21444E6A00C0093F0000F01F0004C02BF490011F437
S21444E6B0000F013BF9D041EA0C018FE70CEAD15335
S21444E6C092EA0C0F18BF93EA0C0F0AD030F0004CB5
S21444E6D018BF31F0004CD8D180EA010000F0004069
S21444E6E0704790F0000F17BF90F0004F084691F027
S21444E6F0000F91F0004F14D092EA0C0F01D1420261
S21444E7000FD193EA0C0F03D14B0218BF084608D129
S21444E71080EA010000F0004040F0FE4040F4000073
S21444E720704740F0FE4040F4400070474FF0FF0C06
S21444E7301CEAD0521EBF1CEAD15392EA0C0F93EA4D
S21444E7400C0F69D0A2EB030280EA010C49024FEA9F
S21444E750402037D04FF0805343EA111143EA101358
S21444E7600CF000408B4238BF5B0042F17D024FF410
S21444E770000C8B4224BF5B1A40EA0C00B3EB510FEB
S21444E78024BFA3EB510340EA5C00B3EB910F24BFD4
S21444E790A3EB910340EA9C00B3EBD10F24BFA3EB59
S21444E7A0D10340EADC001B0118BF5FEA1C1CE0D121
S21444E7B0FD2A3FF650AF8B4240EBC25008BF20F0D4
S21444E7C0010070470CF0004C4CEA50207F32C2BF28
S21444E7D0D2F1FF0340EAC250704740F400004FF0C5
S21444E7E00003013A37E792F0000F00F0004C02BFF6
S21444E7F0400010F4000F013AF9D040EA0C0093F0C0
S21444E800000F01F0004C02BF490011F4000F013B19
S21444E810F9D041EA0C0195E70CEAD15392EA0C0F81
S21444E82008D142027FF47DAF93EA0C0F7FF470AFB9
S21444E830084676E793EA0C0F04D14B023FF44CAFFC
S21444E84008466EE730F0004C18BF31F0004CCAD191
S21444E85030F000427FF45CAF31F000437FF43CAFCD
S21444E8605FE700BF4FF0FF3C06E000BF4FF0010CEF
S21444E87002E000BF4FF0010C4DF804CD4FEA4002D1
S21444E8804FEA41037FEA226C18BF7FEA236C11D01B
S21444E89001B052EA530C18BF90EA010F58BFB2EBCE
S21444E8A0030088BFC81738BF6FEAE17018BF40F04E
S21444E8B0010070477FEA226C02D15FEA402C05D102
S21444E8C07FEA236CE4D15FEA412CE1D05DF8040B87
S21444E8D0704700BF844608466146FFE70FB5FFF71A
S21444E8E0C9FF002848BF10F1000F0FBD4DF808EDD2
S21444E8F0FFF7F4FF0CBF012000205DF808FB00BFC3
S21444E9004DF808EDFFF7EAFF34BF012000205DF81C
S21444E91008FB00BF4DF808EDFFF7E0FF94BF012069
S21444E92000205DF808FB00BF4DF808EDFFF7D2FF66
S21444E93094BF012000205DF808FB00BF4DF808EDA9
S21444E940FFF7C8FF34BF012000205DF808FB00BF76
S21444E9504FEA4002B2F1FE4F0FD34FF09E03B3EBA3
S21444E96012620DD94FEA002343F0004310F0004FE3
S21444E97023FA02F018BF404270474FF00000704739
S21444E98012F1610F01D1420205D110F0004008BFD8
S21444E9906FF0004070474FF00000704742000ED2C0
S21444E9A0B2F1FE4F0BD34FF09E03B3EB126209D481
S21444E9B04FEA002343F0004323FA02F070474FF037
S21444E9C00000704712F1610F01D1420202D14FF0AC
S21444E9D0FF3070474FF00000704700BF53B94AB944
S21444E9E0002908BF00281CBF4FF0FF314FF0FF300E
S21444E9F000F0A6B9ADF1080C6DE904CE00F03EF87F
S21444EA00DDF804E0DDE9022304B0704738B5054676
S21444EA100C462846214600220023FFF7EFFB28B980
S21444EA2028462146BDE8384000F00AB8284604F196
S21444EA30004100F005F8404261EB410138BD00BF9B
S21444EA40D0B50C4B002206460F46FFF765F9FFF794
S21444EA503BFC0446FFF7E6F8074B0022FFF75CF959
S21444EA6002460B4630463946FEF79EFFFFF72CFC1F
S21444EA702146D0BD0000F03D0000F0412DE9F047AE
S21444EA80089D0E4604468C46002B40F081808A4200
S21444EA90174645D9B2FA82F24AB1C2F1200106FAC3
S21444EAA002F320FA01F1974041EA030C94404FEAFE
S21444EAB0174E230CBCFBFEF6B9B20EFB16CC43EA4B
S21444EAC00C4306FB01F0984209D9FB1806F1FF3CBB
S21444EAD080F01581984240F21281023E3B441B1A54
S21444EAE0A4B2B3FBFEF00EFB103344EA034400FB2F
S21444EAF001F1A14209D93C1900F1FF3380F00181AC
S21444EB00A14240F2FE8002383C44641A40EA064081
S21444EB1000211DB1D4400023C5E90043BDE8F08779
S21444EB2002B9FFDEB2FA82F2002A4FD1CB1B4FEA7B
S21444EB30174E1FFA87F80121B3FBFEFC260C0EFB8A
S21444EB401C3346EA034608FB0CF3B34207D9BE1906
S21444EB500CF1FF3002D2B34200F2EB808446F61A40
S21444EB60A3B2B6FBFEF00EFB106643EA064408FB6F
S21444EB7000F8A04507D93C1900F1FF3302D2A0455E
S21444EB8000F2D2801846A4EB080440EA0C40C0E7E2
S21444EB908B4208D9002D00F0AF800021C5E900065D
S21444EBA00846BDE8F087B3FA83F1002949D1B34259
S21444EBB002D3824200F2BB80841A66EB0303012030
S21444EBC09C46002DAAD0C5E9004CA7E7C2F1200315
S21444EBD09740D8409140DE404FEA174E08434FEAEC
S21444EBE0104CB6FBFEF11FFA87F80EFB11664CEA92
S21444EBF0064601FB08F3B34204FA02F409D9BE19E7
S21444EC0001F1FF3C80F08E80B34240F28B800239A3
S21444EC103E44F31A86B2B3FBFEF00EFB103346EACC
S21444EC20034600FB08F3B34207D9BE1900F1FF3C84
S21444EC3074D2B34272D902383E44F31A40EA0141D0
S21444EC407AE7C1F1200703FA01F422FA07F31C43DA
S21444EC5020FA07F906FA01F34FEA144CFE4049EA53
S21444EC6003094FEA1943B6FBFCFE1FFA84F80CFB73
S21444EC701E6643EA06460EFB08FAB24502FA01F25D
S21444EC8000FA01F308D9A6190EF1FF3048D2B2456E
S21444EC9046D9AEF1020E2644A6EB0A061FFA89F9B7
S21444ECA0B6FBFCF00CFB106649EA064600FB08F887
S21444ECB0B04507D9A61900F1FF3C2DD2B0452BD953
S21444ECC00238264440EA0E40A6EB0806A0FB02891A
S21444ECD04E45C446CE4618D315D075B3B3EB0C0296
S21444ECE066EB0E0606FA07F722FA01F3CE401F43F8
S21444ECF0C5E90076002111E7294628460EE7664610
S21444ED00EDE6184601E74345E7D2B8EB020C69EB5B
S21444ED1004040138A646E0E76046D3E760468CE73D
S21444ED208646B9E7614674E702383C442BE7084612
S21444ED3047E7ACF1020C3E4411E72946EEE600BF35
S21444ED40704700BF2DE9F04788B0002B1F46144695
S21444ED50B8BF03F10043129A109DDDF84CA0B6BF2D
S21444ED601F4600232D231370149B23F02008B8F16C
S21444ED70460F05D0B8F1450F00D10135022300E017
S21444ED80032307AA049206AACDE902A2CDE90035D8
S21444ED9022463B4601F0A4FDB8F1470F064602D191
S21444EDA0119BDB0722D5B8F1460F06EB050910D1B7
S21444EDB03378302B0AD10022002320463946FFF709
S21444EDC013FA18B9C5F10105CAF80050DAF800304C
S21444EDD099440022002320463946FFF705FA08B135
S21444EDE0CDF81C903022079B4B4507D3079B159ABA
S21444EDF09B1B3046136008B0BDE8F087591C07914A
S21444EE001A70F0E7F7B503460029B8BF494203F83D
S21444EE10022BB4BF2D222B22092942702ADD0DF184
S21444EE200704A4460A27A6460A4691FBF7F607FBBC
S21444EE3016153035632A04F1FF340EF8015C31466A
S21444EE40F1DC3031AEF1020504F8011C441C2946BD
S21444EE5061450AD30DF10902A2EB0E02654588BF4F
S21444EE6000221344181A03B0F0BD11F8012B04F81D
S21444EE70012FEDE7302330318370C170031DF1E775
S21444EE802DE9F04F91B00C46DDF8688016461F46D3
S21444EE90054602F04BFE036809931846FEF722FD2A
S21444EEA000230E93D8F800300A90073323F0070364
S21444EEB003F1080294F81890D4F800B0C8F800207B
S21444EEC0D3E90023C4E91223D4E9128A2AF0004382
S21444EED00B930B999C4B4FF0FF324046FFF7B6F925
S21444EEE070BB994B0B994FF0FF324046FFF790F9B1
S21444EEF030BB0022002340465146FFF77FF910B14D
S21444EF002D2384F84330914B9148B9F1470F94BF71
S21444EF1098468046032323612BF0040323604FF076
S21444EF20000A009733460FAA2146284600F0D2F935
S21444EF30013040F08F804FF0FF3011B0BDE8F08FC5
S21444EF404246534640465146FFF780F940B1BAF12F
S21444EF50000FBCBF2D2384F843307E487E4BD4E755
S21444EF6063685A1C09F0DF0142D10623636000221D
S21444EF7006920EAACDE904920DAA4BF4806303923E
S21444EF800DF13302CDE901322360636800934246B3
S21444EF90534628460B91FFF7D5FE0B9947298046E2
S21444EFA00D9908D1C81C02DB6368994240DDA9F17B
S21444EFB002095FFA89F9B9F1650F1FD801394A4643
S21444EFC004F150000D91FFF71DFF0E9A1318012A05
S21444EFD08246236102DC2268D20701D501332361CD
S21444EFE09DF83330002B9CD02D2384F8433098E78B
S21444EFF04729BCD1002BBAD10123B7E7B9F1660F34
S21444F00018D1002963680BDD216113B92268D00743
S21444F01002D501330B442361A1654FF0000ADFE7B4
S21444F02013B92268D20701D50233F4E70123F2E785
S21444F0304FF067090E9B994205DB23682161D80788
S21444F040EAD54B1CE7E70029D4BFC1F102020122EE
S21444F0501344E0E723685A0507D4236942463146F9
S21444F0602846B84701302BD165E7B9F1650F40F221
S21444F070DC80D4E9120100220023FFF7B5F800280B
S21444F08033D0364A012331462846B84701303FF448
S21444F09052AFDDE90D239A4202DB2368D8070FD529
S21444F0A0DDE9092331462846B84701303FF443AFEB
S21444F0B04FF0000804F11A090E9B013B434509DC56
S21444F0C023689B0700F10181E0680F9B9842B8BF14
S21444F0D0184632E701234A4631462846B8470130A7
S21444F0E03FF429AF08F10108E6E70D9B002B37DC17
S21444F0F01A4A012331462846B84701303FF41BAF2D
S21444F100DDE90D23134302D12368D907D8D5DDE9B9
S21444F110092331462846B84701303FF40CAF4FF038
S21444F120000904F11A0A0D9B5B424B4501DC0E9B19
S21444F13094E70123524631462846B84701303FF407
S21444F140FAAE09F10109EEE7FFFFEF7FE65D460000
S21444F150EA5D4600F25D4600EE5D4600F65D46001A
S21444F1600E9AA36D9A42A8BF1A46002A914637DCE7
S21444F1704FF0000B29EAE97904F11A02D4F858A0B2
S21444F180AAEB09035B4533DCDDE90D239A423BDBFE
S21444F1902368DA0738D40E9A0D99A2EB0A03A2EB39
S21444F1A001099945A8BF9946B9F1000F34DC4FF0E0
S21444F1B0000829EAE97904F11A0ADDE90D239B1AC5
S21444F1C0A3EB090343457FF77BAF01235246314601
S21444F1D02846B84701303FF4AEAE08F10108ECE7E4
S21444F1E01346314642462846B8470130C0D1A2E6C7
S21444F1F00123314628460B92B84701303FF49BAE74
S21444F2000B9A0BF1010BB9E7DDE909233146284691
S21444F210B8470130BFD18EE64B4608EB0A0231466A
S21444F2202846B8470130C2D185E60E9A012A01DC49
S21444F230DB0737D50123424631462846B8470130D6
S21444F2403FF479AEDDE9092331462846B847013014
S21444F2503FF471AED4E9120100220023FEF7C4FF46
S21444F260D8B90E9B08F10102013B31462846B847FF
S21444F27001300ED15FE601234A4631462846B84758
S21444F28001303FF458AE08F101080E9B013B43455C
S21444F290F1DC534604F15002E1E64FF0000804F175
S21444F2A01A09F2E701234246DFE701234A4631467C
S21444F2B02846B84701303FF43EAE08F10108E368FB
S21444F2C00F995B1A4345F0DCFEE64FF0000804F164
S21444F2D01909F4E72DE9F047164699468A680B69FA
S21444F2E0DDF820809342B8BF1346336091F843203C
S21444F2F007460C460AB1013333602368990642BF79
S21444F300336802333360256815F0060506D104F1E8
S21444F310190AE36832689B1AAB4226DC94F8432009
S21444F320131E226818BF012392062BD404F143020D
S21444F33049463846C04701301ED02368E5683268DF
S21444F34003F00603042B08BFAD1AA36822690CBF5A
S21444F35025EAE57500259342C4BF9B1AED1800269E
S21444F3601A34B5421AD1002008E0012352464946D1
S21444F3703846C047013003D14FF0FF30BDE8F08730
S21444F3800135C6E7E1185A1C302081F84300224470
S21444F39094F8451082F843100233C7E70123224607
S21444F3A049463846C0470130E6D00136D9E7000022
S21444F3B02DE9FF470C469146277E0C99782F8046C8
S21444F3C09A4604F1430207D8622F0AD8002F00F069
S21444F3D0D880582F00F0A38004F1420684F8427087
S21444F3E03AE0A7F16303152BF6D801A050F823F0B2
S21444F3F049F444005DF44400D9F34400D9F344008E
S21444F400D9F34400D9F344005DF44400D9F34400EE
S21444F410D9F34400D9F34400D9F3440069F54400D1
S21444F4208DF444004BF54400D9F34400D9F344002A
S21444F4308BF54400D9F344008DF44400D9F34400DA
S21444F440D9F3440053F544000B681A1D1B680A6040
S21444F45004F1420684F842300123A3E02568086894
S21444F4602E0600F104030AD505680B60002D03DA66
S21444F4702D236D4284F843305E480A2319E015F084
S21444F480400F05680B6018BF2DB2EFE70B68256880
S21444F490181D0860280601D51D6802E06906FBD5DC
S21444F4A01D8854486F2F0CBF08230A23002184F874
S21444F4B043106668A660002EA2BF216821F00401AE
S21444F4C021600DB9002E4DD01646B5FBF3F103FB73
S21444F4D01157C75D06F8017D2F46BB420D46F4D949
S21444F4E0082B0BD12368DF0708D523696168994246
S21444F4F0DEBF302306F8013C06F1FF36921B22613C
S21444F500CDF800A04B4603AA21464046FFF7E2FE4C
S21444F51001304CD14FF0FF3004B0BDE8F087354899
S21444F52084F8457023680E681F0656F8045B0E6020
S21444F53014D5D90744BF43F0200323601DB923687C
S21444F54023F0200323601023B0E7236843F020030E
S21444F55023607823284884F84530E3E75E0648BFAE
S21444F560ADB2E6E71646BBE70B68266860691D1D24
S21444F5700D6035061B6801D5186002E07106FBD5A0
S21444F5801880002323611646BAE70B681A1D0A60E2
S21444F5901E68626800213046FEF7B2F908B1801B47
S21444F5A0606063682361002384F84330A8E72369D6
S21444F5B0324649464046D0470130ABD023689B0785
S21444F5C013D4E068039B9842B8BF1846A4E70123C7
S21444F5D0324649464046D04701309BD00135E36821
S21444F5E003995B1AAB42F2DCEBE7002504F11906FB
S21444F5F0F5E700BFF85D4600095E46002DE9F04F8A
S21444F60087B0174603938B685A1EB2F5AE7F83BF06
S21444F6106FF4AE755B190293002386BF40F25D1308
S21444F6208B6002930B688B46002543F4F0634BF8DB
S21444F6301C3BCDE9045580460C465E46AA46A94680
S21444F6400195A26852B13B681B784E2B64D8402B78
S21444F6503CD8A3F12B01C8B20E283AD9B9F1000F11
S21444F66003D0236823F4807323600AF1FF3ABAF187
S21444F670010F00F213815E4500F2058101252846FC
S21444F68007B0BDE8F08FA3F161020D2AE6D801A1C8
S21444F69051F822F0D3F744005DF644005DF644008A
S21444F6A05DF6440033F844000BF844005DF644002D
S21444F6B05DF64400E1F744005DF644005DF6440020
S21444F6C05DF644005DF6440099F74400A3F1410218
S21444F6D0DBE70E29C2D801A050F821F08BF744008E
S21444F6E05DF644008BF744001FF844005DF6440082
S21444F6F039F7440075F7440075F7440075F744003D
S21444F70075F7440075F7440075F7440075F74400F0
S21444F71075F7440075F744006E2B09D8602BB2D8B1
S21444F720542B77D0592B99D1072D97D1082529E00A
S21444F730742B6FD0792BF6E72168C8051AD5029B3F
S21444F74021F08001216009F101091BB1013B01321E
S21444F7500293A260A368013BA3602369013323613B
S21444F7607B68013B002B7B6040F384803B6801331D
S21444F7703B6066E71AEB050F7FF470AF226822F40D
S21444F780C072226006F8013BE4E7226810067FF563
S21444F79065AF22F08002F4E7BAF1000F0ED1B9F15A
S21444F7A0000F0ED1226802F4E061B1F5E06F08D193
S21444F7B022F4F06222604FF0010AE3E7BAF1020F46
S21444F7C055D0012D02D0042D7FF448AF0135EDB25B
S21444F7D0D8E7BAF1010F7FF441AF4FF0020AD1E700
S21444F7E07DB9B9F1000F7FF43CAF226802F4E061C2
S21444F7F0B1F5E06F7FF439AF22F4F0622260012560
S21444F800C0E7032DE2D0052DDEE7022D7FF426AFB8
S21444F8100325B7E7062D7FF421AF0725B2E7226814
S21444F82091057FF51BAF22F420722260CDF8049038
S21444F830A8E7226802F4A061B1F5806F06D05005AF
S21444F8407FF50CAFB9F1000F3FF40FAF910558BFE9
S21444F850019922F4F06258BFA9EB010142F4C07248
S21444F86058BFCDE9041622604FF000098AE74FF0EE
S21444F870030A87E7D4F8803139464046984700283B
S21444F8803FF4DFAEEAE6D4F87C3116F8011D3A467A
S21444F890404698472369013B2361ECE66B1E062BE2
S21444F8A025D8022D36D85E457FF6E8AED4F87C31AE
S21444F8B016F8011D3A46404698472369013B2361A2
S21444F8C0F1E70298D4F87C3110F8011D02903A46CC
S21444F8D0404698472369013B23610AF1FF3A5FFAA1
S21444F8E08AFABAF1020FECD1033DEDB2761B2368D7
S21444F8F0DA052FD55B0510D55E457FF6BFAED4F846
S21444F9007C3116F8011D3A46404698472369013B28
S21444F9102361F1E7AA460296DFE716F8011C23693D
S21444F920652903F1FF3306F1FF3523610CD04529E1
S21444F9300AD0D4F87C313A4640469847236916F8AC
S21444F940021C013BB51E2361D4F87C313A4640463E
S21444F95098472E46256815F0100559D1357023680A
S21444F96003F4C063B3F5806F1CD1019B4B45A3EBF6
S21444F970090224D100225946404600F081FED4F8BC
S21444F98000C0039B1CF0020F1B6806460F4621D09E
S21444F99003991A1D0A601B68C3E90067E3680133CC
S21444F9A0E3606CE6049B002BE4D005990A232A46C0
S21444F9B00131404600F0E4FE049B059EC21A04F260
S21444F9C06F139E4228BF04F5B7761249304600F0BE
S21444F9D029F8CFE71CF0040F03F1040E03D0039973
S21444F9E0C1F800E0D7E7039AC2F800E0D3F80080F5
S21444F9F002460B46FEF72AFC28B1074800F00EF8EC
S21444FA00C8F80000CAE730463946FEF77DFCF7E7FB
S21444FA10002534E61A5E46000459460000487047FE
S21444FA200000C07F0EB400B59AB01BAB01900590A1
S21444FA306FF00041094806910391094953F8042B95
S21444FA4004910068009301A902F0E2FD019B0022A4
S21444FA501A701AB05DF804EB03B07047DC214020FE
S21444FA600802FFFF2DE9F0410F46904602F082FB64
S21444FA7004460D46B8F1000F11D0C7F30A53C3F13C
S21444FA806B03002B0BDD1B0503F17F55002405F5A6
S21444FA90401522462B46FEF73FF904460D462046BF
S21444FAA02946BDE8F08100002DE9F04FA1B09B4601
S21444FAB000231C939E4B17921F68824638460E4678
S21444FAC0FDF710FF4FF0000804464FF000091B9660
S21444FAD01B9B1A782B2A4CD03AD80D2A33D8082A9E
S21444FAE033D8002A3DD000230C931B9D2B78302B13
S21444FAF040F0A9806B7803F0DF03582B66D10C9B4B
S21444FB0001931CAB00938B4ACDF808B01DAB1BA9E0
S21444FB10504601F01FFD10F00706044605D0062E99
S21444FB2029D1013500231B950C93179B002B40F0DD
S21444FB308E850C9BD3B1424609F1004310461946C4
S21444FB4021B0BDE8F08F202ACDD101331B93BFE707
S21444FB502D2AC8D101220C925A1C1B925B78002B8A
S21444FB60C3D1179B1B96002B40F06F8542464B46ED
S21444FB70E4E70022EFE71C9A3AB135211EA802F0CA
S21444FB80F0FB1C99504602F031F8013E042E06D88C
S21444FB90DFE806F00A0314170A00DDE91E89210788
S21444FBA0C3D549F00049C0E7DDE91E831D9A23F416
S21444FBB0801302F2334243EA0259F0E7DFF87891C1
S21444FBC0EDE76FF000494FF0FF38E8E71B9B5A1CFF
S21444FBD01B925B78302BF9D0002BA6D001230793D9
S21444FBE01B9B08930023CDE905339B460A221B98AA
S21444FBF00578A5F13003D9B2092926D922463946D3
S21444FC0002F01CFE002832D000202B465C460490AE
S21444FC100246652B01D0452B13D11CB9079B0343E1
S21444FC209FD000241B9E731C1B9373782B2B78D079
S21444FC302D2B7BD00027A3F13001092940F2828086
S21444FC401B9600259EE00023C9E7BBF1080FD5BFED
S21444FC500699059902FB013302FB013300F10100CA
S21444FC60D4BF069305930BF1010B1B90BFE71B9B78
S21444FC701A191B921B5DBBF1000F36D004905C46EC
S21444FC80A3F13002092A12D90122C2E71B9B5A1C4F
S21444FC901B925B780130302BF8D0A3F13102082A4E
S21444FCA000F2DA841B9A0490002008920446303B03
S21444FCB000F1010213D00499114404912246051917
S21444FCC00A21954213D12218082A04F10104044457
S21444FCD01BDC06990A2202FB0133069300221B9B77
S21444FCE0591C1B915B781046CAE75846D3E7082A46
S21444FCF004DC069F4F4306970132E2E7571C102F59
S21444FD00DEBF059F4F430597F6E7102CDFBF0599E6
S21444FD100A2202FB01330593E0E700230493012201
S21444FD207CE70027B31C1B93B37884E70127F9E7E5
S21444FD30805F4600205E46000000F07F1B9B591CF7
S21444FD401B915B78302BF9D0A3F1310108293FF69B
S21444FD5078AFA3F1300C1B9B09934FF00A0E1B9B04
S21444FD60591C1B915B78A3F13005092D35D9099DA3
S21444FD70491B082944F61F6502DC6545A8BF65464D
S21444FD8007B16D42002C4CD1079901437FF4CDAEA8
S21444FD90002A7FF4E6AE692B26D023DC492B23D0F9
S21444FDA04E2B7FF4DEAE9C491BA801F00FFE0028C4
S21444FDB03FF4D7AE1B9B1B78282B2CD197491EAA01
S21444FDC01BA801F017FE052825D11F9BDDF8788077
S21444FDD043F0FF4949F4E009A7E60EFB0C3CACF1BE
S21444FDE0300CBCE76E2BDCE78D491BA801F0EEFD1A
S21444FDF000283FF4B6AE1B9B8A49013B1BA81B93C5
S21444FE0001F0E4FD10B91B9B01331B93DFF82492E9
S21444FE104FF0000889E6844802F00AFD8046894689
S21444FE2083E6049B0698EB1ABBF1000F08BFA34673
S21444FE30102C07932646A8BF1026FDF7F3FE092C80
S21444FE408046894613DD794B03EBC60353E91223F8
S21444FE50FDF762FF804605988946FDF7E3FE0246B5
S21444FE600B4640464946FDF7A1FD804689460F2C81
S21444FE7036DC079B002B3FF458AE22DD162B09DCFC
S21444FE806A4C04EBC304D4E9000142464B46FDF7F2
S21444FE9043FFC3E7079AC4F12503934220DB634D2F
S21444FEA0C4F10F0405EBC40142464B46D1E90001B8
S21444FEB0FDF732FF079B1C1B05EBC405D5E9002361
S21444FEC0E5E7079B16330BDB049B584A5D1B02EBA6
S21444FED0C505D5E9002340464946FEF747F89DE761
S21444FEE0079BA61B1E44002E71DD16F00F030AD096
S21444FEF04E4901EBC30142464B46D1E90001FDF7AA
S21444FF000BFF8046894636F00F0650D0B6F59A7FEA
S21444FF1027DD4FF0000BCDF810B0CDF820B0CDF86B
S21444FF2018B02223DFF80C91CAF800304FF00008CE
S21444FF30089B002B3FF4F9AD1C99504601F056FE41
S21444FF400699504601F052FE0499504601F04EFE82
S21444FF500899504601F04AFE5946504601F046FE7E
S21444FF60E3E500233611404649461F46012E21DC70
S21444FF700BB1804689462E4BA9F1547903EBC7074B
S21444FF8042464B46D7E90001FDF7C6FE294B0A46D2
S21444FF900B4029498B428046BBD8A1F580118B4241
S21444FFA086BFDFF898904FF0FF3802F1547900236B
S21444FFB005937EE0F20707D51D4B03EBC703D3E951
S21444FFC00023FDF7A9FE012301377610CEE7EED0D5
S21444FFD0764216F00F020AD0144B03EBC203404697
S21444FFE04946D3E90023FDF7C1FF804689463611CA
S21444FFF0DDD01F2E24DD4FF0000BCDF810B0CDF829
S21445000020B0CDF818B022234FF000084FF0000975
S214450010CAF800308CE700BFF35D4600345E460004
S214450020EB5D4600745F460004594600C05F4600D7
S214450030985F46000000F07F0000A07CFFFFEF7F42
S21445004016F0100318BF6A23B34F0593404649463A
S2144500500023F20704D5D7E90023FDF75DFE01230B
S214450060761007F10807F4D10BB180468946059B03
S214450070BBB1C9F30A53C3F16B03002B494610DDE8
S2144500801F2B40F32881342BDEBF203B4FF0FF3239
S21445009002FA03F34FF00008CCBF4FF05C7903EA51
S2144500A001090022002340464946FEF79DF80028F0
S2144500B0A1D1069B0093089923465A46504601F01F
S2144500C0EAFD089000283FF424AF049B5D1B079B80
S2144500D0002BB4BF2B4600230E93079B4FF0000B17
S2144500E023EAE3731693CDF810B0089B504659683B
S2144500F001F048FD069000283FF413AF089B1A69A7
S214450100023203F10C0192000C3001F02DFD1EABBE
S21445011001931DAB009342464B465046CDE90A89AE
S21445012002F0A2F81C9000283FF4FBAE0121504691
S21445013001F03DFE0490034600283FF4F2AE1D9DB7
S2144501401E9A002DABBF0E9B169B169C0E9EACBFF3
S214450150EE185C1B059BED1A1544704B013D9D4200
S214450160C2F1360280F2C9805B1B1F2BA2EB03024D
S2144501704FF0010700F3B68007FA03F30F93002507
S214450180B718059BBE4214441C443346A8BF3B469D
S214450190A342A8BF2346002BC2BFFF1AE41AF61A8D
S2144501A00E9B002B17DD04991A46504601F0A4FE17
S2144501B0049000283FF4B5AE01461C9A504601F01F
S2144501C0FFFD099000283FF4ACAE1C99504601F05F
S2144501D00DFD099B1C93002F00F39380079B002B76
S2144501E008DD169A0699504601F086FE06900028C8
S2144501F03FF497AE002C08DD06992246504601F09E
S214450200C9FE069000283FF48CAE002E08DD049902
S2144502103246504601F0BEFE049000283FF481AEBB
S214450220069A1C99504601F02FFF834600283FF456
S21445023078AE0024C3680499C4600D9301F009FFA5
S214450240A04271DA0D9B53EA080340F09780C9F344
S2144502501303002B40F0928029F000431B0D1B052D
S214450260B3F1D66F40F28A80DBF8143023B9DBF859
S2144502701030012B40F3828059460122504601F04A
S21445028089FE0499834601F0E4FE002876DD05994B
S214450290234A4B46002900F0928002EA0901B1F153
S2144502A0D66F00F38C80B1F15C7F7FF7ACAE1D4A0C
S2144502B00023CDE914324046DDE914234946FDF7CF
S2144502C02BFD0B46034308BF22238046894608BFBD
S2144502D0CAF8003030E64FF0FF3202FA03F303EA7D
S2144502E00808DEE6C5F17F4505F57F0505F57B453E
S2144502F0E23507FA05F50F9742E7012300250F93E8
S2144503003EE71C993A46504601F044FE1C900028AC
S2144503107FF464AF05E600BF485E460002FCFFFF7B
S2144503200000F07F00005039CDF8249066D10D9A34
S214450330C9F313035AB39C4A93422CD1059B4046B6
S21445034003B39A4A4B461A40B2F1D46F4FF0FF3189
S2144503501BD8120DC2F16B0301FA03F398421AD16A
S214450360934B099A9A4202D101303FF4DAAD8F4B4E
S214450370099A1A4002F580194FF00008059B002B94
S21445038095D1D9E54FF0FF33E8E70B46E6E753EA64
S21445039008033FF47CAFE5B1099B1D42EED00D9BAB
S2144503A0059A40464946C3B1FFF75CFB02460B46F5
S2144503B0DDE90A01FDF7FAFA80468946DEE713408D
S2144503C0A3F580136FEA13596FEA09594FF0FF38C2
S2144503D0D4E70F9B13EA080FE0E7FFF743FB024617
S2144503E00B46DDE90A01FDF7DFFA002200238046C9
S2144503F08946FDF7F9FE0028C0D004E6049958461C
S21445040001F081FF00224FF0804306460F46FDF778
S214450410FFFE002875D00D9B002B47D0654F002664
S214450420644D099B23F000431B0D1B050F930F9A44
S214450430614B9A4240F0C880DDE90A23CDE9142392
S214450440099BA3F154794046494601F093FE02467E
S2144504500B4630463946FDF75FFC42464B46FDF7B0
S214450460A5FA0B465149554A1940914280465ED9F0
S2144504700B9B02F15472934203D10A9B01333FF41E
S21445048050ADDFF82C914FF0FF381C99504601F0DF
S214450490ADFB0699504601F0A9FB0499504601F07C
S2144504A0A5FB5946504601F0A1FB1EE6B8F1000FE4
S2144504B019D1099BC3F31303E3B93E4B00223046DB
S2144504C03946FDF79BFEC8B93D4B002230463946B6
S2144504D0FDF722FC04460D4605F100431894199392
S2144504E0DDE918679DE7B8F1010F03D1099B002B9D
S2144504F03FF489AD334F0026002491E70D9C304DDF
S214450500EAE72F4B002230463946FDF705FC0D9BA2
S21445051004460D4633B901F1004310901193DDE9C9
S21445052010677EE702460B46CDE91023F7E703F151
S2144505305479059B002BA8D129F000430F9A1B0D33
S2144505401B059A42A1D120462946FEF75FFAFDF7DC
S214450550B5FB02460B4620462946FDF725FA0D9A79
S214450560C9F3130343EA0803134304460D4666D00E
S21445057009A3D3E90023FDF741FE00287FF4DCAC50
S21445058007A3D3E9002320462946FDF755FE002854
S2144505903FF47BAFD0E400BF9535A094FFFFDF3F27
S2144505A035E5AF350000E03FFFFF0F000000F07F68
S2144505B0FFFFEF7F0000F03F0000E07FFFFF9F7CDE
S2144505C00000E03F0000F0BF059B13B30F9BB3F15F
S2144505D0D46F1ED826A3D3E9002320462946FDF727
S2144505E017FE90B129462046FDF76EFE012838BF16
S2144505F00120FDF717FB0D9B04460D46D3B901F1C7
S214450600004312901393DDE912670F9A07F1D663FC
S2144506109F1ADDE90A0101F0ADFD02460B4630465C
S2144506203946FDF779FBDDE90A23FDF7BFF9804634
S21445063089467EE702460B46CDE91223E3E70EA33D
S214450640D3E90023FDF7DAFDA1E700230C93179ABB
S2144506501B9B1360FFF76DBA652B3FF45EAB452BCE
S2144506603FF45BAB0122FFF78FBB00BFAFF30080C3
S2144506700000C0FFFFFFDF419535A094FFFFCF3F49
S214450680014BFFF711BA00BF442240202DE9F04741
S2144506903A4E86468C4660461CF8014BA55D15F0DD
S2144506A00805F8D12D2C33D19CF800404FF00108B1
S2144506B000F1020C002B5CD0102B0CD1302C0AD14B
S2144506C09CF8000000F0DF0058284DD19CF801400A
S2144506D010230CF1020C08F10047013F0026B7FB3A
S2144506E0F3F9304603FB197AA4F13005092D18D8DD
S2144506F02C46A34224DD751C07D081451DD301D168
S214450700A2451ADB00FB034001261CF8014BEBE72C
S2144507102B2C08BF9CF80040A84608BF00F1020CE9
S214450720C8E7A4F14105192D01D8373CE1E7A4F106
S2144507306105192D04D8573CDBE74FF0FF36E4E753
S214450740731C06D12223CEF80030384642B9BDE8A0
S214450750F087B8F1000F00D04042002AF7D00EB11E
S2144507600CF1FF311160F2E73024002BB3D108239A
S214450770B1E7302CA4D00A23ADE700BF715E460032
S214450780FFF784BF00B59BB0019105916FF000411E
S214450790069103910549049101A901F039FF019B92
S2144507A000221A701BB05DF804FB00BF0802FFFF6D
S2144507B013460A46014602480068FFF7E3BF00BFF6
S2144507C0DC2140202DE9F74F03690C69A342074613
S2144507D0C0F28180013C01F1140800F1140505EBD7
S2144507E08403019358F8243055F8242001339A425F
S2144507F04FEA840B08EB8409B2FBF3F631D34FF08E
S214450800000E4046AC46F24650F8042B93B206FB23
S21445081003E34FEA134E9BB2AAEB0303120CDCF834
S21445082000A006FB02E213FA8AF34FEA124E1FFABD
S21445083082FADCF80020CAEB124202EB23429BB256
S21445084043EA024381454CF8043B4FEA224ADBD251
S21445085055F80B302BB9019B043B9D421A462ED3C7
S2144508603C61384601F0F5FB002824DB0136284676
S2144508704FF0000C58F8042BD0F800E093B2ACEBE0
S2144508800303120C13FA8EF3C2EB1E4202EB23420D
S2144508909BB243EA0243C14540F8043B4FEA224C2B
S2144508A0E8D255F8242005EB840322B9043B9D4243
S2144508B01A460AD33C61304603B0BDE8F08F12684D
S2144508C0043B002ACCD1013CC7E71268043B002A0A
S2144508D0F0D1013CEBE70020EEE700000000000009
S2144508E02DE9F04F446A99B016461F46CDE9046790
S2144508F0DDF8948005463CB9102001F01BF9C0E9A7
S214450900014468620460C4606B6A196851B15A68EC
S2144509104A60012393408B60284601F067F96B6A6D
S21445092000221A603B1EB9BF23F0004305930023FF
S214450930C8F80030DDF81490A74BBCBF0122C8F8B4
S214450940002033EA090319D1249A42F20F73136043
S214450950C9F31303334300F06D85269B53B99F4B6C
S21445096023E09F4B03930833269A1360039819B0E8
S214450970BDE8F08F994B03930333F5E7DDE904347F
S214450980CDE90C34DDE90C0100220023FDF72CFCF3
S214450990804660B1249A01231360269B002B00F005
S2144509A04685904B269A1360013B0393DEE716ABCC
S2144509B0019317AB00932846DDE90C2301F054FC60
S2144509C0C9F30A548346002C7ED00D9BCDF84C8047
S2144509D0C3F31303DDE90C0143F07F5141F44011A5
S2144509E0A4F2FF34804B0022FCF7DEFF74A3D3E964
S2144509F00023FDF791F974A3D3E90023FCF7D6FF4E
S214450A00064620460F46FDF71DF971A3D3E9002398
S214450A10FDF782F902460B4630463946FCF7C6FFD7
S214450A2006460F46FDF728FC002282460023304640
S214450A303946FDF7E3FB48B15046FDF703F9324624
S214450A403B46FDF7D1FB08B90AF1FF3ABAF1160F56
S214450A5057D8664B03EBCA03D3E90023DDE90C01FF
S214450A60FDF7CCFB00284ED00AF1FF3A00230F9342
S214450A70169B1C1B631E099345BFC4F101030693D1
S214450A80002300234CBF09930693BAF1000F3CDBC5
S214450A90099BCDF838A05344099300230A93229B1B
S214450AA0092B00F2B580052BC4BF043B2293229B3D
S214450AB0A3F10203CCBF00240124032B00F2B4802B
S214450AC0DFE803F02D987AA4DDE916431C4404F2CA
S214450AD03243202BC3BFC3F1400304F2124009FA48
S214450AE003F3C3F12003C6BF26FA00F0184306FAFF
S214450AF003F0FDF797F80123A1F1F871013C139334
S214450B0070E70123B3E70F90B2E7069BA3EB0A0312
S214450B100693CAF100030A9300230E93BFE700230A
S214450B200B93239B002B00F382804FF00109CDF8F1
S214450B3020904B46CDF88C906E6A00227260042257
S214450B4002F114009842716877D9284601F01AF8E0
S214450B506B6A30601B680393089B0E2B00F2EE8091
S214450B60002C00F0EB80BAF1000F7ADD1F4A0AF040
S214450B700F0302EBC303D3E900341AF4807FCDE9B3
S214450B8010344FEA2A145CD0194BDDE90C01D3E941
S214450B900823FDF7EBF9CDE9040104F00F0403271C
S214450BA0134E002C4FD1DDE91023DDE90401FDF796
S214450BB0DDF9CDE904016EE00123B1E7AFF300802E
S214450BC061436F63A787D23FB3C8608B288AC63F09
S214450BD0FB799F501344D33F0000F07F7A5F460071
S214450BE0715F4600F75D46000000F83FC05F46006F
S214450BF0985F460000230B93239B0AEB030909F1F4
S214450C000103012B0893B8BF012395E70123F2E7BB
S214450C100124002322930B944FF0FF390022CDF890
S214450C2020901223239287E701230B93F4E7DDF800
S214450C308C90CDF820904B467EE70131716052008E
S214450C407EE70227ACE7E10708D5DDE91001D6E9DE
S214450C500023FDF761F8CDE9100101376410083629
S214450C609FE700F0A580CAF10004A44BA44E04F00B
S214450C700F0203EBC203D3E90023DDE90C01FDF7C0
S214450C804BF8CDE90401241100230227002C40F03F
S214450C908480002B8DD10F9B002B00F08B80DDE9E7
S214450CA00434CDE91034DDE91001964B0022FDF7FA
S214450CB0A5FA00287ED0089B002B7BD0B9F1000F03
S214450CC038DDDDE91001904B0022FDF725F8CDE92A
S214450CD004010AF1FF3801374C463846FCF7B2FFA7
S214450CE0DDE90423FDF718F8884B0022FCF75EFE85
S214450CF0A1F15076CDE910011196002C5DD1DDE9C4
S214450D000401834B0022FCF74FFE02460B46CDE915
S214450D100423109A3346FDF78FFA002840F0978251
S214450D20DDE90401109A06F10043FDF767FA00284D
S214450D3040F08B82DDE90C34CDE90434179B002B5B
S214450D40C0F25181BAF10E0F00F34D816B4B03EBA8
S214450D50CA03D3E90034CDE90634239B002B80F241
S214450D60DB80089B002B00F3D78040F06D82684BF4
S214450D700022DDE90601FCF7CFFFDDE90423FDF798
S214450D8051FA089C2646002840F04382039F3123AB
S214450D9007F8013B0AF1010A3FE2E20705D5D6E925
S214450DA00023FCF7B9FF01370123641008366DE7C9
S214450DB0022770E7089CD0468FE703994F4B21449E
S214450DC012910B9903EBC403DDE9106753E902233F
S214450DD0002946D04F490020FDF7C8F83B46324625
S214450DE0FCF7E2FDCDE91001039FDDE90401FDF7BF
S214450DF043FA0446FCF726FF02460B46DDE90401A6
S214450E00FCF7D2FD303402460B46CDE9042307F8FD
S214450E10014BDDE91023FDF7F1F9002865D1DDE941
S214450E20042338490020FCF7BFFDDDE91023FDF714
S214450E30E5F9002840F0B680129B9F423FF47AAF12
S214450E40DDE91001304B0022FCF766FF2E4BCDE95D
S214450E5010010022DDE90401FCF75EFFCDE904013F
S214450E60C3E730463946FCF757FFCDE91001129BDC
S214450E70039C1493DDE90401FDF7FEF91590FCF794
S214450E80E1FE02460B46DDE90401FCF78DFD159BA8
S214450E90303304F8013B129B9C4206460F464FF002
S214450EA0000224D11B4BDDE91001FCF77FFD02460D
S214450EB00B4630463946FDF7BFF9002871D1DDE9C6
S214450EC0102314490020FCF76FFD02460B463046BA
S214450ED03946FDF793F900283FF42CAF149F7B1E47
S214450EE0149317F8013C302BF8D0C24649E0064B20
S214450EF0FCF712FFCDE90401BCE700BFC05F460022
S214450F00985F46000000F03F0000244000001C406B
S214450F10000014400000E03FDDE90489039FDDE959
S214450F20062340464946FDF721F8FDF7A5F9044650
S214450F30FCF788FEDDE90623FCF7EEFE04F13006F5
S214450F400B46024649464046FCF72EFD07F8016B20
S214450F50039E089BBE1BB34238D102460B46FCF7A0
S214450F6025FDDDE9062380468946FDF765F958BB2C
S214450F70DDE9062340464946FDF736F908B1E1075F
S214450F8022D42846594600F031FE00233B70249B68
S214450F900AF101001860269B002B3FF4E7AC1F6062
S214450FA0E4E427463B461F4613F8012D392A07D168
S214450FB0039A9A42F7D10399302208F101080A703C
S214450FC01A7801321A7090E7D046EBE7A14B00221B
S214450FD0FCF7A2FE0022002380468946FDF704F969
S214450FE000289CD0CDE70B9A002A00F0CD80229AA7
S214450FF0012A00F3AF80139A002A00F0A78003F277
S21445100033430A9C069F069A1A440692099A01217A
S2144510101A442846099200F0CAFE0646002F0CDD03
S214451020099B002B09DDBB42069AA8BF3B46D21A50
S2144510300692099AFF1AD31A09930A9BF3B10B9B9A
S214451040002B00F0A580002C10DD314622462846B0
S21445105000F052FF5A4601460646284600F0B0FEC6
S21445106059468046284600F0C1FDC3460A9B1A1BD2
S21445107004D05946284600F03FFF834601212846BE
S21445108000F095FE0E9B002B044640F383801A46DF
S2144510900146284600F030FF229B012B04467CDDA6
S2144510A04FF00008236904EB8303186900F031FE0E
S2144510B0C0F12000099B184410F01F0000F08E80F8
S2144510C0C0F12003042B40F38780C0F11C00069B2B
S2144510D003440693099B034407440993069B002B48
S2144510E005DD59461A46284600F054FF8346099BB7
S2144510F0002B05DD21461A46284600F04BFF0446E0
S2144511000F9B002B6CD02146584600F0A2FF0028C6
S21445111066DA002359460A22284600F07EFD0B9BD8
S2144511200AF1FF3A8346002B00F08B8131460023B7
S2144511300A22284600F071FDB9F1000F064600F375
S2144511409180229B022B40F38D8051E0169BC3F184
S214451150360356E7089B5C1E0A9BA342BFBF0A9B05
S2144511600A94E21A0E9BB6BF9B181C1B0E93089B4F
S214451170B8BF0024002BB9BF069B089A069F089B5C
S214451180BCBF9F1A00233EE70A9C069F0B9E45E779
S2144511900A9A6EE7229B012B19DC049BBBB9059B7B
S2144511A0C3F313039BB9059B23F000431B0D1B0597
S2144511B083B1069B01330693099B013309934FF090
S2144511C001080E9B002B7FF46DAF012072E74FF0B0
S2144511D00008F6E79846F4E780D018461C3076E7D0
S2144511E0089B002B38DC229B022B35DDDDF8209052
S2144511F0B9F1000F0DD121464B460522284600F091
S2144512000CFD01460446584600F023FF00283FF7EC
S214451210BDAD239B039F6FEA030A4FF000082146A6
S214451220284600F0E3FC002E3FF4ABAEB8F1000FC5
S21445123005D0B04503D04146284600F0D7FC314698
S214451240284600F0D3FC9CE600242646E1E7C24645
S21445125026469BE5000024400B9BDDF82090002B9E
S21445126000F0F680002F05DD31463A46284600F068
S21445127091FE0646B8F1000F55D07168284600F035
S21445128081FC326902320746920006F10C010C30A9
S21445129000F06AFC01223946284600F07BFE039B97
S2144512A001330893039B4B440A93049B03F00103C5
S2144512B0B04609930646089B2146013B584604938B
S2144512C0FFF780FA034630330690414658460B935F
S2144512D000F0BFFE324681462146284600F0D4FE41
S2144512E0C2680B9B074602BB0146584600F0B1FE56
S2144512F00B9B024639462846CDE90B3200F076FC74
S214451300229B0C9A089F43EA0201099B0B430B9BC1
S2144513100DD1392B29D0B9F1000F01DD069B3133AC
S214451320049A13707BE73046B9E70122E2E7B9F144
S214451330000F06DB229941EA0909099959EA010194
S21445134020D1002AECDD594601222846089300F0B4
S21445135021FE2146834600F07CFE0028089B02DCE1
S214451360DED1DA07DCD5392BD8D1049A3923137068
S2144513703B461F46013B17F8012C392A50D001320F
S2144513801A704CE7002A03DD392BEED00133C7E748
S214451390089A0A9902F8013C8A422AD059460023FF
S2144513A00A22284600F039FCB04583464FF0000334
S2144513B04FF00A024146284607D100F02EFC8046EB
S2144513C00646089B0133089375E700F026FC314630
S2144513D0804600230A22284600F01FFC0646F0E712
S2144513E0B9F1000F039ACCBF4F46012717444FF07B
S2144513F00008594601222846089300F0CBFD2146B1
S214451400834600F026FE0028B2DC02D1089BDB07A7
S214451410AED43B461F4613F8012D302AFAD0FEE6D9
S214451420039A9A42A5D10AF1010A312379E7134B6B
S214451430FFF7BBBA269B002B7FF493AA104BFFF70A
S214451440B4BAB9F1000F03DC229B022B3FF7D0AEAE
S214451450039F21465846FFF7B5F900F1300307F8D4
S214451460013B039ABA1A9145BADD594600230A222A
S214451470284600F0D2FB8346EBE700BFF65D460004
S214451480715F46000369B3EB611F2DE9F0434FEAF0
S214451490611200F1140445DD11F01F0104EB8306CB
S2144514A004EB82050CD100F110072946B14234D32E
S2144514B09B1A9B00EA1E964238BF0023234415E03C
S2144514C054F82270C1F12008CF4005F1040EA1461C
S2144514D07645F44615D89B1A9A00043A0135AE422D
S2144514E038BF0022A318A75007B104331A1BA342DE
S2144514F04FEAA20208BF0023026108BF4361BDE868
S214451500F083DCF800C00CFA08FC4CEA070749F8FB
S214451510047B5EF8047BCF40DAE751F804CB47F806
S21445152004CFC3E72346E1E7A0F13003092B02D8F1
S2144515302038C0B27047A0F16103052B01D8473863
S214451540F7E7A0F14103052B01D82738F1E700203E
S214451550704700002DE9F04F8BB08B460693BA4B8B
S21445156002901B68039318469046FCF7BBF9039B0D
S214451570DBF800200344824613F8013C0793931C8E
S214451580C2F1FF2202F57F02FE32D1181F4613F83C
S214451590010B01913028F8D0FFF7C6FF0446002816
S2144515A03AD103995246384601F048F9054600288F
S2144515B066D117F80A0007EB0A06FFF7B5FF0028BD
S2144515C060D03346187830281F4603F10103F9D01A
S2144515D0FFF7AAFF0123B0FA80F464093546019364
S2144515E03A46164601323078FFF79EFF0028F8D176
S2144515F003995246304601F021F980B94DB906EBBC
S2144516000A052A46164601323078FFF78DFF002830
S214451610F8D1AD1BAD0004E000242546E0E7002DDB
S214451620F7D1337803F0DF03502B39D173782B2B62
S2144516302AD02D2B2CD0711C4FF000090878FFF7C7
S21445164073FF431EDBB2182B2AD8A0F1100211F8FF
S214451650010FFFF769FF431EDBB2182B1BD9B9F103
S214451660000F00D052421544CBF80010D4B1019B70
S214451670002B14BF0027062738460BB0BDE8F08F71
S2144516803E4625460124CCE74FF00009B11CD5E778
S2144516904FF00109FAE70A2303FB0202103AD6E7A0
S2144516A03146E1E7F31B013B2146072B50DC029808
S2144516B000F068FA4FF0000B00F11409CAF1010377
S2144516C00446CDF81090CDF804B00893B74242D3FF
S2144516D0049F019B47F8043BA7EB0907BF1027610A
S2144516E0184600F016FB7F01D8F800603F1AB7424F
S2144516F065DDBF1B3946204600F056FE8246A8B13A
S2144517007B1E591103F01F0259F821104FF0010AAC
S2144517100AFA02F20A4209D0534505DDB91E2046AB
S21445172000F042FE002847D14FF0020A39462046CF
S214451730FFF7A8FE3D44D8F80830AB424DDA02988C
S214451740214600F053FA149A00231360A32793E723
S21445175001315B10A9E7731E079A059316F8013CFD
S214451760934219D0BBF1200F07D1049B019A43F849
S214451770042B0493002301939B4616F8010CFFF7B0
S214451780D3FE019B00F00F0000FA0BF003430193D4
S2144517900BF1040B059B0DE0059B089A1344BB42D1
S2144517A0E0D3184603990993524601F047F8099B3A
S2144517B00028D7D11E4689E74FF0030AB6E709DA6F
S2144517C0F71B214602983A4600F0E4FBED1B04461B
S2144517D000F114094FF0000AADE7D8F80400A84216
S2144517E06DDD451BAE4231DCD8F80C30022B22D0DD
S2144517F0032B24D0012B15D1AE4213D1012E0BD18C
S214451800069AD8F80430136001232361C9F80030DE
S214451810149B62271C602FE7711E204600F0C4FD0E
S2144518200028EDD10298214600F0E0F9149A0023ED
S2144518301360502720E7159B002BF3D1E0E7159B57
S214451840002BDDD1EEE700BF805F46006F1EBAF184
S214451850000F31D127B13946204600F0A5FD824616
S2144518607B11012159F8233007F01F0701FA07F7C6
S2144518701F422946204618BF4AF0020A761BFFF744
S21445188001FED8F804500227BAF1000F48D0D8F820
S2144518900C30022B15D0032B17D0012B09D11AF08B
S2144518A0020F06D0D9F800004AEA000A1AF0010FDE
S2144518B00ED147F0100733E04FF0010AD0E7012775
S2144518C0E2E7159BC3F101031593159B002BF0D05A
S2144518D0D4F8109004F114034FEA890B03EB890101
S2144518E04FF0000C184653F8042BB2F1FF3F1CD0BE
S2144518F001320260022F04F1140338D1D8F80020D3
S214451900013AB2420AD17111012253F8213006F04C
S2144519101F0602FA06F61E4218BF174647F020076E
S214451920149B1C60069B1D60A6E6994243F804CCB2
S214451930D8D8A368994512DB61680298013100F052
S21445194021F92269023204F10C01824692000C30DC
S21445195000F00AF92146029800F048F954462369F2
S2144519605A1C04EB8303226101225A61C2E72269AD
S2144519704A450BDD01212046FFF784FDD8F808309F
S2144519800135AB42FFF6DBAE0127C7E716F01F066B
S214451990FAD09B44C6F120065BF8040C00F0B9F972
S2144519A0B042E7DBF0E700BFC2F10802920070B52F
S2144519B0C2F120064368046803FA06F52C43D34073
S2144519C0046040F8043F8842F4D370BD30B50368E0
S2144519D0013311F8014B14B90360012030BD13F8EB
S2144519E0012BA2F14105192D98BF2032A242F0D015
S2144519F00020F3E72DE9F04F0B6801685E1102EB16
S214451A00860613F01F0387B018BF04360025371F18
S214451A1082469046019346F8045CB9463C46029594
S214451A20AB464A784B1C039342B310460591049245
S214451A30FFF77AFD00284FD1049A0599202A18D831
S214451A40029B9B4513DD4C4506D2072D04DC2A46F2
S214451A5049462046FFF7A8FF444550D90023A4F140
S214451A60040944F8043CCDF808B04C461D46039995
S214451A70D7E7292A56D10231CAF80010BBF1000F24
S214451A8050D04C4506D2072D04DC2A46494620460A
S214451A90FFF78AFF444534D9A8F10402234653F894
S214451AA0041B42F8041F9F42F9D23B1B23F0030355
S214451AB004330134033EB44288BF04234344002222
S214451AC043F8042B9F42FBD23B681BB9474527D1B9
S214451AD001233B60052026E00135082D0BF1010B5F
S214451AE006DD4445C3D9002344F8043C0125043C9F
S214451AF0226800F00F0040EA02122260B7E7082588
S214451B00B5E7019B002BDFD04FF0FF32C3F1200332
S214451B1022FA03F356F8042C1A4046F8042CD3E769
S214451B20043FD1E7042007B0BDE8F08F0048704772
S214451B3034234020024B0146186800F0B3BC00BF72
S214451B40DC21402082B001B901A942B14BB11378DE
S214451B500B601278101E18BF012002B07047104661
S214451B60FBE76FF00100F8E70A44914200F1FF33C6
S214451B7000D1704710B511F8014B03F8014F91425B
S214451B80F9D110BD70B5466A04460D463EB91020DB
S214451B90FFF7D0FFC0E9016660620660C660666A08
S214451BA0F36883B1636ADB6853F82500B8B9012149
S214451BB001FA05F6721D9200204600F016FC60B14B
S214451BC0C0E901560EE021220421204600F00DFC16
S214451BD0636AF060DB68002BE4D1002070BD0268C4
S214451BE043F825200023C0E90333F7E770B5466A76
S214451BF005460C463EB91020FFF79CFFC0E9016636
S214451C0068620660C6603CB16B6A6268DB6853F81A
S214451C102210216043F8224070BD2DE9F0410E693F
S214451C20074698460C4601F1140000230568A9B2FC
S214451C3002FB01814FEA114C2D0C02FB05C589B20A
S214451C40013301EB05419E4240F8041B4FEA154817
S214451C50ECDCB8F1000F1BD0A368B34212DC616818
S214451C6038460131FFF78EFF2269023204F10C0136
S214451C70054692000C30FFF777FF21463846FFF7BA
S214451C80B5FF2C4604EB86030136C3F8148026615F
S214451C902046BDE8F0812DE9F8430C4615461F461B
S214451CA009220833064693FBF2F3002101229A42A5
S214451CB020DB3046FFF766FF089B4361092D4FF052
S214451CC00103036119DD04F10909C8462C4418F8D7
S214451CD0013B0146303B0A223046FFF79EFFA045B2
S214451CE0F5D1A5F108044C442D1B6319BB4207DB0F
S214451CF0BDE8F88352000131D9E70A340925F3E7F0
S214451D0014F8013B0146303B0A223046FFF785FF73
S214451D10EBE7020C12040346CAB90304102013F07D
S214451D207F4F04BF1B02083013F0704F04BF1B01E2
S214451D30043013F0404F04BF9B000230002B05DBF8
S214451D4013F0804F00F1010008BF202070470020A7
S214451D50E5E70368024613F007000BD0D90722D4FF
S214451D60980749BF5B089B08012013605CBF13605A
S214451D700220704799B209B91B0C102013F0FF0FCB
S214451D8004BF1B0A0830190704BF1B09043099070E
S214451D9004BF9B080230D90703D45B0800F1010055
S214451DA003D013607047002070472020704710B559
S214451DB00C460121FFF7E6FE01224461026110BD93
S214451DC02DE9F04F15460A692B699A42B8BF0B466E
S214451DD00C46BCBF2C461D462769D5F81090A3680F
S214451DE0616807EB0906B342B8BF013185B0FFF716
S214451DF0C9FE00F1140101EB86080B460022434557
S214451E001DD304F1140305F1140203EB870702EB17
S214451E10890302933B1B153B23F00303043304F16C
S214451E201505AF4238BF04230193029B03929342A4
S214451E3008D8002E5ADC066105B0BDE8F08F43F899
S214451E40042BDCE7B2F800A0BAF1000F24D004F169
S214451E50140E89464FF0000C5EF8045BD9F800B0C6
S214451E60ABB21FFA8BFB0AFB03B34FEA154BD9F807
S214451E70005063444FEA154C0AFB0BC505EB13456A
S214451E809BB243EA0543774549F8043B4FEA154C70
S214451E90E2D8019B41F803C0039BB3F80290043295
S214451EA0B9F1000F20D00B6804F1140C8E464FF0A4
S214451EB0000ABCF80050BEF802B009FB05B5AA44B6
S214451EC09BB243EA0A434EF8043B5CF8043BBEF833
S214451ED000501B0C09FB035303EB1A4367454FEAB7
S214451EE0134AE6D8019D4B5104319EE758F8043D08
S214451EF0002BA0D1013E9CE72DE9F843154612F08C
S214451F00030206460F4607D0214C013A002354F8F3
S214451F102220FFF782FE0746AD1035D0746A3CB9DD
S214451F201020FFF707FEC0E9014470620460C460F4
S214451F30D6F82480D8F808404CB940F2712130468E
S214451F40FFF735FF0023C8F80800044603604FF046
S214451F500009EB070AD5394622463046FFF730FFDB
S214451F60394680463046FFF741FE47466D100BD052
S214451F70206838B9224621463046FFF721FF2060C3
S214451F80C0F800900446E4E73846BDE8F88300BF4D
S214451F90886046002DE9F0470C464968236903EBFF
S214451FA06218A368074691464FEA621A08F1010689
S214451FB0B3423FDB3846FFF7E5FD0023054600F113
S214451FC0140100F110021846534536DB20692AEA0B
S214451FD0EA7A04F1140319F01F0901EB8A0103EBB1
S214451FE0800C2ED0C9F1200E8A460022186800FAC9
S214451FF009F002434AF8042B53F8042B9C4522FA71
S2144520000EF2F3D8ACEB0403153B23F0030304337D
S21445201004F11500604588BF0423CA500AB108F18B
S2144520200206013E38462E612146FFF7DFFD28466B
S214452030BDE8F08701315B00BAE742F8040F01338B
S214452040C2E7043953F8042B41F8042F9C45F9D8C8
S214452050E7E70A6903460069801A30B50DD114339F
S214452060143103EB820401EB820154F8045D51F808
S214452070042D954202D004D3012030BDA342F4D3AB
S214452080FBE74FF0FF30F8E72DE9F84F0C460646DC
S214452090114620461746FFF7DCFF051E08D12946A0
S2144520A03046FFF76FFD0123C0E90435BDE8F88FDC
S2144520B0A4BF3B46274630467968A6BF1C46002542
S2144520C00125FFF75FFD3E69C560256907F11401E7
S2144520D004F1140900F1140E07F1100201EB860C09
S2144520E009EB8505F246002759F8043B52F804BF2C
S2144520F01FFA83F817FA8BF71B0CA7EB0808C3EBF8
S2144521001B4303EB28431FFA88F81F144D4548EA3E
S21445211003434AF8043BE7D82B1B153B23F0030340
S21445212004331534A54238BF0423194473449E46E8
S2144521300D4665450ED30CF10302521A22F00302F2
S21445214003398C4538BF00221A4452F8043D7BB10A
S2144521500661ABE755F8048B17FA88F4221402EBB0
S2144521601842A4B244EA02444EF8044B1714E0E77A
S214452170013EEAE7114B0B40A3F15073002B02DDFD
S2144521800020194670475B42B3F1A07F4FEA2352C1
S2144521904FF000004FF0000104DA4FF4002343FAF5
S2144521A002F17047A2F114031E2BDABF4FF000422E
S2144521B022FA03F301231846704700BF0000F07F5C
S2144521C02DE9F843076900F1140909EB8707A7F1DC
S2144521D0040857F8046C3046FFF79BFDC0F1200312
S2144521E00A280B601F4917DCC0F10B0CC14526FABF
S2144521F00CF338BF57F8082C43EA010528BF0022E0
S21445220000F1150306FA03F322FA0CF243EA020438
S21445221020462946BDE8F883C1453ABF57F8082CFD
S214452220A7F108080022B0F10B0316D0C3F120072A
S21445223022FA07F1C84506FA03F646EA01068CBFB8
S21445224058F8041C002146F07F5502FA03F0F94081
S21445225045F4401540EA0104DAE746EA0105144626
S214452260D6E700BF0000F03F2DE9F34101211C46AB
S214452270DDE908659046FFF785FCC4F31303C4F310
S2144522800A5407462CBB0193B8F1000326D068468E
S2144522900093FFF75EFD0099F0B1019AC0F1200367
S2144522A002FA03F30B43C2407B610192019BBB617B
S2144522B0002B14BF022101213961C4B1A4F2334475
S2144522C00444C0F1350034602860384602B0BDE8A5
S2144522D0F08143F48013D6E77961E7E701A8FFF775
S2144522E038FD019B7B61012139612030E5E707EB2D
S2144522F08103A0F2324030601869FFF70AFDC0EB53
S21445230041112960E1E72DE9F74F88466946814640
S214452310FFF756FF0F4604460D46404601A9FFF710
S2144523204FFFD9F81030D8F81020A3EB020CDDE9A2
S21445233000329B1A03EB4C13002BD5BF0A462A46A0
S214452340C3EB033302EB03578B46D8BF02EB035B65
S2144523505B46024639462046FBF708FE03B0BDE815
S214452360F08F013970B549111469013102F1140332
S21445237000EB810103EB8404051FA3420CD3A31A8B
S214452380113B23F003031132A24288BF00231844B1
S2144523900023884205D370BD53F8046B45F8046F97
S2144523A0EBE740F8043BF4E700F1140200694B11F3
S2144523B0984210B511DB0ADD11F01F0107D052F81F
S2144523C0234024FA01F000FA01F18C420BD102EBCE
S2144523D08303934203D8002010BD0346F7E753F81E
S2144523E0041D0029F5D00120F6E738B502FB01F5B6
S2144523F0294600F057F8044618B12A46002100F051
S21445240056FA204638BD000038B50546002945D061
S21445241051F8043C0C1F002BB8BFE41800F04FFAE7
S2144524201F4A1368104633B9636014602846BDE8F2
S214452430384000F045BAA3420BD92168621893424A
S21445244004BF1A685B68636004BF52182260046064
S214452450ECE71A465B680BB1A342FAD911685018E7
S214452460A0420BD120680144501883421160DDD14B
S21445247018685B68536001441160D7E702D90C239E
S2144524802B60D3E7206821188B4204BF19685B6828
S214452490636004BF091821605460C7E738BD00BFB4
S2144524A0F4FE4120F8B5CD1C25F0030508350C2D66
S2144524B038BF0C25002D064601DBA94203D90C235F
S2144524C033600020F8BD00F0FAF921490A68144641
S2144524D09CB9204F3B6823B92146304600F098F911
S2144524E038602946304600F093F9431C23D10C2327
S2144524F03360304600F0E4F9E3E723685B1B17D406
S2144525000B2B03D923601C44256004E06368A24274
S2144525100CBF0B605360304600F0D2F904F10B0057
S214452520231D20F00700C21ACCD01B1AA350C9E7BA
S21445253022466468CCE7C41C24F00304A042E3D0DA
S214452540211A304600F064F90130DDD1CFE700BFEF
S214452550F4FE4120F8FE41202DE9F0478E689E4264
S21445256082460C4690461F4638D88A8912F4906FA4
S21445257032D025680969A5EB0109656905EB45056E
S21445258005EBD57501334B446D109D4238BF1D464E
S214452590530531D52946FFF785FF064650B90C2326
S2144525A0CAF80030A38943F04003A3814FF0FF30BB
S2144525B0BDE8F08721694A46FFF7D6FAA38923F492
S2144525C0906343F08003A381266165614E44A5EB85
S2144525D009052660A5603E46BE4200D93E463246BF
S2144525E02068414600F049F9A36822689B1B32449F
S2144525F0A36022600020DBE72A4600F062F9064623
S2144526000028E1D121695046FFF7FEFEC7E70000E6
S2144526102DE9F04F98468B891B069DB007460D461B
S21445262014460ED50B6963B94021FFF73BFF28607A
S214452630286120B90C233B604FF0FF30D1E04023A2
S2144526406B610023099320238DF82930CDF80C8043
S2144526503023DFF8A8818DF82A304FF0010923464C
S2144526609A4613F8012B0AB1252AF9D1BAEB040B81
S2144526700BD05B46224629463846FFF76DFF0130AC
S21445268000F0AA80099A5A4409929AF80030002B1D
S21445269000F0A28000234FF0FF32CDE905230AF172
S2144526A0010A049307938DF853301A93544605222E
S2144526B014F8011B5148FBF723F9049AD8B9D006FC
S2144526C044BF20238DF85330110744BF2B238DF884
S2144526D053309AF800302A2B15D0079A54460020D6
S2144526E04FF00A0C214611F8013B303B092B4ED9D9
S2144526F0B0B1079214E0A0EB080309FA03F31343BD
S2144527000493A246D2E7039B191D1B680391002B31
S214452710BBBF5B4242F0020207930793B8BF0492E1
S21445272023782E2B0CD163782A2B35D1039B1A1D83
S2144527301B680392002BB8BF4FF0FF330234059356
S214452740DFF8C8A0217803225046FBF7D9F840B1F8
S2144527504023A0EB0A0003FA00F0049B0343013430
S214452760049314F8011B26488DF828100622FBF71B
S214452770C7F8002838D0234B1BBB039B073323F0F1
S214452780070308330393099B3344099367E70CFB18
S21445279002320C460120A5E700230134059319466D
S2144527A04FF00A0C204610F8012B303A092A03D977
S2144527B0002BC5D00591C3E70CFB01210446012338
S2144527C0F0E703AB00932A460F4B04A93846FCF7BF
S2144527D057FB421C0646D6D1AB895B063FF52CAF68
S2144527E009981DB0BDE8F08F03AB00932A46064B0B
S2144527F004A93846FCF7DCFDEBE700BF94604600CD
S2144528009E60460081EE4400592545009A60460084
S21445281038B5064D0023044608462B6000F0C8F838
S214452820431C02D12B6803B1236038BDFCFE412012
S21445283001490020704700BF0000F87F10B56AB117
S2144528400139841810F8013B11F8012F934203D142
S214452850A04201D0002BF5D1981A10BD1046FCE7D2
